:100000000C94B7210C94E8210C94E8210C94E8217D
:100010000C94E8210C94E8210C94E8210C94E8213C
:100020000C94E8210C94E8210C94E8210C94E8212C
:100030000C94E8210D9411410C94E8210C94E821D2
:100040000C94E8210C9452DD0C94E8210C94E821E6
:100050000C94E8210C94E8210C945BDA0D94C740D1
:100060000C94E8210C94494C0C943F4C0C94E821DE
:100070000C94E8210C94E8210C94E8210C94E821DC
:100080000C94E8210C94E8210C94E8210C94E821CC
:100090000C94E8210C94E8210C94E8210C94E821BC
:1000A0000C94E8210C94E8210C94E8210C94E821AC
:1000B0000C94E8210C94E8210C94E8210C94E8219C
:1000C0000C94E8210C94E8210C94E8210C94E8218C
:1000D0000C94E8210C94E8210C94E8210C94E8217C
:1000E0000C94E821084AD73B3BCE016E84BCBFFD8F
:1000F000C12F3D6C74319ABD56833DDA3D00C77FF8
:1001000011BED9E4BB4C3E916BAAAABE0000008090
:100110003F05A84CCDB2D44EB93836A9020C50B91F
:10012000918688083CA6AAAA2ABE000000803F004B
:100130000D94D3390C94EE7C0C9452C10C9485220E
:100140000D94213B0C94FA840C9452A20C94FB7AEB
:100150000D94083B0C94E74C0C94D4880C94D44C2C
:100160000C947E830C94C5880C94C9AB0C948A8340
:100170000C94BC870C946CB30C94D5780C947B7C59
:100180000C94DE880D94493A0D945A3A0C94273316
:100190000D94964C0C941EB00C94D9840C94EBB630
:1001A0000C94D8870C9472B30C94757B0C94828356
:1001B0000C94B3CB0C94C57E0C947B7E0C948E83F4
:1001C0000C94EA7C0D94FE3A0C944EB30C9437C018
:1001D0000C94E1B60C9496B30C9476830C94DFC720
:1001E0000D94353B0C9452910C94C0840C94C27CB9
:1001F0000C94DE800C94577D0D94103A0C948683F9
:100200000C94277B0C94E3780C9488800C946C8677
:100210000C94C54C0C94C4870C94B0A80C94CE8854
:100220000C9496830C9447CD0C94C7CC0C94D09E20
:100230000C949D7B0C946D220C9458380C94DF4CDC
:100240000D94CD390C948A7D0C94697D0D94D03A2F
:100250000C945F9D0C94874C0C94F97B0C94B6879E
:100260000C94EC7C0D94DA3A0D94C5390D94E53973
:100270000C94CB7B0C9460B30D946A3A0C94CB88AD
:100280000D94753A0C946C7D0D94493B0C94A57AB1
:100290000C94E6B60D94BB390C94EB4C0D94D73905
:1002A0000C9449780C94ED210C94DA800C94817DA7
:1002B0000C9478B70C94B6780C94027D0C94B79596
:1002C0000C94B64C0C9477780C94FA4C0D942F192E
:1002D0000C94EF4C0C94C8880D94F43A0C94F38B66
:1002E0000D94E23A0C9428C10C9475840C94E27B32
:1002F0000C945DC70D94603A0C94627B0C94D37E91
:100300000D94A6390C94C88D0C948C7A0C94E0C78B
:100310000C946C780C94CF7A0C948E7B0D94B53938
:100320000C941B850C947EB30D94DB390C944A9B82
:100330000C9478B30C942CCD0D94AA390C94C97EEE
:100340000C94D1880C9437890D948F390C94B47A1D
:100350000C9410230C943E9A0C944FCC0C94B2B78E
:100360000C94FD7C0C943A7D0C9465850C94F4936C
:100370000C94E8CC0C9436900C94E87A0C9498AADF
:100380000C940D4D0C94E99B0C94D4970C9448A2BA
:100390000D94EA3A0C94F87C0C94CB7E0C9455891D
:1003A0000C9441840C9432CC0C94CD7E0C94398402
:1003B0000C94E4840C94BF880C94829C0C94B1A59A
:1003C0000D94B2390C9403B70C94CB7C0C94BC7E86
:1003D0000C94C2880C94B47B0C94D6800C94F021BD
:1003E0000D942B3B0C9472830C942A7E0C945E9992
:1003F0000C94A7840C943A890C94437F0D94B73ADB
:100400000C9497B40C94D7CD0D94C63A0C94A0B329
:100410000C947C800C94AB850C9437230C94A6A090
:100420000C94D38E0C94054D0D94BC3A0D943F3B27
:100430000C940E7B0D945C190C94D77C0C94EA21DF
:100440000C94B49A0C94CF7E0C9429840D947E194C
:100450000C94667D0C948E840C94B4880C94DB4CC4
:100460000D94E1390C94E34C0C94E1880C94737A6C
:100470000C944F7B0C94A9C00C945AB30C9484B385
:100480000D94173B0C9433C90C946F7D0C94DB884E
:100490000C94D9880C94CD870C94C5CD0D94C93992
:1004A0000C948AB30C94F34C0D94AE390C94DFA3E6
:1004B0000C9490B30C94CF780D94F5390C94407B48
:1004C0000C9404CE0C94AE220C9454B30C94CECE67
:1004D0000C94C77E0C9456C00C946C7E0C9466B33E
:1004E0000C94867D0C944E850D944E3A0C94F37CBE
:1004F0000C9461BB0C947A830C944E810D94E94C5E
:100500000C94D17E0C9409C10D9494390C94DCB6F2
:100510000D94074D0D94AF3A0D94BF390C9492830E
:100520000C94C8C04E414E494E495459494E46CD8F
:10053000CCCC3D0AD7233C17B7D13877CC2B32959A
:1005400095E6241FB14F0A000020410000C8420078
:10055000401C4620BCBE4CCA1B0E5AAEC59D740042
:10056000407A10F35A00A0724E18090010A5D4E882
:100570000000E87648170000E40B54020000CA9A15
:100580003B000000E1F50500008096980000004067
:10059000420F000000A086010000001027000000AC
:1005A00000E803000000006400000000000A0000F2
:1005B0000000000100000000002C76D888DC674FA6
:1005C0000823DFC1DFAE59E1B1B796E5E3E453C6D6
:1005D0003AE651997696E8E6C28426EB898C9B62CE
:1005E000ED407C6FFCEFBC9C9F40F2BAA56FA5F478
:1005F00090055A2AF75C936B6CF9676DC11BFCE0A0
:10060000E40D47FEF520E6B500D0ED902E030094F2
:100610003577050080841E080000204E0A00000087
:10062000C80C333333330F986E12831141EF8D2191
:1006300014893BE65516CFFEE6DB18D1844B381BF8
:10064000F77C1D901DA4BBE424203284725E2281BD
:1006500000C9F124ECA1E53D27434F4D4D554E49CE
:10066000434154494F4E0044525952554E00455251
:10067000524F525300494E464F004543484F0045A4
:1006800072726F722077726974696E6720746F205E
:10069000454550524F4D210A0053544F5050454448
:1006A0002E20005072696E7465722073746F7070C2
:1006B00065642064756520746F206572726F727353
:1006C0002E2046697820746865206572726F7220EA
:1006D000616E6420757365204D39393920746F203F
:1006E000726573746172742E202854656D70657222
:1006F00061747572652069732072657365742E204C
:100700005365742069742061667465722072657324
:1007100074617274696E67290A004E6F20436865C0
:10072000636B73756D2077697468206C696E6520E2
:100730006E756D6265722C204C617374204C696E0D
:10074000653A20004E6F20436865636B73756D20BA
:1007500077697468206C696E65206E756D6265726C
:100760002C204C617374204C696E653A20006368DC
:1007700065636B73756D206D69736D617463682C4F
:10078000204C617374204C696E653A20004C696E90
:1007900065204E756D626572206973206E6F7420DE
:1007A0004C617374204C696E65204E756D62657284
:1007B0002B312C204C617374204C696E653A2000FB
:1007C0004D3131300053657269616C20737461740E
:1007D0007573206D69736D617463680A0077616970
:1007E000740A0053442072656164206572726F72EE
:1007F0000A00486F74656E642049646C6520546912
:100800006D656F757400486F74656E642049646C23
:10081000652054696D656F75740A002121204B496C
:100820004C4C20636175736564206279204B494CA0
:100830004C20627574746F6E2F70696E0A002121EE
:10084000204B494C4C2063617573656420627920AC
:10085000746F6F206D75636820696E61637469766B
:10086000652074696D65202D2063757272656E74E4
:1008700020636F6D6D616E643A2000706175736501
:10088000004D363030002066696C616D656E745FB6
:1008900072756E6F7574200066696C616D656E743B
:1008A0005F72756E6F757420540046696C616D657A
:1008B0006E7452756E6F75742054004D6564696175
:1008C0002052656D6F766564004D656469612049ED
:1008D0006E736572746564004D3130303053006260
:1008E0007573793A2070617573656420666F722044
:1008F000696E7075740A00627573793A207061755B
:1009000073656420666F7220757365720A00627584
:1009100073793A2070726F63657373696E670A004A
:10092000506C65617365205265736574005052495F
:100930004E5445522048414C5445440025533A20DA
:10094000255300706F7765726F6666004B494C4C9B
:1009500045442E20005072696E7465722068616C87
:100960007465642E206B696C6C28292063616C6C43
:100970006564210A006563686F3A004572726F72A0
:100980003A000A4D6561737572656420706F696E17
:1009900074733A0A00357835206D6573682E205AD5
:1009A000206F66667365743A20005072696E7469D0
:1009B0006E67204F626A65637400255320256900C5
:1009C0002F2F616374696F6E3A00737461727400E3
:1009D00070726F6D70745F00656E6400486F74654F
:1009E0006E6420746F6F20636F6C640A0053656ED1
:1009F00064204D31303820746F20726573756D65D9
:100A00000A00496E736572742066696C616D656E6B
:100A10007420616E642073656E64204D3130380A35
:100A20000052656865617420446F6E6500526568A8
:100A3000656174696E672E2E2E005265686561745B
:100A4000004865617465722054696D656F75740046
:100A500053656E64204D31303820746F20686561B5
:100A600074206E6F7A7A6C650A004E6F7A7A6C65C4
:100A7000205061726B65640070617573656400502D
:100A80006175736500726573756D65640052657399
:100A9000756D696E67004732362043616E63656C21
:100AA0006564004732362048656174696E67204E80
:100AB0006F7A7A6C65004732362048656174696EDA
:100AC00067204265640057616974696E6720666FCC
:100AD00072206865617475702E0A004669786564D5
:100AE000204C656E677468205072696D6500446FB4
:100AF0006E65205072696D696E67004D616E75613B
:100B00006C207072696D696E672E2E2E004C6561C7
:100B100076696E6720473236003F537065636966B9
:100B200069656420582C5920636F6F7264696E6127
:100B30007465206F7574206F6620626F756E6473C4
:100B40002E0A003F28522965706561742076616C19
:100B50007565206E6F7420706C61757369626C6569
:100B60003B206D757374206265206174206C656133
:100B7000737420312E0A003F53706563696669659E
:100B800064206E6F7A7A6C652074656D7065726131
:100B900074757265206E6F7420706C617573696214
:100BA0006C652E0A003F5370656369666965642051
:100BB00066696C616D656E742073697A65206E6F0D
:100BC0007420706C61757369626C652E0A003F5306
:100BD0007065636966696564207072696D65206C13
:100BE000656E677468206E6F7420706C61757369D0
:100BF000626C652E0A003F537065636966696564BF
:100C0000206E6F7A7A6C652073697A65206E6F74D6
:100C100020706C61757369626C652E0A003F5265C5
:100C20007472616374696F6E204D756C7469706C59
:100C3000696572206D7573742062652073706563D9
:100C400069666965642E0A003F5370656369666969
:100C500065642052657472616374696F6E204D75AE
:100C60006C7469706C696572206E6F7420706C6151
:100C7000757369626C652E0A003F5370656369661F
:100C8000696564206C61796572206865696768745C
:100C9000206E6F7420706C61757369626C652E0ACA
:100CA0000043292E0A003F537065636966696564D5
:100CB000206265642074656D70657261747572651B
:100CC000206E6F7420706C61757369626C6520288A
:100CD00034302D00473236207374617274696E6748
:100CE0002E2E2E0A004F46460A00466164652048B3
:100CF00065696768742000426564204C6576656CA0
:100D0000696E6720004661696C656420746F2065B8
:100D10006E61626C6520426564204C6576656C6925
:100D20006E670A004D65736820426564204C6576E5
:100D3000656C20646174613A0A00496E76616C6981
:100D400064206D6573682E0A00206E6F7420656ED6
:100D500074657265642E0A0050726F62696E672056
:100D6000506F696E740025532025692F2569002076
:100D70006F6620004D424C2047323920706F696EFB
:100D8000742000290A004A206F7574206F66207253
:100D9000616E67652028302D00290A0049206F7593
:100DA00074206F662072616E67652028302D0047C1
:100DB00032384C30004D6573682070726F62696E16
:100DC0006720646F6E65004D6573682070726F6296
:100DD000696E6720646F6E652E0A005374617274C9
:100DE000206D6573682070726F62696E6720776925
:100DF0007468202247323920533122206669727389
:100E0000742E0A004732395332004732384C300AC8
:100E1000473239533200686173206E6F2064617409
:100E2000612E0A004D65736820426564204C65762A
:100E3000656C696E67200053206F7574206F6620A3
:100E400072616E67652028302D35292E0A004D65A8
:100E5000736820706F696E74206F7574206F6620E0
:100E600072616E67650A004D34323120696E636FBE
:100E7000727265637420706172616D657465722051
:100E800075736167650A005741524E494E472120EC
:100E90004C6F77205A204A65726B206D6179206C07
:100EA00065616420746F20756E77616E746564206F
:100EB0007061757365732E0A004F4646004F4E00F1
:100EC00020204D61783A2000200020204D696E3AA4
:100ED0002000536F667420656E6473746F70733A8C
:100EE00020004D32342053256C642054256C64005E
:100EF0004739322E39204525730047312046256475
:100F0000004739322E39205A2573004731205A3094
:100F10002046323030004731205825732059257340
:100F2000204633303030004D343230205325692094
:100F30005A2573004D3130362050256920532569DC
:100F4000004D32303020442573004732385230583B
:100F500059004739322E39204530205A300A47315E
:100F60005A2573004D31303920532569004D3139F0
:100F70003020532569004D343230205330205A3010
:100F80000020496E76616C696420657874727564BE
:100F90006572200047322F47332062616420706100
:100FA00072616D65746572730A00536C6565702EAD
:100FB0002E2E004D65736820706F696E74206F75FA
:100FC00074206F662072616E67650A004D30205391
:100FD000746F70004D312053746F7000436C6963FF
:100FE0006B20746F20526573756D652E2E2E004E2A
:100FF0006F204D6F76652E00456E642066696C65C6
:10100000206C6973740A00426567696E2066696CBA
:1010100065206C6973740A004E6F206D65646961A8
:101020000A00526573756D696E6720534400286E1F
:101030006F2066696C65290043757272656E742055
:1010400066696C653A20005072696E742074696D2F
:10105000653A20000A53746174733A2046696C61E2
:101060006D656E7420757365643A20002C204C6F9A
:101070006E67657374206A6F623A2000546F746102
:101080006C2074696D653A200053746174733A2062
:10109000002C204661696C65643A20002C2046696A
:1010A0006E69736865643A20005072696E74733AB1
:1010B000200053746174733A2000436F6F6C696E43
:1010C000672E2E2E0048656174696E672E2E2E00E5
:1010D00045202553006F6B006F6666007A06750623
:1010E0006E066706590644454255473A004D313170
:1010F0003320530042656420436F6F6C696E672E26
:101100002E2E004265642048656174696E672E2E3C
:101110002E0050533A300A0050533A310A00544DD1
:1011200033442032303230204F46462E002F2F00DD
:101130004D31343520533C696E6465783E206F75BF
:1011400074206F662072616E67652028302D31290A
:101150000A00205200416363656C65726174696FB7
:101160006E3A2050004D32303620580046523A0038
:1011700020466C6F773A20004D424C2041646A75DE
:101180007374205A0020643A0020693A0020703AB3
:1011900000496E76616C6964206578747275646567
:1011A000720A0020643A0020693A0020703A004C2C
:1011B000434420436F6E74726173743A2000646913
:1011C0007300656E0043290A0061626C6564202823
:1011D0006D696E2074656D702000436F6C642065CE
:1011E0007874727564657320617265200046696C5D
:1011F000616D656E742072756E6F757420646973AD
:1012000074616E636520286D6D293A200046696C13
:10121000616D656E742072756E6F757420004F6617
:101220006673657473204170706C69656400457203
:10123000723A20546F6F206661722100546F6F20E4
:101240006661722066726F6D207265666572656E8A
:10125000636520706F696E740A00454550524F4DAA
:10126000204F4B0A002E0A002028302D3130290053
:101270002076616C7565206F7574206F66207261D1
:101280006E676500416476616E6365204B3D004F7B
:101290004E0A004F46460A0043617365206C696739
:1012A00068743A2000506F7765722D6C6F737320ED
:1012B0007265636F7665727920004D383400446F33
:1012C0006E65207072696E74696E672066696C6500
:1012D0000A004D3737004D3331004361703A004DFD
:1012E0004541545041434B00434F4F4C45525F548E
:1012F000454D5045524154555245004348414D4299
:1013000045525F54454D5045524154555245004257
:101310004142595354455050494E4700415243535E
:10132000004D4F54494F4E5F4D4F44455300544874
:1013300045524D414C5F50524F54454354494F4ED6
:10134000004C4F4E475F46494C454E414D4500418C
:1013500055544F5245504F52545F53445F5354417C
:101360005455530053445F57524954450052455019
:10137000454154005344434152440050524F4D5054
:10138000545F535550504F525400454D45524745B8
:101390004E43595F50415253455200434153455FBC
:1013A0004C494748545F4252494748544E4553536D
:1013B00000544F47474C455F4C49474854530053EE
:1013C0004F4654574152455F504F57455200425582
:1013D000494C445F50455243454E54004C45564598
:1013E0004C494E475F44415441005A5F50524F426E
:1013F000450052554E4F5554004155544F4C45569B
:10140000454C005052494E545F4A4F420050524F93
:101410004752455353004155544F5245504F525433
:101420005F54454D5000564F4C554D45545249431D
:1014300000454550524F4D0042494E4152595F467A
:10144000494C455F5452414E534645520053455214
:1014500049414C5F584F4E5F584F464600464952EF
:101460004D574152455F4E414D453A4D61726C6951
:101470006E20322E302E375F4457372E3320544D96
:101480003344203230534D444E4E20284170722058
:10149000323420323032312032303A30383A323938
:1014A0002920534F555243455F434F44455F5552A2
:1014B0004C3A68747470733A2F2F67697468756258
:1014C0002E636F6D2F496E73616E69747941757407
:1014D0006F6D6174696F6E2F4D61726C696E2F74E0
:1014E0007265652F437265616C6974794477696EC2
:1014F0005F322E302050524F544F434F4C5F564571
:101500005253494F4E3A312E30204D414348494EB7
:10151000455F545950453A544D33442032303230AF
:101520002045585452554445525F434F554E543A06
:101530003120555549443A63656465326132662D00
:10154000343161322D343734382D396231322D63E4
:1015500035356336326633363766660A0043616E68
:101560006E6F74206F70656E20737562646972208F
:10157000002569730025696D202569730025696858
:101580002025696D20256973002569642025696817
:101590002025696D202569730025697920256964F6
:1015A000202569682025696D2025697300236465FD
:1015B00066696E652044454641554C545F0062653E
:1015C00064004B6420004B6920004B7020005049A0
:1015D00044204175746F74756E652066696E697319
:1015E000686564212050757420746865206C61738F
:1015F00074204B702C204B6920616E64204B64205A
:10160000636F6E7374616E74732066726F6D2062A7
:10161000656C6F7720696E746F20436F6E666967C3
:1016200075726174696F6E2E680A005049442041DA
:1016300075746F74756E65206661696C65642120D0
:1016400074696D656F75740A005049442041757462
:101650006F74756E65206661696C656421205465E0
:101660006D706572617475726520746F6F20686942
:1016700067680A00204B643A2000204B693A20003A
:10168000204B703A200020436C61737369632050D3
:101690004944200A00204E6F206F76657273686F90
:1016A0006F740A002054753A2000204B753A2000D0
:1016B000206D61783A2000206D696E3A2000206428
:1016C0003A200020626961733A2000504944204169
:1016D00075746F74756E652073746172740A00504E
:1016E0004944204175746F74756E65206661696C3C
:1016F0006564212054656D70657261747572652032
:10170000746F6F20686967680A005049442041750A
:10171000746F74756E6500504944204175746F7420
:10172000756E65206661696C656421204261642084
:101730006865617465722069640A004572723A20B6
:101740007574663820666F6E74206E6F7420696ED3
:10175000697469616C697A65642E004572723A2019
:101760007574663820666F6E74206E6F7420696EB3
:10177000697469616C697A65642E004572723A20F9
:101780007574663820666F6E74206E6F7420696E93
:10179000697469616C697A65642E00FFE0FFD1406D
:1017A000A0C8A6A22FF80023AC00AF10FFFEFF05D3
:1017B000FFD0FFE0FFC1FFD1E240A0C8A6A22FF8F2
:1017C00000238127AC00AFFFD0FF64FFD1A5FFD07D
:1017D000FF64FF64FFD1A4FFD0FF16FFFE000C0FD3
:1017E00000FE07022503BB017FFE08FE08FE050878
:1017F0000806000040F0C888889878100508080698
:101800000000C0F88888888888F80505050600016A
:101810002030F830200508080600002070F820204D
:101820002020E00509090600FF2070A8A8B88888D4
:101830007020070505070001D86C366CD80509092A
:101840000600FFF8A88888888888A8F8050A0A068C
:1018500000FE205050505088A8A88870030303064B
:10186000000340A040FFFFFFFFFFFFFFFFFFFFFF60
:10187000FFFFFFFFFFFFFFFFFFFFFF000000060568
:10188000FF0107070602008080808080008003033C
:1018900003060105A0A0A005060606000050F850AA
:1018A00050F8500509090600FF2070A8A07028A86C
:1018B0007020050707060000C8C81020409898054A
:1018C000070706000040A0A040A890680103030697
:1018D00002058080800309090601FF2040408080C6
:1018E000804040200309090601FF8040402020205D
:1018F00040408005070706000020A8702070A8203F
:101900000505050600012020F8202002030306013A
:10191000FFC04080050101060003F8020202060133
:1019200000C0C005070706000008101020404080D6
:10193000050707060000708898A8C8887003070785
:1019400006010040C040404040E005070706000097
:10195000708808102040F8050707060000F80810F6
:101960003008887005070706000010305090F81006
:1019700010050707060000F880F0080888700507C2
:1019800007060000304080F08888700507070600D1
:1019900000F80810102020200507070600007088B6
:1019A00088708888700507070600007088887808A6
:1019B0001060020505060100C0C000C0C002060696
:1019C0000601FFC0C000C0408003050506010120DC
:1019D00040804020050303060002F800F8030505D7
:1019E000060101804020408005070706000070883E
:1019F00010202000200507070600007088B8A8B84E
:101A00008070050707060000708888F888888805B8
:101A10000707060000F04848704848F00507070629
:101A2000000070888080808870050707060000F03D
:101A30004848484848F0050707060000F88080F04D
:101A40008080F8050707060000F88080F08080801D
:101A500005070706000070888080988870050707D2
:101A6000060000888888F888888803070706010030
:101A7000E04040404040E0050707060000381010F5
:101A8000101090600507070600008890A0C0A09085
:101A900088050707060000808080808080F80507A1
:101AA0000706000088D8A8888888880507070600E8
:101AB000008888C8A89888880507070600007088ED
:101AC0008888888870050707060000F08888F080FD
:101AD000808005070706000070888888A890680540
:101AE0000707060000F08888F0A090880507070621
:101AF000000070888070088870050707060000F8ED
:101B000020202020202005070706000088888888DC
:101B1000888870050707060000888888885050204C
:101B200005070706000088888888A8A850050707C9
:101B300006000088885020508888050707060000A6
:101B400088885020202020050707060000F808108C
:101B5000204080F80309090601FFE0808080808032
:101B60008080E00507070600008040402010100834
:101B70000309090601FFE020202020202020E005A5
:101B800003030600052050880501010600FEF80346
:101B900003030601058040200505050600007008C6
:101BA0007888780507070600008080F0888888F02C
:101BB000050505060000708080887005070706008F
:101BC0000008087888888878050505060000708870
:101BD000F08070050707060000304840E0404040B4
:101BE0000507070600FE70888888780870050707D3
:101BF0000600008080F088888888030707060100B7
:101C00004000C0404040E00409090601FE100030D9
:101C10001010101090600507070600008080889063
:101C2000E09088030707060100C04040404040E0C4
:101C3000050505060000D0A8A8A8A805050506000A
:101C400000B0C88888880505050600007088888867
:101C5000700507070600FEF0888888F08080050779
:101C6000070600FE788888887808080505050600BC
:101C700000B0C880808005050506000078807008E7
:101C8000F00507070600002020F820202018050591
:101C90000506000088888898680505050600008804
:101CA000888850200505050600008888A8A85005EA
:101CB000050506000088502050880507070600FE2D
:101CC00088888850204080050505060000F810200F
:101CD00040F80309090601FF204040408040404091
:101CE000200109090602FF8080808080808080803A
:101CF0000309090601FF8040404020404040800524
:101D0000030306000248A890FF554E4C4F41442063
:101D100046494C414D454E54004C4F4144204649A4
:101D20004C414D454E540046494C414D454E542082
:101D30004348414E47450042656400456E636C6F01
:101D400073757265002568753A253032687500250F
:101D5000303268753A253032687500202020202006
:101D600020200020202020001FE020102010201024
:101D70001020102020102010303008400480030074
:101D80001FE03FF03FF03FF01FE01FE03FF03FF06B
:101D90003FF00FC0078003003FFFF038007030FCB9
:101DA0003020FC102078102030102C00D02E31D0A4
:101DB0002F7BD02F7BD02E31D02C00D02030102084
:101DC000781020FC1030FC303800703FFFF03FFFEF
:101DD000F03800703186302387102787902F87D006
:101DE0002F03D02030102078102078102030102FB2
:101DF00003D02F87D0278790238710318630380073
:101E0000703FFFF01FFFF81FFFF80410400208208A
:101E100002082004104008208010410010410008F2
:101E200020800410400000001FFFF81FFFF8FFFF94
:101E3000FF8000018E00E19F01F19381399F81F9BC
:101E40009F81F99FB9F98F28F18038018000019FA7
:101E5000FFF99174999B06A99B54A99B56A99B5481
:101E6000999FFFF9FFFFFF6E6F7469666963617484
:101E7000696F6E200063616E63656C005072696EFD
:101E8000742041626F72746564004469736D697394
:101E9000730055492041626F72746564004D32359C
:101EA00020500A4D323400526573756D65005549F6
:101EB0002050617573650050617573696E672E2ED1
:101EC0002E00726573756D65004D32340052756E6B
:101ED0006F75742044697374206D6D004C6F61647C
:101EE000206D6D00556E6C6F6164206D6D004669EC
:101EF0006C2E204469612E004520696E206D6D5E58
:101F00003300416476616E6365204B004D3330339E
:101F1000205531204525692053256900504944202A
:101F20004175746F74756E65202A005049442D44C4
:101F3000202A005049442D49202A005049442D5060
:101F4000202A0020082046616374002008204D618B
:101F500078002008204D696E004F6666004F6E00C5
:101F60004175746F74656D70005654726176204DC2
:101F7000696E00566D696E00566D61782045005699
:101F80006D6178205A00566D6178205900566D6158
:101F900078205800416D6178204500416D617820BE
:101FA0005A00416D6178205900416D6178205800D8
:101FB000412D54726176656C00412D5265747261D9
:101FC000637400416363656C0056652D4A65726BEE
:101FD00000565A2D4A65726B0056592D4A65726B30
:101FE0000056582D4A65726B0045207374657073F6
:101FF0002F6D6D005A2053746570732F6D6D0059ED
:102000002053746570732F6D6D0058205374657084
:10201000732F6D6D00416476616E63656420536556
:102020007474696E6773003F0043616E63656C0092
:10203000496E6974004D34323800496E69746961C3
:102040006C697A6520454550524F4D0046696C6178
:102050006D656E740054656D70657261747572653E
:102060000053746570732F6D6D004A65726B00418B
:102070006363656C65726174696F6E0056656C6F41
:10208000636974790053657420486F6D65204F66ED
:10209000667365747300436F6E6669677572617409
:1020A000696F6E003F004E65787420506F696E74E2
:1020B00000446F6E65004E657874004C6576656C03
:1020C000696E6720446F6E6521004D6F7665205AFA
:1020D000004732395332004E65787420506F696E74
:1020E00074002569202F20257500473239533100AF
:1020F000473239533200436C69636B20746F20425E
:102100006567696E00486F6D696E672058595A009F
:102110005A2056616C756500496E646578205900D7
:10212000496E64657820580053746F72652053655A
:102130007474696E6773004C6F61642053657474C6
:10214000696E6773004C6576656C20436F726E65CF
:10215000727300426564205A0046616465204865D8
:1021600069676874004F6666004F6E0042656420C0
:102170004C6576656C696E670045646974204D65D1
:102180007368004C6576656C20426564004D6F7421
:10219000696F6E003F0043616E63656C204F626A39
:1021A000656374004E4F005945530043616E63658B
:1021B0006C204F626A656374203D004D61696E005A
:1021C000426564004E6F7A7A6C650046616E2053FA
:1021D0007065656400436F6E6669677572617469E6
:1021E0006F6E00526573746F726520446566617529
:1021F0006C7473004C6F61642053657474696E670E
:10220000730053746F72652053657474696E6773DD
:102210000050726568656174202420436F6E66000B
:10222000506F776572204F7574616765004F666601
:10223000004F6E0052756E6F75742053656E736F2C
:1022400072004C434420436F6E747261737400419A
:102250006476616E6365642053657474696E677338
:10226000004D61696E004D37303220542564004DB9
:1022700036303020423020542564004D3730322033
:102280003B2564004D37303120542564004D3730F4
:1022900032004D373031004D363030204230004D65
:1022A00061696E00436F6E74696E7565004F666696
:1022B000004F6E0052756E6F75742053656E736FAC
:1022C00072005075726765206D6F726500524553DC
:1022D000554D45204F5054494F4E533A00505249A6
:1022E0004E54205041555345440020204E6F7A7A79
:1022F0006C653A20005061726B696E672E2E2E005D
:1023000000005761697420666F720066696C616DC8
:10231000656E74206368616E676500746F20737406
:10232000617274005761697420666F720066696C2F
:10233000616D656E7420756E6C6F616400004E6F28
:102340007A7A6C652068656174696E6700506C65A7
:1023500061736520776169742E2E2E0000507265BE
:10236000737320627574746F6E00746F206865619A
:1023700074206E6F7A7A6C650000496E73657274B2
:102380002066696C616D656E7400616E64207072A8
:1023900065737320627574746F6E00746F20636F61
:1023A0006E74696E7565005761697420666F72009E
:1023B00066696C616D656E74206C6F6164000050BD
:1023C0007265737320427574746F6E00746F20723F
:1023D0006573756D65207072696E74000057616970
:1023E0007420666F72207072696E7400746F207250
:1023F0006573756D652E2E2E000057616974206619
:102400006F720066696C616D656E742070757267BD
:102410006500003E2000256C642E25696D0045781E
:1024200074727564656420546F74616C003E2000A2
:102430004C6F6E67657374204A6F622054696D65D6
:10244000003E2000546F74616C205072696E7420DD
:1024500054696D6500436F6D706C65746564003A16
:1024600020005072696E7420436F756E74003A20BC
:10247000003135300035004245443A204154432074
:1024800031303447542D320052756E6177617920B6
:1024900057617463683A204F4E004D61782054654F
:1024A0006D7000333135004D696E2054656D7000DC
:1024B000350045313A204550434F53203130304BA1
:1024C00000505355004154580050726F746F636F41
:1024D0006C00312E3000426175640032353030308E
:1024E0003000437265616C69747933442052414D08
:1024F0005053004D657368204C6576656C696E6756
:102500000045787472756465727300310074696E89
:10251000796D616368696E657333642E636F6D00F6
:10252000544D3344203230323000323032312D308D
:10253000342D313800322E302E375F4457372E334A
:10254000004D61726C696E005072696E7465722024
:10255000537461747300546865726D6973746F723B
:102560007300426F61726420496E666F0050726939
:102570006E74657220496E666F004D61696E004D24
:10258000313030300053746F70205072696E7400B7
:10259000526573756D65205072696E7400506F7767
:1025A0006572204F7574616765004F6666004F6EF7
:1025B0000043617365204C69676874004D61696E02
:1025C000003F004261636B0053746F70005072698A
:1025D0006E742066726F6D204D656469610043689A
:1025E000616E6765204D65646961004D323100534D
:1025F000776974636820506F776572204F6E004D65
:1026000038300053776974636820506F77657220A3
:102610004F6666004D3831004C696768747300413D
:10262000626F7574205072696E74657200436861E0
:102630006E67652046696C616D656E7400436F6EF0
:1026400066696775726174696F6E0054656D706557
:10265000726174757265004D6F74696F6E00486FBA
:102660007374205374617274004E6F204D656469F9
:102670006100526573756D65205072696E74004318
:10268000616E63656C204F626A6563740054756E99
:10269000650053746F70205072696E7400506175DC
:1026A0007365205072696E7400496E666F205363C3
:1026B0007265656E003F00537461727420507269D8
:1026C0006E740043616E63656C005072696E7400D5
:1026D00043616E6E6F7420656E74657220737562EF
:1026E0006469723A2000022E2E004D61696E00214D
:1026F00000486F74656E6420746F6F20636F6C6444
:10270000004261636B0050726F63656564004F66E1
:1027100066004F6E00536F667420456E6473746F6D
:102720007073004D6F74696F6E0044697361626C01
:1027300065205374657070657273004D38340042C3
:102740006564204C6576656C696E6700486F6D65E1
:10275000205A004732385A00486F6D6520590047AB
:1027600032385900486F6D6520580047323858009C
:102770004175746F20486F6D6500473238004D61B8
:10278000696E0050726568656174202420456E642E
:1027900000507265686561742024204265640054AD
:1027A000656D706572617475726500436F6F6C64FE
:1027B0006F776E0050726568656174202400466111
:1027C0006E205370656564207E00426564004E6F24
:1027D0007A7A6C65004D61696E004261627973744A
:1027E0006570205A00416476616E6365204B004637
:1027F0006C6F770046616E205370656564207E00C3
:10280000426564004E6F7A7A6C6500426564205AB6
:10281000005370656564004D61696E00486F6D69B5
:102820006E67204661696C6564006F70656E005468
:102830005249474745524544003A200066696C6159
:102840006D656E74007A5F6D696E00795F6D696E9B
:1028500000785F6D696E005265706F7274696E67A3
:1028600020656E6473746F70207374617475730A7D
:102870000020746F6F206C6F6E67206578747275BE
:1028800073696F6E2070726576656E7465640A0098
:1028900020636F6C6420657874727573696F6E2045
:1028A00070726576656E7465640A00000000000051
:1028B000000000000000005761726E696E673A20E8
:1028C000486F6D696E672042756D70204469766946
:1028D000736F72203C20310A00020204000048435A
:1028E00000804A43000052430000004100000041C4
:1028F0000000004000000001000000010000800016
:10290000555555000000400033333300AAAA2A0071
:102910004992240000002000C7711C0099991900F9
:10292000D1451700555515003BB11300244912003D
:1029300011111100000010000F0F0F00E3380E00FE
:1029400043790D00CCCC0C00C3300C00E8A20B0086
:1029500064210B00AAAA0A00703D0A009DD8090054
:10296000427B090092240900DCD308008888080013
:102970001042080000000800F0C107008787070028
:1029800075500700711C07003EEB0600A1BC060055
:102990006990060066660600703E06006118060033
:1029A00017F4050074D105005BB00500B290050076
:1029B000627205005555050078390500B81E0500FE
:1029C000050505004EEC040087D40400A1BD0400F9
:1029D00090A7040049920400C17D0400EE69040040
:1029E000C7560400444404005C320400082104007B
:1029F00041100400000004003FF00300F8E0030071
:102A000026D20300C3C30300CCB503003AA80300D9
:102A10000A9B0300388E0300C08103009F750300EA
:102A2000D0690300505E03001D53030034480300C7
:102A3000913D03003333030016290300381F0300C0
:102A400097150300300C0300030303000BFA020088
:102A500049F10200BAE802005CE002002DD8020051
:102A60002DD0020059C80200B0C0020031B90200E6
:102A7000DAB10200AAAA0200A0A30200BC9C0200D4
:102A8000FA9502005C8F0200DF8802008282020059
:102A9000457C02002776020027700200436A02008C
:102AA0007C640200D05E02003F590200C85302005D
:102AB000FFFDFCFAF8F6F4F2F0EEECEAE9E7E5E304
:102AC000E1E0DEDCDAD9D7D5D4D2D0CFCDCBCAC8BD
:102AD000C7C5C3C2C0BFBDBCBAB9B7B6B4B3B2B044
:102AE000AFADACAAA9A8A6A5A4A2A1A09E9D9C9AA0
:102AF00099989795949392908F8E8D8B8A898887D9
:102B00008684838281807F7E7D7B7A7978777675F3
:102B100074737271706F6E6D6C6B6A6968676665ED
:102B200064636261605F5E5D5C5B5A5958585756DA
:102B3000555453525150504F4E4D4C4B4A4A4948B0
:102B4000474646454443424241403F3E3E3D3C3B72
:102B50003B3A393838373635353433323231303024
:102B60002F2E2E2D2C2B2B2A2929282727262525C9
:102B700024232322212120201F1E1E1D1C1C1B1B61
:102B80001A191918181716161515141313121211ED
:102B900011100F0F0E0E0D0D0C0C0B0A0A0909086F
:102BA00008070706060505040403030202010000E6
:102BB0000000484300804A430000524300000000E8
:102BC000000000000000000053657474696E6773B4
:102BD0002053746F72656400454550524F4D204933
:102BE0006E697469616C697A65640A003B20002033
:102BF000204D363033200020440020204D34313227
:102C000020530046696C616D656E742072756E6F3D
:102C100075742073656E736F723A002055004C0016
:102C200046696C616D656E74206C6F61642F756EA2
:102C30006C6F6164206C656E677468733A00202065
:102C40004D393030204B004C696E65617220416413
:102C500076616E63653A0020204D34313320530095
:102C6000506F7765722D4C6F7373205265636F766A
:102C70006572793A0020204D3235302043004C43B4
:102C80004420436F6E74726173743A0020440020D4
:102C9000490020204D33303420500020440020498A
:102CA0000020204D333031205000504944207365BE
:102CB0007474696E67733A00204600204800202033
:102CC0004D3134352053004D6174657269616C205B
:102CD00068656174757020706172616D657465728C
:102CE000733A002020473239205334205A00204ABA
:102CF00000202047323920533320490020204D3412
:102D000032302053004D65736820426564204C6565
:102D100076656C696E673A0020204D323036205857
:102D200000486F6D65206F66667365743A002058C1
:102D30000020530020204D3230352042004164767F
:102D4000616E6365643A20423C6D696E5F736567CE
:102D50006D656E745F74696D655F75733E20533C7D
:102D60006D696E5F66656564726174653E20543C92
:102D70006D696E5F74726176656C5F6665656472BD
:102D80006174653E20583C6D61785F785F6A65725A
:102D90006B3E20593C6D61785F795F6A65726B3E6E
:102DA000205A3C6D61785F7A5F6A65726B3E2045A0
:102DB0003C6D61785F655F6A65726B3E0020540010
:102DC00020520020204D3230342050004163636592
:102DD0006C65726174696F6E2028756E6974732FEB
:102DE0007332293A20503C7072696E745F6163637C
:102DF000656C3E20523C726574726163745F6163FE
:102E000063656C3E20543C74726176656C5F6163EF
:102E100063656C3E0020204D3230312058004D61FA
:102E200078696D756D20416363656C657261746965
:102E30006F6E2028756E6974732F7332293A0020E3
:102E4000204D3230332058004D6178696D756D200A
:102E50006665656472617465732028756E69747344
:102E60002F73293A00537465707320706572207552
:102E70006E69743A0020440020204D3230302053D7
:102E8000002044697361626C65640A0046696C6184
:102E90006D656E742073657474696E67733A002093
:102EA000204D3134392043203B20556E6974732006
:102EB000696E2043656C736975730A0020286D6D17
:102EC00029002020473231202020203B20556E69E8
:102ED000747320696E206D6D0000803B4400803B60
:102EE0004400002041000096420000A0420000A0E3
:102EF000420000C8430000E242D0070000D00700B3
:102F000000640000004B00000024F4D43050C38E55
:102F100020C2A24017828B7011127A910D816CD958
:102F20000AA861E108C7586607615143061E4B5D58
:102F300005C145A7041A411104093D9803713931AF
:102F4000034036DB0265339102D4305402802E1DDB
:102F500002632CEE01752AC501B028A0011027815B
:102F6000018F2564012B244B01E0223401AC211F89
:102F7000018D200D01801FFC00841EED00971DDFD8
:102F800000B81CD200E61BC600201BBC00641AB2AD
:102F900000B219A8000A19A0006A189900D1179167
:102FA0000040178B00B516840031167E00B31579EA
:102FB000003A157300C7146F0058146A00EE1366C8
:102FC000008813630025135E00C7125B006C125764
:102FD0000015125400C111510070114F0021114B06
:102FE00000D61049008D10470046104400021042E0
:102FF00000C00F4000800F3E00420F3C00060F3B18
:1030000000CB0E3800930E37005C0E3500270E34CF
:1030100000F30D3200C10D3100900D3000600D2E17
:1030200000320D2D00050D2C00D90C2B00AE0C2903
:1030300000850C29005C0C2700350C27000E0C269F
:1030400000E80B2400C40B2400A00B23007D0B23FD
:10305000005A0B2100390B2100180B2000F80A1F21
:1030600000D90A1E00BB0A1E009D0A1D00800A1D11
:1030700000630A1C00470A1B002C0A1B00110A1AD5
:1030800000F7091A00DD091900C4091900AB091974
:1030900000920917007B091800630917004C0916F4
:1030A0000036091600200916000A091500F5081552
:1030B00000E0081400CC081400B8081400A4081498
:1030C00000900813007D0812006B081300580812C6
:1030D00000460812003408110023081100120811DC
:1030E0000001081100F0071000E0071000D00710E1
:1030F00000C0071000B0070F00A107100091070ED5
:103100000083070F0074070F0065070E0057070EB6
:103110000049070E003B070D002E070E0020070D8B
:103120000013070D0006070D00F9060C00ED060D53
:1031300000E0060C00D4060C00C8060C00BC060C0F
:1031400000B0060C00A4060B0099060C008D060BBF
:103150000082060B0077060B006C060B0061060A66
:103160000057060B004C060A0042060A0038060A01
:10317000002E060A0024060A001A060A0010060994
:103180000007060A00FD050900F4050900EB050922
:1031900000E2050900D9050900D0050900C70509A5
:1031A00000BE050900B5050800AD050800A5050924
:1031B000009C050800940508008C0508008405089B
:1031C000007C050800740508006C0507006505080B
:1031D000005D050700560508004E05070047050776
:1031E000004005080038050700310507002A0507DB
:1031F00000230507001C050600160507000F05073C
:10320000000805060002050700FB040600F5040798
:1032100000EE040600E8040600E2040700DB0406F2
:1032200000D5040600CF040600C9040600C3040646
:1032300000BD040600B7040600B1040500AC040696
:1032400000A6040600A00405009B040600950405E2
:1032500000900406008A0405008504050080040629
:10326000007A04050075040500700405006B040570
:103270000066040500610405005C040500570405B0
:1032800000520405004D04050048040500430405F0
:10329000003E0404003A040500350405003004042F
:1032A000002C04050027040400230405001E040468
:1032B000001A04040016040500110404000D04049F
:1032C00000090405000404040000040400FC0304D5
:1032D00000F8030400F4030400F0030400EC03040A
:1032E00000E8030400E4030400E0030400DC03043A
:1032F00000D8030400D4030400D0030400CC03046A
:1033000000C8030300C503030024F404D9201BC430
:103310000C5C0E9804C4095F0265077101F405F99D
:1033200000FB04B30048048700C10369005803553B
:103330000003034500BE023A008402310053022A12
:10334000002902250004022000E4011C00C8011924
:1033500000AF0117009801140084011300710110DF
:10336000006101100051010E0043010D0036010BF8
:10337000002B010B0020010B00150109000C0109B5
:103380000003010800FB000800F3000800EB000741
:1033900000E4000600DE000600D8000600D20006A9
:1033A00000CC000500C7000500C2000500BD0004F8
:1033B00000B9000400B5000400B1000400AD000431
:1033C00000A9000400A5000300A20003009F000460
:1033D000009B000300980003009500020093000387
:1033E00000900003008D0002008B000300880002A3
:1033F000008600020084000300810002007F0002BA
:10340000007D0002007B00020079000200770001CD
:1034100000760002007400020072000100710002D8
:10342000006F0002006D0001006C0002006A0001E4
:1034300000690002006700010066000100650001EC
:1034400000640002006200010061000100600001F0
:10345000005F0002005D0001005C0001005B0001F4
:10346000005A0001005900010058000100570001F6
:1034700000560001005500010054000100530000F7
:1034800000530001005200010051000100500001F2
:10349000004F0001004E0000004E0001004D0001F1
:1034A000004C0001004B0000004B0001004A0001ED
:1034B00000490001004800000048000100470001E9
:1034C00000460000004600010045000000450001E4
:1034D00000440001004300000043000100420000DE
:1034E00000420001004100000041000100400001D5
:1034F000003F0000003F0001003E0000003E0001D0
:10350000003D0000003D0001003C0000003C0000C8
:10351000003C0001003B0000003B0001003A0000BD
:10352000003A0001003900000039000100380000B5
:1035300000380000003800010037000000370001AB
:1035400000360000003600000036000100350000A3
:103550000035000000350001003400000034000098
:10356000003400010033000000330000003300018C
:103570000032000000320000003200010031000083
:103580000031000000310001003000000030000078
:1035900000300001002F0000002F0000002F00006D
:1035A000002F0001002E0000002E0000002E000160
:1035B000002D0000002D0000002D0000002D000156
:1035C000002C0000002C0000002C0000002C00014A
:1035D000002B0000002B0000002B0000002B00013E
:1035E000002A0000002A0000002A0000002A000132
:1035F0000029000000290000002900000029000027
:103600000029000100280000002800000028000018
:10361000002800000028000100270000002700000B
:1036200000270000002700000027000100260000FE
:1036300000260000002600000026000000260001F1
:1036400000250000002500000025000000250000E6
:1036500000250000002500010024000000240000D7
:1036600000240000002400000024000100230000CA
:1036700000230000002300000023000000230000BE
:1036800000230000002300010022000000220000AF
:1036900000220000002200000022000000220001A1
:1036A0000021000000210000002100000021000096
:1036B0000021000000210000002100010020000086
:1036C000002000000020000000200000002000007A
:1036D000002000000020000000200001001F00006A
:1036E000001F0000001F0000001F0000001F00005E
:1036F000001F0000001F0001001E0000001E00004F
:10370000001E0000001E000000232C0000B8220054
:1037100000561800003A0F0000B8080000B104007D
:1037200000710200003E01000020436F756E74209E
:10373000583A0042656400453100626564002C20FF
:1037400073797374656D2073746F70706564212074
:103750004865617465725F49443A20004865617448
:10376000696E67204661696C6564004865617469CB
:103770006E67206661696C6564004D31313220539B
:10378000687574646F776E001000C90210012C0117
:103790004001220170011801B0010E01F001040185
:1037A0005002FA00B002F0003003E600D003DC0063
:1037B0009004D2007005C800A006BE000008B40046
:1037C000B009AA00D00BA000600E960060118C001A
:1037D0000015820020197800C01D6E00A022640030
:1037E000B0275A00902C500000314600E0343C00D5
:1037F00010383200903A2800603C1E00A03D1400B2
:10380000803E0A00203F0000544845524D414C2064
:1038100052554E4157415900546865726D616C2094
:1038200052756E61776179004572723A204D415848
:1038300054454D50004D415854454D5020747269C7
:10384000676765726564004572723A204D494E544F
:10385000454D50004D494E54454D50207472696796
:10386000676572656400202F002042403A002040C6
:103870003A0020573A0020573A00496E76616C6949
:10388000642065787472756465720A007C3C3E5EE3
:103890002B3D3F2F5B5D3B2C2A225C0043616E6E0B
:1038A0006F74206F70656E2073756264697220009A
:1038B000534420496E6974204661696C005344206A
:1038C00063617264206F6B0A006F70656E526F6F78
:1038D00074206661696C65640A00766F6C756D654D
:1038E0002E696E6974206661696C65640A004E6FAA
:1038F00020534420636172640A000A4D3234004D43
:1039000032332025730041425300504C41002E0AAF
:10391000006F70656E206661696C65642C20466975
:103920006C653A200046696C652073656C6563744C
:1039300065640A002053697A653A200046696C651F
:10394000206F70656E65643A2000454E44205355E3
:1039500042524F5554494E450A002220706F730061
:103960002220706172656E743A2200535542524FA4
:103970005554494E452043414C4C20746172676553
:10398000743A220053756263616C6C204F766572E5
:10399000666C6F77004578636565646564206D616A
:1039A0007820535542524F5554494E452064657016
:1039B00074683A002E0A0044656C6574696F6E2065
:1039C0006661696C65642C2046696C653A20004626
:1039D000696C652064656C657465643A00534420C5
:1039E0007072696E74696E67206279746520004E2A
:1039F0006F74205344207072696E74696E670A0098
:103A00002F6175746F25632E670057726974696E34
:103A10006720746F2066696C653A20006672657372
:103A20006800646F696E67002066696C653A200003
:103A30004E6F77200002FD55555555555FFFFFFF2E
:103A4000FFFFFFFFFFFFFE00000000003FFFFFFF42
:103A5000FFFFFFFFFFFFFD000007FFFFFFFFFFFF6E
:103A6000FFFFFFFFFFFFFE07C00555555555555F8A
:103A7000FFFFFFFFFFFFFC0A200600000000003FE1
:103A8000FFFFFFFFFFFFFE141005000007FFFFFF11
:103A9000FFFFFFFFFFFFFC28080607C0055555552F
:103AA00055555FFFFFFFFE5404040A200600000086
:103AB00000003FFFFFFFFC60040614100500000734
:103AC000FFFFFFFFFFFFFE50040428080607C005A4
:103AD00055555555555FFC6004065404040A2006EC
:103AE00000000000003FFE54041C60040614100592
:103AF00000000000001FFC28082E500404280806BF
:103B000007C00001F03FFE14105460040654040482
:103B10000A200002081FFC0A206654041C600406E8
:103B200014100005043FFE07C05428082E5004045A
:103B30002808000A021FFC00002E1410546004061E
:103B400054040015013FFE00001C0A206654041CAA
:103B500060040018011FFC00000607C05428082E4E
:103B600050040014013FFE00000400002E14105405
:103B700060040018011FFCFFFFFE00001C0A206605
:103B800054041C15013FFED5555400000607C054CF
:103B900028082A0A021FFC84104600000400002E98
:103BA00014105105043FFEC41044FFFFFE00001C2A
:103BB0000A206102881FFC841046D5555400000677
:103BC00007C05101F03FFE841044841046000004F9
:103BD00000002A00001FFCC41046C41044FFFFFE72
:103BE00000001C00003FFE841044841046D555544C
:103BF00000000000001FFCD5555684104484104678
:103C000000000000003FFCFFFFFCC41046C410444D
:103C1000FFFFFFFFFF9FFE00000684104484104654
:103C2000D555555555BFFD555554D5555684104459
:103C300084104104109FFFFFFFFCFFFFFCC41046EF
:103C4000C410410411BFFFFFFFFE000006841044B2
:103C500084104104109FFFFFFFFD555554D5555664
:103C600084104104109FFFFFFFFFFFFFFCFFFFFCDC
:103C7000C410410411BFFFFFFFFFFFFFFE0000065D
:103C800084104104109FFFFFFFFFFFFFFD555554B7
:103C9000D555555555BFFFFFFFFFFFFFFFFFFFFC49
:103CA000FFFFFFFFFF9FFFFFFFFFFFFFFFFFFFFE85
:103CB00000000000003FFFFFFFFFFFFFFFFFFFFDD1
:103CC00055555555555FFFFFFFFFFFFFFFFFFFFFF6
:103CD000FFFFFFFFFFFFFFFFFFFFFFFFFFFFFFFFF4
:103CE000FFFFFFFFFFFFFFFFFFFFFFFFFFFFFFFFE4
:103CF000FFFFFFFFFFFFFFFFFFFFFFFFFFFFFFFFD4
:103D0000FFFFFFFFFFFFE02EFB7DFBFBCFC1DFBB13
:103D10003EC0E1FE3C1FFDEE7B39F9F3CF9EDFBBD9
:103D20003EDFDEFCDDE7FDEE3BBBF9EBD7BF5FBB63
:103D30005EDFDEFDEDF7FDEEBBD3FAEBB73FDFBB99
:103D40004EDFDFFFCDF3FDEEDBC7FAEBBB7FC03B01
:103D50006EC0E3FF1DF3FDEECBEFFADBBB7FDFBBF5
:103D600066DFF8FFCDF3FDEEEBEFFB5B033F5FBBE0
:103D700076DFFE7FEDF3FDEEF3EFFB5B79BEDFBB9D
:103D80007ADFDE7DEDF7FDEEF3EFFBBAFD9EDFBBE4
:103D90007CDFDEFDCDE7FDEEFBEFFBBAFDC1DFBB57
:103DA0007EC0E0FE1C1F6D61726C696E66772E6FBF
:103DB000726700322E302E375F4457372E33001F84
:103DC000FFFFFFFFFFFF600000000001FF40000059
:103DD000000000FF8000000000007F83CF00000C87
:103DE000303F87FF80000C301F867980000C000F69
:103DF0008C30C7838C30E78C30CFC7CC31F38C301C
:103E0000DCECEC33B98C30D86C6C33198C30D06C62
:103E10000C33198C30D86C0C33198C30DC6C0E3BA5
:103E2000198C30CF7C079F198C30C77C038F1940C9
:103E3000000000000002600000000000061FFFFFFD
:103E4000FFFFFFF870012C0190012701B001220152
:103E5000C0011D01F00118011002130130020E0112
:103E60006002090190020401C002FF000003FA0091
:103E70004003F5008003F000D003EB002004E600CF
:103E80007004E100E004DC004005D700C005D2006A
:103E90004006CD00D006C8008007C3003008BE0031
:103EA000F008B900C009B400B00AAF00B00BAA0016
:103EB000D00CA500000EA000500F9B00C010960073
:103EC0005012910000148C00C0158700B0178200BA
:103ED000B0197D00D01B7800001E730040206E00DA
:103EE00090226900F024640040275F0090295A0066
:103EF000E02B5500102E500020304B0010324600B1
:103F0000E033410090353C00103737007038320004
:103F1000A0392D00B03A2800A03B2300603C1E00D1
:103F2000103D1900903D1400103E0F00703E0A0035
:103F3000C03E0500003F0000403FFBFF803FF6FF12
:103F4000C03FF1FF2020506C616E6E657242756655
:103F500066657242797465733A2000204672656521
:103F6000204D656D6F72793A2000436F6D70696CFA
:103F700065643A2041707220323420323032310A86
:103F800000204C61737420557064617465643A203C
:103F9000323032312D30342D3138207C204175744F
:103FA000686F723A2054696E794D616368696E6515
:103FB0007333440A00322E302E375F4457372E3386
:103FC0000A004D61726C696E0020536F66747761F0
:103FD00072652052657365740A00205761746368C6
:103FE000646F672052657365740A002042726F77B0
:103FF0006E206F75742052657365740A00204578D1
:104000007465726E616C2052657365740A00506F3E
:1040100077657255700A0073746172740A004732D2
:10402000385859004D31303031006572726F72204E
:1040300077726974696E6720746F2066696C650AAF
:1040400000446F6E6520736176696E672066696CE7
:10405000652E0A004D323900456E6473746F7073BB
:104060000025532025632025632025632025630038
:10407000205A3A0020593A0020583A00656E64737D
:10408000746F7073206869743A200000000A0B0294
:10409000090C0D0E080703040100000000000000D9
:1040A0000000000000000000000000000000000010
:1040B00000000000000000121110000000000000CD
:1040C00000000000000000000000000000000000F0
:1040D00000004D6F76652025736D6D004D6F766520
:1040E00020302E316D6D004D6F766520316D6D0085
:1040F0004D6F76652031306D6D004D6F76652041D6
:10410000786973004578747275646572004D6F76D6
:1041100065205A004D6F76652059004D6F766520F9
:1041200058000A3906394368616E67652046696C34
:10413000616D656E7400556E6C6F61642046696CCC
:10414000616D656E74004C6F61642046696C616DD1
:10415000656E740050726568656174204375737490
:104160006F6D005072656865617420240042616360
:104170006B00FFFFFF486F6D652025732573257366
:104180002046697273740073686F77006275747487
:104190006F6E00626567696E0044697361626C6589
:1041A00052756E6F75740050757267654D6F7265EC
:1041B0000050617573656400436F6E74696E756558
:1041C000004C6F61642046696C616D656E742054AB
:1041D00000496E736572742066696C616D656E74FA
:1041E00020616E642073656E64204D3130380A00A2
:1041F000220A00556E6B6E6F776E20636F6D6D6176
:104200006E643A2022002042002050006F6B005460
:104210004D334420323032302052656164792E00B3
:104220005072696E74696E672E2E2E005072696E20
:10423000742050617573656400204500205A002089
:104240005900204D393220580020453A00205A3A72
:104250000020593A00583A0020746F6F206C6F6E3E
:104260006720657874727573696F6E2070726576F9
:10427000656E7465640A0020636F6C6420657874F1
:10428000727573696F6E2070726576656E746564A1
:104290000A00526573656E643A20006E6F74696639
:1042A00069636174696F6E20000000220025002898
:1042B000002B002E0031003400020100000501082F
:1042C000010B0100002100240027002A002D0030EE
:1042D00000330001010000040107010A0105050582
:1042E00005070508080808020202020A0A0808046D
:1042F000040404010101010101010103030303039B
:10430000030303040707070C0C0C0C0C0C0C0C0229
:1043100002020206060606060606060B0B0B0B0B30
:104320000B0B0B0102102020080810204010204029
:104330008002010201080402010102040810204069
:104340008080402010080402018004020180402087
:1043500010080402010804020101020408102040B0
:104360008001020408102040800088027E0211248F
:104370001FBECFEFD1E2DEBFCDBF00E00CBF13E028
:10438000A0E0B2E0EEEAF6EC02E00BBF02C007905C
:104390000D92A437B107D9F728E1A4E7B3E001C033
:1043A0001D92AE3EB207E1F711E2C6EBD1E200E0AA
:1043B00006C021970109802FFE010F94B45FC53B11
:1043C000D10780E00807A9F70F945A4E0D94456372
:1043D0000C940000FC0184910895FC0180810895F3
:1043E00090E080E00895CF93DF93DB01F9019C9189
:1043F0009130C1F0943080F094509C938830D1F487
:1044000080819181009771F0019791838083480F9B
:10441000591FEA01188206C08C3539F49C5F9C93C1
:10442000943041F4DF91CF9108958B3339F781E0D7
:104430008C93F8CF20813181B9016F5F7F4F7183F9
:104440006083420F531FEA018883808191818F35F9
:1044500091056CF7E7CF0F931F9381E00091D5167C
:104460001091D6162091D7163091D8164091D116BA
:104470005091D2166091D3167091D4160417150777
:104480002607370708F480E01F910F91089590E008
:1044900080E00895282F90917E08833021F495FDC7
:1044A0000FC094FD0FC0892F90E0B0E0A0E004C0E1
:1044B000B695A795979587952A95D2F78170089517
:1044C00081E0089580E008958091DB07882321F042
:1044D000999AA19A1092DB0708951092650880912D
:1044E000550290915602A0915702B09158028093C4
:1044F0004E0690934F06A0935006B0935106089530
:10450000129A0895269A2E9A0895EF92FF920F9389
:104510001F93CF93DF93EC018B017A018A859B85F2
:104520008617970731F0888199810F94A6431B87DE
:104530000A87B701888199810F946B352E813F815D
:10454000820F932F911D9F838E8390E080E0DF91F7
:10455000CF911F910F91FF90EF9008959F92AF928E
:10456000BF92CF92DF92EF92FF920F931F93CF9360
:10457000DF93EC018B01942EA52E8A859B858617EF
:10458000970731F0888199810F94A6431B870A878A
:1045900088859985019649F5BC800A818E81080F2E
:1045A000C880D980D6015596ED91FC91C601199528
:1045B000B80EE92CFA2C10E0F70121917F012111AE
:1045C00027C08E819F81810F911D9F838E8390E0F4
:1045D00080E0DF91CF911F910F91FF90EF90DF90DE
:1045E000CF90BF90AF909F9008950E811F81692D4D
:1045F0007A2D888199810F946B35800F912F911DB1
:10460000288539852817390738F681E090E0E1CF11
:104610004B2D602FC6010F94FE43080F180FCCCF0F
:10462000DF92EF92FF920F931F93CF93DF93EC01F2
:10463000D62E1CAD0BAD7C0184E0E80EF11CE98D9B
:10464000FA8DC7011995412F480F2D2D602FC701F5
:104650000F94FE439BAD890F8BAF81E090E0DF911B
:10466000CF911F910F91FF90EF90DF900895AF923F
:10467000BF92DF92EF92FF920F931F93CF93DF933E
:104680008C01EB01D42E79018FE0481709F486C024
:10469000A5E14A17B1F1BAE04B130EC0EC81FD81E0
:1046A00030E020E042E061E0C801199540EB57E1BD
:1046B000BE01C8010F94A9440A80DB81C02DF2E33A
:1046C000DF1609F4E2C0FD1508F491C085E1D816A3
:1046D00009F4E0C0A7E1DA1609F4EFC0B4E1DB1297
:1046E0007BC0EE81FF818D8190E0880F991F8E0F36
:1046F0009F1F11928E179F07E1F7CE010F94C641BD
:104700006BC0AA80BB804BE957E1C8010F94A94454
:10471000F5014481440F406BBE01C8010F949144E0
:1047200041E0BE01C8010F949944D50116962D9120
:104730003C911797EC81FD8115964C9166E0C8017C
:10474000199540E0BE01C8010F94A1444BE957E11F
:10475000BE01C8010F94A944F5014481440F4F5F85
:10476000406BBE01C8010F94914441E0BE01C801F5
:104770000F949944D50115964C91159716962D9145
:104780003C91240F311DEC81FD8166E0C801199533
:1047900040E0BE01C8010F94A1448ECF41E0C801A2
:1047A0000F94A14440E0BE01C8010F94994441E830
:1047B000BE01C8010F949144F701408150E0559526
:1047C000479555954795BE01C8010F94914440E027
:1047D000BE01C8010F94A14481E0DF91CF911F91E8
:1047E0000F91FF90EF90DF90BF90AF900895E6E4B7
:1047F000DE1609F471C0F7E4DF1609F471C08BE32B
:10480000D812EACFD70111969C91119713968C91EB
:1048100038E0390F813031F0833011F0392F02C088
:10482000392F985021E04B81491708F420E041E0EE
:10483000391708F040E091E05A81351708F490E00C
:10484000322F342B932311F4242331F2F7011281F8
:1048500000E0D12C843048F490E0FC01E155FD4F9C
:10486000D08085559D4FDC010C9117FF04C0B70126
:10487000CE010F94CD41F70180818D0D8083818120
:10488000800F8183110F89F7A7CFB701CE010F9455
:10489000CD41A2CFCE010F94B041882309F49DCF22
:1048A000EE81FF818D8190E0880F991F8E0F9F1FF1
:1048B00011928E179F07E1F78FCFD7011C928A8143
:1048C00011968C9311978D81815012968C9312972B
:1048D0008B8113968C9380CF8D81F70180837CCF61
:1048E0008981D7018C9378CFAB01BC014093D51659
:1048F0005093D6166093D7167093D8168EE398E12E
:104900000C941CD4809323028032B8F59091190541
:10491000891724F091E0980F90931905409115059F
:10492000509116056091170570911805082E04C066
:1049300076956795579547950A94D2F741704093BD
:104940006A1087FD1DC0282F082E000C330B3F93E3
:104950008F938AEA99E09F938F938AEB99E09F93D4
:104960008F931F920E9419B78DB79EB707960FB607
:10497000F8949EBF0FBE8DBF089510926A10E1CFCC
:104980000D94C0480F931F93CF93DF9300D01F92D5
:10499000CDB7DEB79C010CE418E090E1E5EBF0E167
:1049A000D80101900D929A95E1F7F90120813181AA
:1049B00042815381F80160857185828593850F94CA
:1049C000BD5FF801608771878287938780E090E000
:1049D000A0EAB0E489839A83AB83BC83CE010196BD
:1049E0000E94F8FE0F900F900F900F90DF91CF91E3
:1049F0001F910F9108952F923F924F925F926F9265
:104A00007F928F929F92AF92BF92CF92DF92EF925E
:104A1000FF921F93CF93DF93CDB7DEB72C970FB6DE
:104A2000F894DEBF0FBECDBF7A011901DC012D91D4
:104A30003D914D915C912D833E834F835887FB01BF
:104A400040805180628073808090B5109090B61045
:104A5000A090B710B090B810A50194016D817E812F
:104A60008F8198850F94CB5881110EC011E0A3015E
:104A700092016091B9107091BA108091BB10909121
:104A8000BC100F94CB58811110E0D1012D913D91B4
:104A90004D915C9129873A874B875C87F701C080ED
:104AA000D180E280F3802091090230910A02409186
:104AB0000B0250910C02C701B6010F94CB5888230A
:104AC00009F44EC0C0920902D0920A02E0920B0291
:104AD000F0920C028091C1109091C210A091C3106D
:104AE000B091C4104091B9105091BA106091BB10B0
:104AF0007091BC1080924C0890924D08A0924E0884
:104B0000B0924F0840935008509351086093520858
:104B100070935308C0925408D0925508E0925608FA
:104B2000F09257088093580890935908A0935A0818
:104B3000B0935B0820E030E040E05FE360919810C4
:104B40007091991080919A1090919B100F94315907
:104B500069837A838B839C83CE0101960E94F8FE41
:104B60002D813E814F81588520934C0830934D080C
:104B700040934E0850934F0840925008509251086D
:104B80006092520870925308D1012D913D914D9140
:104B90005C91609158087091590880915A089091E1
:104BA0005B080F94BD5F6093580870935908809319
:104BB0005A0890935B0811112FC020E030E0A90142
:104BC00069857A858B859C850F94CB58811133C07C
:104BD00060E070E088EC92E469837A838B839C8345
:104BE000CE0101960E94F8FE2C960FB6F894DEBF17
:104BF0000FBECDBFDF91CF911F91FF90EF90DF905F
:104C0000CF90BF90AF909F908F907F906F905F906C
:104C10004F903F902F9008952AEF3EE74AE25FE3DE
:104C200060919C1070919D1080919E1090919F10AA
:104C30000F943159D1CF60E070E080EA91E4CCCF9D
:104C40008091D0049091D104009731F04AE050E077
:104C500070E060E00D94E65660E070E0CB010895EE
:104C60008091770982FF0BC063E686E99AE00E9493
:104C700034B70F94BA3B0E948BBE81E0089580E068
:104C800008958091D0049091D104009731F04AE0CA
:104C900050E070E060E00D94B85560E070E0CB014A
:104CA0000895AF92BF92CF92DF92EF92FF920F934F
:104CB0001F93CF93DF93EC015B018A01FB011995F0
:104CC00087FD16C0C82ED12CF12CE12C2196F801BD
:104CD000C082D182E282F382CE01DF91CF911F9117
:104CE0000F91FF90EF90DF90CF90BF90AF9008951D
:104CF000982F907E903CA9F48F7190E0B0E0A0E0F6
:104D00006C017D0156E0CC0CDD1CEE1CFF1C5A959D
:104D1000D1F7CE010196F50119958F73C82A229615
:104D2000D6CF982F907F903E11F58F7090E0B0E035
:104D3000A0E06C017D0136E0CC0CDD1CEE1CFF1CFC
:104D40003A95D1F7CE010196F50119958F73C82ACE
:104D500046E0CC0CDD1CEE1CFF1C4A95D1F7CE01C1
:104D60000296F50119958F73C82A2396B0CF982F14
:104D7000987F903F79F5877090E0B0E0A0E06C01FB
:104D80007D0186E0CC0CDD1CEE1CFF1C8A95D1F762
:104D9000CE010196F50119958F73C82A96E0CC0CC7
:104DA000DD1CEE1CFF1C9A95D1F7CE010296F50191
:104DB00019958F73C82A26E0CC0CDD1CEE1CFF1C55
:104DC0002A95D1F7CE010396F50119958F73C82A5C
:104DD00024967DCF982F907C903841F4807C803849
:104DE00069F42196CE01F5011995F8CF8E7F8D3F9C
:104DF00028F02196CE01F5011995F8CFC12CD12CC0
:104E0000760165CF9CE0899F802D112491E0980F59
:104E100090931A052CE0280F2093460830E02E5F6F
:104E20003F4F40919F164217130619F014F080E08F
:104E300008952091A1169217D0F7662341F08E5F56
:104E40000F94C042809146088E5F0F94C0428091BB
:104E5000460890919F16891750F32091A1169091C2
:104E60001A05291720F31092A2168093A31681E049
:104E7000089520910B05022E000C330B82171306A8
:104E800041F080930B056DED77E18BE696E10D9493
:104E9000A64308951F93CF93DF931F92CDB7DEB73C
:104EA0008F3F910519F014F08FEF90E0883791054E
:104EB00014F488E790E09093530280935202182FE5
:104EC0008091A416811105C081E08093A4160F94EF
:104ED000E74160916D1670916E1619839E012F5FE8
:104EE0003F4F4FE08BE696E10F94E3410F90DF9147
:104EF000CF911F910895CF9380910C0581114FC0E0
:104F00001092A2161092A3161092A4161092701668
:104F100010926F16109272161092711610927416EB
:104F200081E08093731682E28093751610927A1650
:104F300010927916EEE8F6E12CE936E18FEF8193D5
:104F40002E173F07E1F7C1E0C0938B1626E232E04F
:104F50003093811620938016C09382161092831688
:104F60001092841690E490938516109286162AE18A
:104F700032E030939D1620939C1626E132E0309368
:104F80006E1620936D1699E1909390169BE1909385
:104F90008F1680938E160F94E741C0930C05809175
:104FA0005202909153020E944A2781E080930D059E
:104FB0008BE997E19093DE158093DD151092E01553
:104FC0001092DF15CF910895CF92DF92EF92FF926A
:104FD0000F931F93CF93DF93CDB7DEB72C970FB608
:104FE000F894DEBF0FBECDBF6F3F710581059105FF
:104FF00009F0D0F487E696E10E941023E0916F1645
:10500000F09170163196849190E02C960FB6F8943A
:10501000DEBF0FBECDBFDF91CF911F910F91FF90EB
:10502000EF90DF90CF900895F090A216E090A31635
:1050300020910D0521110FC04BE757E16E2D8F2DEB
:105040000F946A4490E080E0F80EF092A216E0928D
:10505000A3169927DACFC0906F16D09070162BE662
:1050600036E13A8329832F2D30E03C832B832E2D8C
:1050700030E03E832D8318861F822FEF3FEF3A8763
:1050800029871C861B860EEA12E29E012F5F3F4F86
:10509000AB01BC01C6010F94A82BB6018BE696E1CB
:1050A0000F94A6438F819885CFCFCF93DF93FC01D8
:1050B00025AD211104C021E025AF0F94E741C09137
:1050C0006D16D0916E16E0919C16F0919D1682E0BF
:1050D0001995E0919C16F0919D1681E0199530E0AC
:1050E00020E044E1BE018BE696E10F94E3412EE916
:1050F00036E147E1BE018BE696E10F94E341E09192
:105100009C16F0919D1680E0DF91CF911994CF927B
:10511000DF92EF92FF920F931F93CF93DF93CDB760
:10512000DEB72C970FB6F894DEBF0FBECDBFF09060
:10513000A216E090A31620910D0521111DC04BE58C
:1051400057E16E2D8F2D0F946A4490E080E0F80EA9
:10515000F092A216E092A31699272C960FB6F89417
:10516000DEBF0FBECDBFDF91CF911F910F91FF909A
:10517000EF90DF90CF900895C0906F16D09070168A
:105180002BE636E13A8329832F2D30E03C832B83B5
:105190002E2D30E03E832D8318861F827A87698703
:1051A0001C861B860EEA12E29E012F5F3F4F4AEEDD
:1051B00051E2BC01C6010F946C2CB6018BE696E15E
:1051C0000F94A6438F819885C2CF6FEF7FEF0C9429
:1051D0008728CF92DF92EF92FF920F931F93CF9386
:1051E000DF93CDB7DEB72C970FB6F894DEBF0FBEB6
:1051F000CDBFF090A216E090A31620910D052111CD
:105200001DC04BE357E16E2D8F2D0F946A4490E043
:1052100080E0F80EF092A216E092A31699272C9641
:105220000FB6F894DEBF0FBECDBFDF91CF911F91B7
:105230000F91FF90EF90DF90CF900895C0906F1680
:10524000D09070162BE636E13A8329832F2D30E07B
:105250003C832B832E2D30E03E832D8318861F82C6
:105260007A8769871C861B860EEA12E29E012F5FF1
:105270003F4F4DEE51E2BC01C6010F946C2CB601BC
:105280008BE696E10F94A6438F819885C2CFBF929B
:10529000CF92DF92EF92FF920F931F93CF93DF9302
:1052A0008B01F42EE90141FB662760F90E94022779
:1052B000882309F45AC0B12C0115110521F0C80149
:1052C0000E945CBFB82EE12C209721F0CE010E94F5
:1052D00047C1E82E80E8C82ED12CF0FE1EC085E123
:1052E00090E08B199109B7FC93958E199109E7FC11
:1052F000939597FD019695958795F82E30E8C32EE6
:10530000D12CFA94F7FC09C060E270E080E090E0F4
:105310000E94E427C81AD90AF4CFBB2099F0C6012D
:1053200066E070E00F948C5F262F40914808509102
:10533000490860914708C8010E949CBE96E0899F79
:1053400060011124EE2031F0B601CE010E94E9285F
:10535000C81AD90A87E0C816D10438F060E270E0B4
:1053600080E090E00E94E427F3CFDF91CF911F917E
:105370000F91FF90EF90DF90CF90BF9008956FEF67
:105380007FEF0C94E928AF92BF92CF92DF92EF9219
:10539000FF920F931F93CF93DF935C016B010E94E9
:1053A0005CBFE82EC6010E9447C1F12C03E110E06A
:1053B000081B1109C5E20E151F050CF4CFE18C2F57
:1053C00090E09C012E5F3F4F40919F1642171306BD
:1053D00009F0CCF509972091A116281719069CF120
:1053E0004091480850914908609147081092A216D0
:1053F000C093A31625E1C5010E949CBED1E0C11453
:10540000D104B1F06AE370E080E090E00E94E4270C
:105410000E151F05D4F4C45F80919F16C81740F085
:105420002091A1164C2F4950550B241715067CF4DA
:10543000DF91CF911F910F91FF90EF90DF90CF9070
:10544000BF90AF900895D0E0DACFDD2389F3802FAD
:10545000880F080F000F0093A216C093A31660E2F6
:1054600070E080E090E00E94E427C601DF91CF91D8
:105470001F910F91FF90EF90DF90CF90BF90AF9072
:105480000C94BF298F929F92AF92BF92CF92DF92DE
:10549000EF92FF920F931F93CF93DF93CDB7DEB7B9
:1054A0002C970FB6F894DEBF0FBECDBF982F862F76
:1054B0005A017901D02E692F0E940227882309F40E
:1054C00089C0C701002391F10E945CBFC82E809063
:1054D0006F169090701680910D05811145C01FEFD9
:1054E00023E12C19409148085091490860914708E0
:1054F000C5010E949CBECC2009F46CC0B6E08B9F15
:10550000500111246AE370E080E090E00E94E427FB
:1055100057E0A516B10408F444C060E270E080E0F2
:1055200090E00E94E427A81AB90AF2CF0E9447C16E
:10553000C82E80906F169090701680910D0588236C
:1055400071F2FE0133968AE0DF011D928A95E9F738
:105550008BE696E19A83898305E812E29E012F5F2C
:105560003F4F4DEE51E212C0FE0133968AE0DF015B
:105570001D928A95E9F78BE696E19A83898305E87F
:1055800012E29E012F5F3F4F4AEE51E2B701C40184
:105590000F946C2CB4018BE696E10F94A6431F8107
:1055A0009FCF40914608212F30E0A6E0CA9EC0015F
:1055B00011242E5F3F4F281739070CF49C0180E817
:1055C000821B8093A2164093A316C701DD20A9F089
:1055D0000E94E5282C960FB6F894DEBF0FBECDBF13
:1055E000DF91CF911F910F91FF90EF90DF90CF90BF
:1055F000BF90AF909F908F9008950E94BF29EACFEF
:10560000E7E6F6E183AF64AFCA010C94BF292F929D
:105610003F924F925F926F927F928F929F92AF9242
:10562000BF92CF92DF92EF92FF920F931F93CF938F
:10563000DF93D62FC72FFC0180809180A280B3809A
:10564000C501B40120E831E541E050E00F940F5F5F
:10565000C9016DE671E00F948C5F6B017C01C5019F
:10566000B40120E13EE040E050E00F940F5FCA013A
:10567000B90128E130E040E050E00F940F5F362E92
:10568000272E062F172F8CE3482E512C612C712CBE
:10569000C501B401A30192010F940F5FB62EA72E8E
:1056A000CA01B901A30192010F940F5FCB01C1148C
:1056B000D10479F1AF92BF927F936F932F923F9273
:1056C000FF92EF92DF92CF9289E995E19F938F93BA
:1056D000CF93DF930F9462588DB79EB70E960FB697
:1056E000F8949EBF0FBE8DBF8D2F9C2FDF91CF9161
:1056F0001F910F91FF90EF90DF90CF90BF90AF90F0
:105700009F908F907F906F905F904F903F902F90E1
:105710000895E114F104C9F0AF92BF927F936F93A3
:105720002F923F92FF92EF9289E895E19F938F939A
:10573000CF93DF930F946258EDB7FEB73C960FB648
:10574000F894FEBF0FBEEDBFCFCF012BB9F0AF92E3
:10575000BF927F936F932F923F928DE795E19F9336
:105760008F93CF93DF930F9462588DB79EB70A96AD
:105770000FB6F8949EBF0FBE8DBFB6CF892BA9F090
:10578000AF92BF927F936F9385E795E19F938F933D
:10579000CF93DF930F946258EDB7FEB738960FB6EC
:1057A000F894FEBF0FBEEDBF9FCFAF92BF9281E7CF
:1057B00095E19F938F93CF93DF930F9462580F904F
:1057C0000F900F900F900F900F908ECF8F929F920F
:1057D000AF92BF92CF92DF92EF92FF920F931F93FF
:1057E000CF93DF9310920A05109209052FE32093BF
:1057F00008051092070510920605109205051092F3
:1058000001051092020510920305109204059C01F7
:10581000F90190812F5F3F4F9032D1F39E34C9F44C
:10582000818190ED980F9A3020F08D3211F08B32FB
:1058300081F432969F012F5F3F4F808180538A30E1
:1058400008F47BC09F012F5F3F4F8081803209F4B5
:1058500076C0F0936B08E0936A088F010F5F1F4FCB
:10586000C0816AE270E0C8010F940B63009731F0C9
:10587000FC01319780818032E1F31182CD3429F02F
:10588000C43519F0C73409F04BC0F80180810F5FAF
:105890001F4F8032D1F380538A3008F041C0C0934B
:1058A000080530E020E04AE0DF011196429FC00188
:1058B000439F900D11249C01205331098081280FB2
:1058C000311D87FD3A95818190ED980F9A30C8F18E
:1058D00030930705209306058E3261F4329690E0EE
:1058E0004AE0DF0131968C9150ED580F5A3058F153
:1058F00090930505CD01DC0101964C914032D9F31E
:10590000CD3489F52E31310539F018F527313105BF
:1059100019F02C31310539F5B0930A05A09309052A
:10592000DF91CF911F910F91FF90EF90DF90CF907B
:10593000BF90AF909F908F900895F9017BCFF901B0
:1059400081CFFD01B1CF949F800D112490ED980F70
:10595000C8CF2537310538F027373105E8F2203A2E
:1059600083E03807C9F2D0916A0840E050E0BA01FC
:1059700010E000E0C12CD12C7601C394FD013196DA
:105980008C91882309F47FC08132E1F4CD34D1F4C5
:1059900020323105B9F4409301055093020560931C
:1059A000030570930405F0930A05E093090563E28B
:1059B00070E0CF010F940B63009709F4B1CFFC01A5
:1059C0001082AECF81548A3108F058C0DF019D911A
:1059D000903291F0A0EDA90FAA30E8F09E3271F458
:1059E000918190539A30B8F00115110519F48F0187
:1059F0000150110990E013C0FD01E8CF9D3211F074
:105A00009B3291F79181A0EDA90FAA3020F09E3230
:105A100059F79281E6CF9E2F9D1B309759F3A82FFF
:105A2000B0E04601570104C0880C991CAA1CBB1C9D
:105A30008A95D2F7482959296A297B29A951BB4F50
:105A40009C9380818154DF018A3108F497CFDF0174
:105A50008191882309F492CF90ED980F9A30B8F392
:105A600093ED980F923098F38B3289F3CD01019624
:105A7000EC91E03209F082CFDC01F8CF011511057D
:105A800001F78D01DECF10930A05009309054093BD
:105A9000010550930205609303057093040540CF00
:105AA0009B01AC01485F5F4FBC016C5F7F4F0C9462
:105AB000FB240F931F93CF93DF9300D000D01F924E
:105AC0001F92CDB7DEB7FC018B0183A5811112C0F7
:105AD00081E083A784819581A681B781B0588983AD
:105AE0009A83AB83BC83BE016F5F7F4F8CE498E0E9
:105AF0000E94502D1D821E821F82188620E030E0F9
:105B000040E05FE36091BD107091BE108091BF10C6
:105B10009091C0100F94BD5F69837A838B839C83BF
:105B20009E012B5F3F4FAE014F5F5F4F69EB70E10E
:105B300085EB90E10E94FB241D821E821F82188645
:105B400020E030E040E05FE3F80160857185828508
:105B500093850F94BD5F69837A838B839C83B8019F
:105B60006C5F7F4F9E012B5F3F4FAE014F5F5F4FDA
:105B7000C8010E94FB2428960FB6F894DEBF0FBE22
:105B8000CDBFDF91CF911F910F9108952F923F923A
:105B90004F925F926F927F928F929F92AF92BF923D
:105BA000CF92DF92EF92FF920F931F93CF93DF93E9
:105BB000CDB7DEB7A2970FB6F894DEBF0FBECDBF4C
:105BC0008C011B015E834D834090B5105090B61040
:105BD0006090B7107090B8108090B9109090BA1083
:105BE000A090BB10B090BC10DB018D919D910D90E9
:105BF000BC91A02D8F87988BA98BBA8B9C01AD018E
:105C0000C301B2010F94BC5F6B017C01D1011496FA
:105C10008D919D910D90BC91A02D8B8B9C8BAD8B0C
:105C2000BE8B9C01AD01C501B4010F94BC5F6F8BAD
:105C3000788F898F9A8FAD81BE818D919D910D90C6
:105C4000BC91A02D8F839887A987BA879C01AD014D
:105C5000C301B2010F94BC5F6B8F7C8F8D8F9E8FC1
:105C6000AD81BE8114968D919D910D90BC91A02D1A
:105C70008B879C87AD87BE879C01AD01C501B401B0
:105C80000F94BC5F6F8F78A389A39AA3A701960195
:105C9000C701B6010F9431596B017C012F89388DF2
:105CA000498D5A8DCA01B9010F9431599B01AC013C
:105CB000C701B6010F94BD5F4B015C012F85388988
:105CC00049895A896F81788589859A850F94BC5F47
:105CD0002B013C012B893C894D895E896B857C8534
:105CE0008D859E850F94BC5F6B017C01A3019201A1
:105CF000C301B2010F9431592B013C01A701960158
:105D0000C701B6010F9431599B01AC01C301B20127
:105D10000F94BD5F0F946B626B017C012B8D3C8DEA
:105D20004D8D5E8DCA01B9010F9431592B013C0193
:105D30002F8D38A149A15AA1CA01B9010F94315937
:105D40009B01AC01C301B2010F94BD5F9B01AC018B
:105D5000C501B4010F941D621816B4F520E030E0BF
:105D6000A901C701B6010F941D6287FF2AC0C701B0
:105D7000B601905820E030E040EA50E40F941D62F4
:105D8000181614F5A1016D817E81C8010E94C62DEF
:105D9000A2960FB6F894DEBF0FBECDBFDF91CF91B4
:105DA0001F910F91FF90EF90DF90CF90BF90AF9039
:105DB0009F908F907F906F905F904F903F902F902B
:105DC0000895C701B601D6CF20E030E040E050E4AE
:105DD000C501B4010F941D62181624F4B101C80165
:105DE0000E94592D19821A821B821C82BE016F5F8C
:105DF0007F4FC1010E94502D2DEC3CEC4CEC5CE33C
:105E0000C701B6010F9431599B01AC01F8016081C3
:105E10007181828193810F94315969837A838B8355
:105E20009C83C8010F949D34BE016F5F7F4F8D81AD
:105E30009E810E94502DACCF2F923F924F925F9245
:105E40006F927F928F929F92AF92BF92CF92DF928A
:105E5000EF92FF920F931F93CF93DF93CDB7DEB7EF
:105E60006D970FB6F894DEBF0FBECDBF922EDB014B
:105E7000FC90542F5F0D553008F05CC11196BC9119
:105E8000B98F6B2F620F653008F054C1EB2FF0E033
:105E9000E953FB4F008110E030E020E00F2C04C0FC
:105EA00036952795179507950A94D2F700FF42C1BA
:105EB000262E312CF101E953FB4F008110E030E038
:105EC00020E0A52EB12C04C036952795179507958F
:105ED0005A95D2F700FF2EC1642F8C01660F770B05
:105EE000072E000C880B990B0F94D2582B013C0104
:105EF0002F2D84E02802F0011124E654F94E208170
:105F0000318142815381C301B2010F94BD5F6B01A6
:105F10007C01CD86DE86EF86F88AF501EE0FFF1F45
:105F2000EE0FFF1FE654F94EA301920160817181CB
:105F3000828193810F94BC5F6A8F7B8F8C8F9D8F42
:105F400069837A838B839C83692D660F770B072E79
:105F5000000C880B990B0F94D2584B015C01998D62
:105F6000A4E09A02F0011124EA55F94E2081318112
:105F700042815381C501B4010F94BD5F2B013C01E7
:105F8000498A5A8A6B8A7C8AF101EE0FFF1FEE0F55
:105F9000FF1FEA55F94EA50194016081718182814C
:105FA00093810F94BC5F4B015C018D829E82AF8216
:105FB000B886F80180859185A285B38589879A87FF
:105FC000AB87BC878D8B9E8BAF8BB88F20E030E08A
:105FD00040E85FE3C301B2010F94CB5887FFC3C011
:105FE00080E090E0A0E8BFE3898B9A8BAB8BBC8B01
:105FF00020E030E040E85FE3C501B4010F94CB58E6
:1060000087FFC1C080E090E0A0E8BFE38D839E835E
:10601000AF83B88720E030E040E85FE3C701B60116
:106020000F94CB5887FFBFC080E090E0A0E8BFE3AB
:106030008D879E87AF87B88B20E030E040E85FE334
:106040006A8D7B8D8C8D9D8D0F94CB5887FFBBC047
:1060500080E090E0A0E8BFE389839A83AB83BC83B0
:10606000C988DA88EB88FC8827E137EB41ED58EBEB
:10607000C701B6010F941D6287FD5CC027E030E8C0
:106080004AE453E4C701B6010F94CB5818160CF438
:1060900051C0CD84DE84EF84F88827E137EB41EDF1
:1060A00058EBC701B6010F941D6287FD43C027E07E
:1060B00030E048E453E4C701B6010F94CB581816FA
:1060C000CCF1CD80DE80EF80F88427E137EB41ED25
:1060D00058EBC701B6010F941D6287FD2BC027E066
:1060E00030E84AE453E4C701B6010F94CB581816C0
:1060F0000CF1C980DA80EB80FC8027E137EB41EDC1
:1061000058EBC701B6010F941D6287FD13C027E04D
:1061100030E048E453E4C701B6010F94CB58181699
:106120004CF0AE014F5F5F4FBE01635F7F4FC80110
:106130000E94C62D6D960FB6F894DEBF0FBECDBF80
:10614000DF91CF911F910F91FF90EF90DF90CF9053
:10615000BF90AF909F908F907F906F905F904F9087
:106160003F902F90089520E030E849E453E4C301C4
:10617000B2010F941D6218160CF03ACF80E090E83F
:10618000A9E4B3E431CF20E030E849E453E4C501A9
:10619000B4010F941D6218160CF03CCF80E090E81B
:1061A000A9E4B3E433CF20E030E047E453E4C7018F
:1061B000B6010F941D6218160CF03ECF80E090E0FF
:1061C000A7E4B3E435CF20E030E047E453E46A8D40
:1061D0007B8D8C8D9D8D0F941D6218160CF040CF19
:1061E00080E090E0A7E4B3E437CF0E94412697FD1A
:1061F0000CC00E9441266F3F71058105910509F091
:1062000034F40E944126862F089580E008958FEF90
:1062100008958091D0049091D104892B41F00E947F
:10622000F53091E0811101C090E0892F089591E04F
:10623000FCCF0E944126CB0108950F931F93CF936B
:106240008091D0049091D1040097E9F0FC018F0176
:10625000C1912C2F2F7D81F0C53411F0C536B9F7CF
:10626000F801108270E060E00F945A54F801C08386
:10627000CF911F910F91089570E060E0CF911F9131
:106280000F910D945A5460E070E0CB01F1CF2FEBE9
:10629000280F2A3108F047C0E22FF0E08091010575
:1062A00090910205A0910305B091040504C0B69534
:1062B000A795979587952A95D2F780FD02C08170A2
:1062C0000895E951FB4FE081EE2341F180916A0886
:1062D00090916B08E80FF92FF11D808190ED980FD8
:1062E0009A3030F08E3251F4818180538A3098F4A4
:1062F000F093D104E093D00481E008958D3211F041
:106300008B3249F4818190ED980F9A3088F38E3268
:1063100011F48281EACFF0E0E0E0EACF1092D104FC
:106320001092D004E9CF80E008950E94473188237D
:1063300041F081E02091D0043091D104232B09F465
:1063400080E00895CF93DF93EB010E94953188237D
:1063500019F00E944126EB01CE01DF91CF91089503
:10636000CF92DF92EF92FF926A017B010E949531FA
:10637000882331F0FF90EF90DF90CF900C941D3187
:10638000C701B601FF90EF90DF90CF9008954F9234
:106390005F926F927F928F929F92AF92BF92CF92B5
:1063A000DF92EF92FF921F93CF93DF9300D01F9263
:1063B000CDB7DEB719821A821B821C82CE010196EC
:1063C0004C0185EBC82E80E1D82E9CE4E92E98E0A4
:1063D000F92E27E6A22E29E0B22E10E088E5810FE3
:1063E0000E949531F40181934F01882341F00E946E
:1063F0001D312B013C0180916A10882359F0F60170
:1064000080819181A281B381F70180839183A283EE
:10641000B38314C0812F0E944A22882309F4D0C07C
:10642000F6012081318142815381C301B2010F9471
:10643000BD5FF70160837183828393831F5FF4E004
:10644000CF0ED11C84E0E80EF11C94E0A90EB11C23
:10645000133021F685E40E9495318C83882309F45A
:10646000B9C00E941D316B017C0183E00E944A2269
:10647000882371F02091C1103091C2104091C31057
:106480005091C410C701B6010F94BD5F6B017C0130
:10649000C0925808D0925908E0925A08F0925B08CE
:1064A0008091E005882359F18091D91682FF27C099
:1064B0008C81882321F18981811103C08A818823FD
:1064C000F1F02DEC3CEC4CE45DE36091BE08709182
:1064D000BF088091C0089091C1080F94BD5F9B01D7
:1064E000AC016091BD107091BE108091BF10909171
:1064F000C0100F941D62181614F40F94004640E06B
:1065000050E0BA0186E40E94B03120E030E0A901F9
:106510000F941D62181684F40E941D3120E030E0B3
:1065200040E752E40F94B760609380027093810259
:10653000809382029093830280916B1083FD2CC024
:1065400080916A10811128C08091C507882321F1AC
:106550002091C1103091C2104091C3105091C410CD
:10656000609158087091590880915A0890915B0881
:106570000F94BC5F2091D2073091D3074091D4078C
:106580005091D5070F94BD5F6093D2077093D307E6
:106590008093D4079093D5070F900F900F900F9092
:1065A000DF91CF911F91FF90EF90DF90CF90BF9040
:1065B000AF909F908F907F906F905F904F900895D5
:1065C000F5012081318142815381C301B2010F94D1
:1065D000BC5F2FCF8091C1109091C210A091C310C9
:1065E000B091C4108093580890935908A0935A080A
:1065F000B0935B0855CFCF93DF93EB010E949531A9
:10660000882321F0DF91CF910C941931CE01DF91D5
:10661000CF910895CF93DF93C82FD62F0E94953145
:10662000882321F0DF91CF910C9409318C2F0E94A7
:106630004731811101C08D2FDF91CF910895E5EB96
:10664000F8E082EBDF011D928A95E9F708958091C9
:10665000E005811104C00E941F330D94C54780914D
:10666000D91682FD0D94004608958091B5088823BF
:1066700061F090916609891308C08091D91683FF53
:1066800004C083EF98E00D94D04780E00895FC01AA
:10669000238121110C9478D70895CF92DF92EF9245
:1066A000FF920F931F93CF9390912402913009F49E
:1066B00061C0662351F01092AF041092AB041092A7
:1066C000AC041092AD041092AE04C82F0F94813B1D
:1066D000C090AB04D090AC04E090AD04F090AE0458
:1066E0009B01AC012C193D094E095F0969017A0132
:1066F000F7FC40C02091AF04C7FD15C04C2F0C2EF5
:10670000000C550B4C5F5F4FE22F022E000CFF0B6D
:106710004E175F077CF144EFC42EDD24D394E12CA7
:10672000F12C2C1734F438EEC32E33E0D32EE12CA9
:10673000F12CC60ED71EE81EF91EC092AB04D092F3
:10674000AC04E092AD04F092AE04022F017010E0B0
:1067500084E2809FB001819F700D701B11246059ED
:106760007C4F82E390E00E9494808091AF048F5F21
:106770008093AF04CF911F910F91FF90EF90DF9026
:10678000CF90089590912502911102C0811104C00B
:10679000809154028093AA04809108019111809500
:1067A00088708093060108950F931F9301E010E015
:1067B00020E030E0082E04C0000F111F221F331FFD
:1067C0000A94D2F74091150550911605609117056E
:1067D00070911805402B512B622B732B409315059C
:1067E0005093160560931705709318059091230236
:1067F000891303C081E080936A101F910F9108955F
:1068000010924506109246061092470610924806CE
:10681000E1EEF5E084E6DF011D928A95E9F708953F
:106820009091B4109817B1F00E94FEE18091B410DD
:10683000882341F085EB90E10E9421E21092B41090
:106840000C94F9F781E08093B41085EB90E10E94FD
:106850004AE1F6CF08954F925F926F927F928F92A6
:106860009F92AF92BF92CF92DF92EF92FF921F93CF
:10687000CF93DF93EC01162F20917F083091800891
:106880004091810850918208688179818A819B8139
:106890000F94CB58882309F4AEC0B090B41080E0B8
:1068A0000E941034C880D980EA80FB8020E030E06C
:1068B000A901C701B6010F941D6218161CF0C12C66
:1068C000D12C7601C0927F08D0928008E092810896
:1068D000F09282082DEB37E346E855EBC701B6018D
:1068E0000F941D6287FD0BC02DEB37E346E855E39F
:1068F000C701B6010F94CB5818160CF078C0A70149
:10690000960160E070E080E89FE30F94B7606093C9
:10691000C4057093C5058093C6059093C70580EFA5
:106920009FEFA9E7B4EC8093C8059093C905A093A5
:10693000CA05B093CB05BB2009F45DC04090B510EB
:106940005090B6106090B7107090B8108090B91049
:106950009090BA10A090BB10B090BC10C090BD1029
:10696000D090BE10E090BF10F090C01081E00E9467
:106970001034112309F43FC02091B5103091B610A6
:106980004091B7105091B810C301B2010F94CB5889
:1069900081111CC02091B9103091BA104091BB10E8
:1069A0005091BC10C501B4010F94CB5881110EC099
:1069B0002091BD103091BE104091BF105091C01079
:1069C000C701B6010F94CB588823A9F0DF91CF916E
:1069D0001F91FF90EF90DF90CF90BF90AF909F906E
:1069E0008F907F906F905F904F900D94B00060E01B
:1069F00070E0CB018CCFDF91CF911F91FF90EF9092
:106A0000DF90CF90BF90AF909F908F907F906F90CE
:106A10005F904F900895EF92FF920F931F93CF9343
:106A2000DF9301EE15E0C5E07801D5E0F701619153
:106A30007191819191917F0120E030E0A9010F9443
:106A4000CB5881110EC0D15089F7C1500C5E1F4F39
:106A5000C111EACFDF91CF911F910F91FF90EF907D
:106A6000089581E0F7CFEFE6F0E0808182608083D7
:106A700008958091600890916108892B79F4809144
:106A8000600890916108892B49F420916008309149
:106A9000610881E0232B19F480E0089581E00895D6
:106AA000CF92DF92EF92FF926B017C0183E3C816D5
:106AB000D104E104F10470F082E3C81AD108E108BE
:106AC000F10862E370E080E090E00F944E3B0E949A
:106AD000FBF7ECCFC701B6010F944E3BFF90EF9050
:106AE000DF90CF900C94FBF70F94813B6093C3042D
:106AF0007093C4048093C5049093C6048091DB070F
:106B000081110BC0999AA19881E08093DB076AEF0D
:106B100070E080E090E00C9450350895CF93DF93BF
:106B2000EC01892B39F00E947435CC38D10514F072
:106B3000CCE8D0E0D0938A08C0938908DF91CF9148
:106B40000C94B3CB8091640681110AC080917D08BA
:106B5000813041F08091D91682FB882780F9089511
:106B600080E0089581E008955F9A8091D9078E7F33
:106B70008093D9078A9A8091D9078D7F8093D9070E
:106B80008091080180958170809306018091D907DA
:106B90008B7F8093D9070C9480229091D91693FB18
:106BA000882780F993FF06C081E0909141189111E8
:106BB00001C080E0089580916406811110C0809129
:106BC0007D08823061F00E94CD35882349F08091A4
:106BD000D91682FB882780F991E08927089581E002
:106BE00008950E94DB3581110DC010921505109299
:106BF00016051092170510921805109219058FEFBF
:106C00000E9482240D941C04E5EAF9E010821182AE
:106C1000089581E008958F929F92AF92BF92CF9294
:106C2000DF92EF92FF920F93CF93DF931F92CDB736
:106C3000DEB75C017B0149016B01C40ED51EF50175
:106C4000808191810F94E95E8983002311F0F7011F
:106C50008083BE016F5F7F4FC4010F94922BF501BB
:106C600080819181019691838083FFEFEF1AFF0A63
:106C7000EC14FD0421F780E00F90DF91CF910F918C
:106C8000FF90EF90DF90CF90BF90AF909F908F904C
:106C900008959091C00095FFFCCF8093C6000895A1
:106CA000CF93DF93EC018991882319F00E94493634
:106CB000FACF8DE00E9449368AE0DF91CF910C94A3
:106CC0004936CF92DF92EF92FF92CF936B017C0116
:106CD000C42F4A3069F4F7FE0BC0F094E094D094CE
:106CE000C094C11CD11CE11CF11C8DE20E944936EC
:106CF0004C2FC701B601CF91FF90EF90DF90CF905E
:106D00000D946245CF93DF93EC01FE0184912196AF
:106D1000882319F00E944936F8CFDF91CF9108956A
:106D20000F931F93CF938C01C62F8AED92E10E949F
:106D30008236C8010E9482368AE30E94493680E387
:106D40008C0F0E9449368AE0CF911F910F910C94CD
:106D500049368DE594E10E94823660E08DE494E14D
:106D60000E94903660E088E394E10E94903661E0F2
:106D700081E394E10E94903661E086E294E10E9412
:106D8000903661E086E194E10E94903660E08DE00B
:106D900094E10E94903661E083E094E10E94903695
:106DA00060E089EF93E10E94903661E082EF93E129
:106DB0000E94903660E08AEE93E10E94903661E096
:106DC0008CED93E10E94903661E08EEC93E10E949D
:106DD000903661E08FEB93E10E94903661E081EBA9
:106DE00093E10E94903660E08BE993E10E94903637
:106DF00061E08AE893E10E94903661E08BE793E1DD
:106E00000E94903661E084E793E10E94903660E052
:106E10008DE693E10E94903661E084E693E10E9462
:106E2000903661E08FE493E10E94903661E081E466
:106E300093E10E94903661E08EE293E10E949036E9
:106E400060E081E293E10E94903661E08CE193E1A1
:106E50000E94903661E08FE093E10E94903660E0FE
:106E60008BEF92E10E94903660E088EE92E10E9402
:106E7000903660E08DED96E10E944722682F6170A8
:106E80008FED92E10C94903680910105827149F466
:106E9000809103058C7829F480910405837009F4AE
:106EA00075C082E40E944731882351F00E94202659
:106EB00060937C1070937D1080937E1090937F1070
:106EC00083E50E944731882351F00E941D31609371
:106ED000AC107093AD108093AE109093AF1084E51A
:106EE0000E944731882351F00E941D316093B010F9
:106EF0007093B1108093B2109093B31088E50E9404
:106F00004731882351F00E941D3160938D097093A1
:106F10008E0980938F099093900989E50E944731EB
:106F2000882351F00E941D3160939109709392095A
:106F300080939309909394098AE50E9447318823AE
:106F4000B1F00E941D31609395097093960980936A
:106F50009709909398092DEC3CEC4CEC5DE30F9471
:106F6000CB58181624F087E89EE00E94823685E40C
:106F70000E944731882351F00E941D316093990986
:106F800070939A0980939B0990939C0908950E949D
:106F9000493689E49DE00C9482360F931F93CF937A
:106FA0008C01C62F80EC99E00E948236C8010E94B5
:106FB0008236CC2331F08AE0CF911F910F910C944F
:106FC0004936CF911F910F9108950F931F93CF933F
:106FD0008C01C62F60E080ED99E00E94CD37C8019A
:106FE0000E948236CC2331F08AE0CF911F910F911D
:106FF0000C944936CF911F910F91089561E088ED6F
:1070000099E00C94E537EF92FF920F931F93CF9383
:107010007C018B01C42F60E080ED99E00E94CD37A8
:10702000C7010E94823680E20E944936C8010E9450
:107030008236CC2319F08C2F0E9449368AE0CF91FA
:107040001F910F91FF90EF900C944936DF92EF92D1
:10705000FF920F931F93CF93DF93D82E7B018A016A
:10706000E9010E94FE37D092640840E0B70183E94D
:1070700091E40E9403380115110531F040E0B80198
:107080008CE891E40E940338209731F040E0BE0183
:107090008CE891E40E94033861E087E891E4DF9195
:1070A000CF911F910F91FF90EF90DF900C94E537F7
:1070B00061E08AEC99E00C94CD37AF92BF92CF9209
:1070C000DF92EF92FF920F931F93CF93DF9385E9A7
:1070D00099E00E9482366091450670914606809143
:1070E00047069091480645E00F94620D82E899E0CA
:1070F0000E948236C0E0D9E0D15021F080E20E94A7
:107100004936FACF8C2F0F94C945CF5FC53099F718
:107110008AE00E94493601EE15E0C0E080E20E945C
:1071200049368C2F0F94C9455801D5E080E20E9462
:107130004936F501C080D180E280F380A701960135
:10714000C701B6010F94AF6281112CC020E030E07E
:10715000A901C701B6010F941D6287FD03C08BE230
:107160000E94493645E0C701B6010F94620DD15027
:1071700084E1A80EB11CD111D9CF8AE00E94493612
:10718000CF5F0C5F1F4FC53049F68AE0DF91CF918A
:107190001F910F91FF90EF90DF90CF90BF90AF9035
:1071A0000C944936F12C80E20E944936F3948DE329
:1071B000F8E0FF12F9CFDBCF811107C089EB9EE029
:1071C0000E9482368AE00C9449368DEB9EE0F8CF1F
:1071D000CF93DF93EB010E948236CE01DF91CF91F6
:1071E0000D94D045CF93C62F0E9482368C2FCF911D
:1071F0000D94C945CF92DF92EF92FF926A017B0115
:107200000E94823642E0C701B601FF90EF90DF9006
:10721000CF900D94620DCF92DF92EF92FF926A01B0
:107220007B010E9482364AE0C701B601FF90EF90D1
:10723000DF90CF900C9461362F923F924F925F92E5
:107240006F927F928F929F92AF92BF92CF92DF9276
:10725000EF92FF920F931F93CF93DF93CDB7DEB7DB
:10726000C654D1090FB6F894DEBF0FBECDBF70E093
:1072700060E085E40E94FB32182F8F3F09F483C041
:107280008823E9F087E197E1CA5BDF4F0FB6F894F6
:10729000DEBF0FBECDBFDF91CF911F910F91FF9049
:1072A000EF90DF90CF90BF90AF909F908F907F90A6
:1072B0006F905F904F903F902F900C94823624EB0C
:1072C00030E03A83298383E50E949531882321F0B9
:1072D0000E9419319A83898365E070E083E40E94FB
:1072E000FB328AA760E085E50E940A3325968FAFBE
:1072F000259760E08AE097E10E9434B7A981BA81BE
:10730000BD01BB0F880B990B0F94D2586D837E8300
:107310008F8327969FAF27970F94813B688B798B3C
:107320008A8B9B8B1F3F09F047C420E030E04CE084
:1073300053E46D817E818F8127969FAD27970F94AF
:107340001D6218160CF0AAC18FED96E10E948236DC
:10735000CA5BDF4F0FB6F894DEBF0FBECDBFDF9123
:10736000CF911F910F91FF90EF90DF90CF90BF9042
:10737000AF909F908F907F906F905F904F903F90D5
:107380002F900D94C04846E450E05A8349839BCF28
:107390001FAEB1C12496EEADFFAD2497808385C2A8
:1073A000FBEE4F2E512C612C712C06C384E190E032
:1073B000A0E0B0E08C8B9D8BAE8BBF8BE4E14E2EBA
:1073C000512C612C712C06C34C8A5D8A6E8A7F8A8F
:1073D00001C32496EEADFFAD24978083D6C3898187
:1073E0009A81AB81BC8129A93AA94BA95CA9821BCE
:1073F000930BA40BB50BB7FD59C08FAD0F94060EC0
:107400008AE00E94493689819A81AB81BC81805390
:10741000984FAF4FBF4F89AB9AABABABBCAB9DA9FD
:10742000911177C02EA93FA948AD59ADB101802F68
:1074300026969FAD26970F941D6218160CF053C028
:1074400020E030E040E050E4B101802F26969FAD6F
:1074500026970F94BD5F6EAB7FAB88AF99AF2CA51D
:107460003DA54EA55FA589819A81AB81BC81280F7E
:10747000391F4A1F5B1F2AAF3BAF4CAF5DAF20E007
:1074800030E040EC50E46D817E818F8127969FAD86
:1074900027970F94BC5F9101402F26965FAD2697EA
:1074A0000F94CB58881F8827881F8DAB88899989AE
:1074B000AA89BB89C816D906EA06FB0610F4D701CB
:1074C000C60129813A814B815C81281B390B4A0B0B
:1074D0005B0BDA01C90181389F44A241B105A8F1D3
:1074E0008BE296E110C289819A81AB81BC812AAD81
:1074F0003BAD4CAD5DAD821B930BA40BB50B4CE5C6
:1075000057E36BE677E3B7FDD1CF812F0E945EDBB7
:10751000CDCF20E030E040EF51E46D817E818F815E
:1075200027969FAD27970F94BC5F9B01AC01B101DB
:10753000802F26969FAD26970F94CB5887FFB6CF06
:1075400048E058E368E178E3E0CF4AA55BA5888D81
:10755000998D481759070CF09EC003970CF49BC0F7
:107560008EEC95E10E9482361F3F09F076C0AEEBAB
:10757000B5E1BA83A9838DEA95E10E9482368981BB
:107580009A810E948236488559856A857B858AEC76
:1075900095E10E94FA388AE00E9449368DEA95E129
:1075A0000E94823689819A810E94823649A15AA11D
:1075B0006BA17CA186EC95E10E94FA388AE00E94DA
:1075C00049368DEA95E10E94823689819A810E942E
:1075D0008236B501A40182EC95E10E94FA388AE076
:1075E0000E9449362596FFAD2597FF2391F12CEA9D
:1075F00035EC47E25EE369A17AA18BA19CA10F94CF
:1076000031596B017C012CEA35EC47E25EE3C501A0
:10761000B4010F94B760288539854A855B851F3F83
:1076200009F520938C0830938D0840938E08509371
:107630008F08C0929008D0929108E0929208F09240
:10764000930860939408709395088093960890939C
:10765000970881E0809369027BCEE1EDF0E4FA8344
:10766000E98389CF2093F0153093F1154093F215FB
:107670005093F315C092F415D092F515E092F615DB
:10768000F092F7156093F8157093F9158093FA1539
:107690009093FB15DECF0E94CEBB82C08BEC96E1AF
:1076A0000E9482360E9493DA0E9474358FE780939D
:1076B0008B0824EB30E0A8EEB3E00F94635F6CA777
:1076C0007DA78EA79FA7288939894A895B89260FBC
:1076D000371F481F591F2AAF3BAF4CAF5DAF109209
:1076E000690281E08093780232E0310F3EAF3230A0
:1076F00008F44ECE1FAFC888D988EA88FB88C9AA8B
:10770000DAAAEBAAFCAA812C912C540189A29AA294
:10771000ABA2BCA288869986AA86BB868FE790E03A
:10772000A0E0B0E08C8B9D8BAE8BBF8B1C8690E471
:107730009A8FACE1AB8FB6E4BC8F1D8E1E8E1F8E70
:1077400018A23FE7432E512C612C712C1DAA8EAA42
:107750009FAAA8AEB9AE1EA21FA218A619A6E1E064
:10776000EDA3198E188E212C312C00E026961FAE29
:107770002697F5E11F02C00111249C0129513A4EC0
:1077800022963FAF2EAF2297285F3F4F24963FAF00
:107790002EAF24974AA5042E000C550B5BA74AA7D1
:1077A00080917802882309F4B0C00F94813B6983EB
:1077B0007A838B839C835091620658AB552309F4DE
:1077C0008BC00E9446DB60918708709188081F3F3C
:1077D00039F02296AEADBFAD229714966D917C9193
:1077E000072E000C880B990B0F94D2581B01082F01
:1077F00026969FAF26972D8D3E8D4F8D58A12696AC
:107800009FAD26970F941D6218163CF42D8E3E8E68
:107810000F8F2696BFAD2697B8A32C853A8D4B8D3A
:107820005C8DB101802F26969FAD26970F94CB5883
:1078300087FF07C02C863A8E0B8F2696EFAD2697D2
:10784000EC8FFDA19101402F26965FAD26976D81AB
:107850007E818F8127969FAD2797FF2309F45AC019
:107860000F94CB5887FF38C049815A816B817C8146
:107870004C195D096E097F09DB01CA0188589341E3
:10788000A109B109B7FD28C08C899D89AE89BF893E
:1078900084199509A609B709B595A7959795879570
:1078A0001F3F09F077CD80938B084EA35FA368A795
:1078B00079A7FD81FD8F2E812E8F3F813F8F2796E7
:1078C0004FAD279748A389819A81AB81BC81888B72
:1078D000998BAA8BBB8B1DA220E030E040EF51E4D6
:1078E0006D817E818F8127969FAD27970F94BD5F15
:1078F0009101402F26965FAD26970F94CB5887FFB6
:107900006ECD89E496E10E948236109278020E9440
:1079100093DA9FCE0F941D621816F4F689819A812E
:10792000AB81BC81288939894A895B89821B930B89
:10793000A40BB50BAC01BD01485853416109710955
:1079400077FDCACF488D598D452B09F40DC1CEA0C6
:10795000DFA0E8A4F9A4C80ED91EEA1EFB1E2EA1C2
:107960003FA148A559A5281B390B4A0B5B0BC30146
:10797000B2010F94FF5EA70196010F94315F4C880E
:107980005D886E887F88420E531E641E751E54E10A
:1079900045165104610471040CF408CD8CEE4816B0
:1079A0005104610471040CF0FBCC90E849165104B9
:1079B000610471040CF408CD4C8A5D8A6E8A7F8A5A
:1079C0002EEF30E040E050E0241935094609570910
:1079D00029013A014C895D896E897F8983EC96E1A2
:1079E0000E940B39B301A2018EEB96E10E940B3984
:1079F0004C855A8D6B8D7C8D87EB96E10E94FA3811
:107A00004D8D5E8D6F8D78A180EB96E10E94FA38E6
:107A1000A88DB98D13970CF4A7C0C301B2010F94C0
:107A2000D25820E030E040E850E40F9431594B0147
:107A30005C012C853A8D4B8D5C8D6D8D7E8D8F8D8F
:107A400098A10F94BC5F2BED3FE049E450E40F9404
:107A5000315920E030E040E05FE30F9431599B0161
:107A6000AC01C501B4010F94B7606C877D878E8728
:107A70009F87C701B6010F94D2582FE632E143E841
:107A80005AE30F9431596B017C011E3F59F02AE9EA
:107A900039E949E15FE3812C912CA12C6EE3B62EEC
:107AA0001F3F59F42DEC3CEC4CE45EE37BEA872E5F
:107AB0007AEA972EA92C7EE3B72E6C857D858E857C
:107AC0009F850F943159688779878A879B879B01A7
:107AD000AC010F94BD5FA70196010F94B76069A335
:107AE0007AA38BA39CA3288539854A855B85C7012A
:107AF000B6010F943159A50194010F9431594B01EE
:107B00005C014C855D856E857F858AEA96E10E94E1
:107B1000FA38B701A60184EA96E10E94FA388AE0B1
:107B20000E944936BEAD85E996E1B23010F086E894
:107B300096E10E948236488559856A857B8580E872
:107B400096E10E94FA3849A15AA16BA17CA18AE76B
:107B500096E10E94FA38B501A40184E796E10E94FB
:107B6000FA388AE00E9449368C899D89AE89BF899E
:107B7000840D951DA61DB71DB595A795979587955D
:107B80001F3F09F026CC80938B08288D398D2F5FFD
:107B90003F4F398F288F3D813C874E814A8F5F81CF
:107BA0005B8F27968FAD27978C8FC980DA80EB800B
:107BB000FC8098A99DA390CEE12E012E000CFF0819
:107BC000F70183E0EE0FFF1F8A95E1F7E059FD4FC3
:107BD000668177816F507109072E000C880B990B15
:107BE0000F94D2589B01AC016D817E818F812796C5
:107BF0009FAD27970F941D6218160CF4A5CB8BEC44
:107C000096E10E9482360E9493DA0E94743585E1E3
:107C10008E9DF0018F9DF00D1124E951FA4E8FE7F2
:107C2000808722E330E047CDCF93DF93EB010E94C2
:107C30008236CE01DF91CF910D94B12C2F923F92DD
:107C40004F925F926F927F928F929F92AF92BF926C
:107C5000CF92DF92EF92FF920F931F93CF93DF9318
:107C6000CDB7DEB7C058D1090FB6F894DEBF0FBE4E
:107C7000CDBF84ED9CE00E9482360F94E2488111D2
:107C80008FC084E50E949531882329F00E94193124
:107C900081110E9449DA80E090E0A0E8BFE3898387
:107CA0009A83AB83BC838D839E83AF83B8878DEC2F
:107CB0009CECACE4BEE389879A87AB87BC8780E005
:107CC00090E0A0E2B1E48D879E87AF87B88B8CE30C
:107CD00090E09A8B898B8DEC90E09C8B8B8B8DEC5C
:107CE0009CECACECBEE38D8B9E8BAF8BB88F80E0B1
:107CF00090E0A0EEBFE3898F9A8FAB8FBC8F1BA65D
:107D00001CA64AE959E969E97EE38FE40E94B03193
:107D10006D8F7E8F8F8F98A360E083E40E940A337B
:107D200089A360E08BE40E940A338AA389E40E945D
:107D3000953110E0F12CE12C8823C1F00E94F53040
:107D400090E01816190614F481E090E011E0180F85
:107D5000212F2150330BC90126E0289FF001299FD4
:107D6000F00D1124E05EF74FE280F38082E40E9480
:107D70009531882319F00E9419317C01E114F10436
:107D800059F1C70188978536910520F16CE870E0BC
:107D900086EA9CE00E94143E81EA9CE00E948236C2
:107DA000C058DF4F0FB6F894DEBF0FBECDBFDF91D6
:107DB000CF911F910F91FF90EF90DF90CF90BF90E8
:107DC000AF909F908F907F906F905F904F903F907B
:107DD0002F900895FA8AE98A8CE40E9495318823CD
:107DE000E1F00E941D316B017C01C986DA86EB86C9
:107DF000FC8620E030E0A9010F941D6287FD0AC0D7
:107E000020E030E040E050E4C701B6010F94CB58C9
:107E100018161CF489E79CE0C1CF81E50E94473128
:107E2000882331F18091D0049091D104892BE9F01D
:107E30000E941D316B017C01CD82DE82EF82F886CB
:107E40002DEC3CEC4CE45DE30F941D6287FD0AC011
:107E500020E030E040E751E4C701B6010F94CB5871
:107E6000181634F488E49CE099CF8DE19CE096CF1D
:107E700083E50E9495318823E9F00E941D316B0152
:107E80007C01CD8ADE8AEF8AF88E2DEC3CEC4CEC3E
:107E90005DE30F941D6287FD0AC020E030E040E002
:107EA00050E4C701B6010F94CB5818161CF486EFA6
:107EB0009BE074CF80E50E944731882341F0809198
:107EC000D0049091D104892B29F58FEF8BA786E4FC
:107ED0000E949531882309F43DC00E941D316B0139
:107EE0007C01C98EDA8EEB8EFC8E20E030E040E81B
:107EF0005FE30F941D6287FD0AC020E030E040E898
:107F000050E4C701B6010F94CB5818161CF585EA4A
:107F10009BE044CF8BA58F5F8BA70E941D316B0127
:107F20007C01CD86DE86EF86F88A20E030E0A9016C
:107F30000F941D6287FD0BC020E030E048EC51E457
:107F4000C701B6010F94CB5818160CF0C0CF8EECB9
:107F50009BE024CFC98CDA8CEB8CFC8C8D889E88BE
:107F6000AF88B88CA7019601C701B6010F943159AB
:107F70009B01AC0160E070E084E490E40F94B76092
:107F800029813A814B815C810F9431592B013C014D
:107F9000A5019401C501B4010F943159A7019601BF
:107FA0000F9431592CEE31E548EB5DE30F94B76047
:107FB0009B01AC01C301B2010F94315969837A83EB
:107FC0008B839C83112309F1412F4150550B26E0EF
:107FD000249FF001259FF00D1124E05EF74F0081F2
:107FE000118188E40E949531882319F00E9419318B
:107FF0008C010115110571F0C801855A9109883865
:10800000910530F087E79BE0C9CE10E000E0E9CFB2
:108010001C8B0B8B85E50E9447318823C9F00F9498
:10802000813B611571058105910511F00F94515443
:108030008091D0049091D104892BC9F00E941D3108
:108040006093CC047093CD048093CE049093CF04BE
:108050006AE170E082E50E94FB32E5969FAF8EAF49
:10806000E5971816190644F083E49BE097CE60E08C
:1080700070E088E492E4E4CF89E50E94953188239A
:1080800009F40AC10E941D3120916B0930916C09DD
:1080900040916D0950916E090F94BC5F4B015C01DA
:1080A00088E50E949531882309F4FFC00E941D31A4
:1080B00020916709309168094091690950916A09D6
:1080C0000F94BC5F6B017C01CBA2DCA2EDA2FEA2EF
:1080D0008FA298A6A9A6BAA627E137EB41ED58EBE7
:1080E000C501B4010F941D6287FDE8C027E030E8A8
:1080F0004AE453E4C501B4010F94CB5818160CF4AC
:10810000DDC027E137EB41ED58EBC701B6010F9415
:108110001D6287FDD3C027E030E048E453E4C70187
:10812000B6010F94CB5818160CF4C8C084E40E9412
:10813000473111E081270E94103480E090E0A0EAEE
:10814000B0E48DA79EA7AFA7B8ABCE018D960F94D4
:10815000423450919C08EC965FAFEC9710929C08CB
:108160000E9433C986EC9AE00E94823689899A89F6
:108170004A970CF0A6C063E683EA9AE00E9434B7FF
:108180000F94BA3B8B899C890E9477E141E061E0C2
:1081900080E00F94FE0F882309F4A6C00F94C04816
:1081A0000F94BA3B1092C1101092C2101092C310DB
:1081B0001092C41081EC90E10E94F1F31BA51123F1
:1081C00009F4F5C020E030E040E751E460919C10F4
:1081D00070919D1080919E1090919F100F94B760A8
:1081E00021966CAF7DAF8EAF9FAF21971F3F09F0F7
:1081F000F9C481E08093120563E68BEF9AE00E9458
:1082000034B768E873E182E090E00E94948080E1F6
:10821000E5EBF0E1ACE4B8E001900D928A95E1F76E
:10822000CE0101960F949D34C12CD12C7601809102
:10823000770982FDB1C068E873E182E090E00E94B6
:10824000948020E030E040E85EE36091580870914F
:10825000590880915A0890915B080F94BD5F609314
:1082600058087093590880935A0890935B0820E04F
:1082700030E040E85EE3C701B6010F94BD5F6B01DB
:108280007C0120E030E84BE354E40F941D6287FD4D
:1082900073C01092120528C08090B9109090BA1047
:1082A000A090BB10B090BC10FBCEC090B510D09089
:1082B000B610E090B710F090B81006CF89E19BE0BF
:1082C0006DCD63E686EB9AE00E9434B70F94BA3B1B
:1082D0001093120589899A890E948E3561E081E0A8
:1082E0000F94790E811147CF6FEF8DE09BE00E94D4
:1082F00034B78CA5811112C081E08CA78D819E813D
:10830000AF81B885B0588DA79EA7AFA7B8ABBE0107
:10831000635D7F4F8CE498E00E94502D80E090E0F8
:10832000A0EAB0E48093540890935508A0935608AF
:10833000B09357081DA61EA61FA618AABE01635D0E
:108340007F4F8CE498E00E94502DEC965FADEC9747
:1083500050939C080E9433C9109212058AA1811182
:108360001FCD10928A08109289080E94B3CB90E02A
:1083700080E00E9477E114CDCE01CD960E94F8FEF8
:1083800080E1E5EBF0E1ACE4B8E001900D928A9574
:10839000E1F70E94FEE14BCF0E948BBE63E68EEEBA
:1083A0009AE00E9434B70F94BA3B10921205E7ECA2
:1083B000F4E085E0DF011D928A95E9F780E1E5EBC5
:1083C000F0E1ACE4B8E001900D928A95E1F789857F
:1083D0009A85AB85BC858093540890935508A093EB
:1083E0005608B09357081DA61EA61FA618AABE01C0
:1083F000635D7F4F8CE498E00E94502DBE01635E68
:108400007F4F8CE498E00E94502D81E0809312050C
:1084100089A1882309F43CC42091B5103091B6108D
:108420004091B7105091B810AC962CAF3DAF4EAF05
:108430005FAFAC978091B9109091BA10A091BB102A
:10844000B091BC10E0968CAF9DAFAEAFBFAFE097E0
:10845000AAEBB6E1A196BFAFAEAFA197312C212C0C
:10846000BFEF6C96BFAF6C97EFEFA496EFAFA497FA
:10847000FFEFE396FFAFE3972FE4EA962FAFEA977B
:1084800033ECEB963FAFEB9707E481E090E0A0E0A0
:10849000B0E0022C04C0880F991FAA1FBB1F0A94CA
:1084A000D2F7C458DF4F88839983AA83BB83CC5704
:1084B000D040A7ECB4E0E296BFAFAEAFE297E6EAF9
:1084C000F6E1A396FFAFEEAFA39710E0C058DF4FE1
:1084D0002882C058D040E296AEADBFADE2978D91F4
:1084E000E296BFAFAEAFE29790E0B0E0A0E0C45834
:1084F000DF4F288139814A815B81CC57D04082236C
:108500009323A423B523892B8A2B8B2B09F0E5C059
:10851000A196AEADBFADA197CD90DD90ED90FC9052
:10852000A396AEADBFADA3972D913D914D915C91BA
:10853000A8962CAF3DAF4EAF5FAFA897A7019601AD
:10854000AC966CAD7DAD8EAD9FADAC970F94BC5F1E
:108550002B013C01A8962CAD3DAD4EAD5FADA8976B
:10856000E0966CAD7DAD8EAD9FADE0970F94BC5F96
:108570004B015C01A3019201C301B2010F94315977
:108580002B013C01A5019401C501B4010F9431599F
:108590009B01AC01C301B2010F94BD5F0F946B62EC
:1085A0004B015C01A70196016BA17CA18DA19EA14D
:1085B0000F94BC5F6B017C01A8962CAD3DAD4EAD18
:1085C0005FADA8976FA178A589A59AA50F94BC5F08
:1085D0002B013C01A7019601C701B6010F94315947
:1085E0006B017C01A3019201C301B2010F943159C7
:1085F0009B01AC01C701B6010F94BD5F0F946B6284
:1086000020E030E040E751E40F94B760A501940109
:108610000F94BD5F6B017C018090CC049090CD04E1
:10862000A090CE04B090CF0420E030E040E85FE3BB
:10863000C501B4010F941D621816F4F4C501B4010C
:108640000F9429614B015C0160E070E0CB011814CC
:1086500019041A041B0434F40F940254A501940164
:108660000F94315F0F94D2589B01AC01B601C70142
:108670000F94BD5F6B017C01E3962FADE397EA9603
:108680003FADEA97EB964FADEB97502FB601C70180
:108690000F94CB5887FF21C06C961FAF6C97C058C2
:1086A000DF4FB881C058D040A496BFAFA497E696DC
:1086B000CFAEE697E796DFAEE797E896EFAEE8979E
:1086C000E996FFAEE997E396CFAEE397EA96DFAE81
:1086D000EA97EB96EFAEEB970F2D1F5FA396EEADEB
:1086E000FFADA3973496A396FFAFEEAFA3971530D7
:1086F00009F0F1CEFFEF2F1A3F0AA1962EAD3FAD44
:10870000A1972C5F3F4FA1963FAF2EAFA19735E0C9
:108710002316310409F0B9CE6C964FAD6C97E42F57
:10872000F0E0E953FB4F208181E090E0A0E0B0E071
:10873000A4960FACA49704C0880F991FAA1FBB1F53
:108740000A94D2F7822B8083A4965FADA497629699
:108750005FAF629763964FAF6397E6968FADE697EC
:10876000E7969FADE797E896AFADE897E996BFAD7E
:10877000E99767968CAF9DAFAEAFBFAF67975F3F8E
:1087800009F414C24F3F09F411C284E04802F00119
:108790001124EA55F94E108101813280238027E1AE
:1087A00037EB41ED58EB612F702F832D922D0F94F5
:1087B0001D6287FDFFC127E030E84AE453E4612FE2
:1087C000702F832D922D0F94CB5818160CF4F2C1F4
:1087D000A4969FADA497A4E09A02F0011124E65458
:1087E000F94EC080D180E280F38027E137EB41ED84
:1087F00058EBB601C7010F941D6287FDDBC127E06E
:1088000030E048E453E4B601C7010F94CB58181682
:108810000CF4D0C120E030E040EA50E4B601C701DA
:108820000F94BD5FA0966FAFA097A2967FAFA2975F
:10883000A5968FAFA597A9969FAFA997CB01A596AF
:10884000AFADA597A996BFADA99721968CAF9DAF67
:10885000AEAFBFAF2197812F902FA32DB22D2596BC
:108860008CAF9DAFAEAFBFAF2597A496BFADA49719
:10887000B11150C26C96EFAD6C97E11118C220E0B7
:1088800030E040EA50E4612F702F832D922D0F9439
:10889000BD5FA4966FAFA497AD967FAFAD97E196FD
:1088A0008FAFE197E3969FAFE3976C96FFAD6C9720
:1088B000FF2309F4F1C26C963FAD6C97A096CFAE42
:1088C000A097A296DFAEA297A596EFAEA597A99620
:1088D000FFAEA99734300CF014C222ED822E23E5AE
:1088E000922E2BE7A22E21E4B22E21964CAC5DAC49
:1088F0006EAC7FAC219725962CAD3DAD4EAD5FADF6
:1089000025976F962CAF3DAF4EAF5FAF6F97A3012A
:108910009201B601C7010F94BC5F2D966CAF7DAF7D
:108920008EAF9FAF2D976F962CAD3DAD4EAD5FAD29
:108930006F97612F702F832D922D0F94BC5F6196DE
:108940006CAF7DAF8EAF9FAF6197A3019201609135
:10895000B5107091B6108091B7109091B8100F9427
:10896000BC5F2B013C016F962CAD3DAD4EAD5FADB4
:108970006F976091B9107091BA108091BB1090916F
:10898000BC100F94BC5F6F966CAF7DAF8EAF9FAF86
:108990006F97A0968FADA097A2969FADA297A59630
:1089A000AFADA597A996BFADA9978DA79EA7AFA775
:1089B000B8ABA4968FADA497AD969FADAD97E19659
:1089C000AFADE197E396BFADE39789AB9AABABABA5
:1089D000BCABC984DA84EB84FC84CDAADEAAEFAAFE
:1089E000F8AE2DEC3CEC4CEC5CE3C501B4010F940B
:1089F000315929813A814B815C810F943159209101
:108A0000C1103091C2104091C3105091C4100F9406
:108A1000BD5F69AF7AAF8BAF9CAFA3019201C30179
:108A2000B2010F9431592B013C016F962CAD3DAD35
:108A30004EAD5FAD6F97CA01B9010F9431599B01DB
:108A4000AC01C301B2010F94BD5F20E030E040E013
:108A500050E40F941D621816ACF420E030E040E0C2
:108A60005FE3C701B6010F94BD5F29966CAF7DAF80
:108A70008EAF9FAF2997BE01635C7F4FCE010196F9
:108A80000E94592D89859A85AB85BC8529968CAF26
:108A90009DAFAEAFBFAF29976B961CAE1DAE1EAE9D
:108AA0001FAE6B97BE01695A7F4FCE01CD960E94D3
:108AB000502DCE0101960F949D34A0909410B0904B
:108AC0009510C0909610D0909710E0909010F09074
:108AD000911000919210109193109701A801B50187
:108AE000C6010F941D62181614F07501860180905E
:108AF000800290908102A0908202B09083022DECBF
:108B00003CEC4CEC5DE3B701C8010F943159609324
:108B1000800270938102809382029093830240E0EE
:108B2000BE01675B7F4FCE018D960F947B3C80E149
:108B3000E5EBF0E1ACE4B8E001900D928A95E1F745
:108B40008092800290928102A0928202B09283026F
:108B50000E9430268111C8CB20E04FEFBE016F5A32
:108B60007F4FCE0101960E941C2F20E041E0BE0104
:108B70006F5A7F4FCE0101960E941C2F2FEF40E0CD
:108B8000BE016F5A7F4FCE0101960E941C2F21E03B
:108B900040E0BE016F5A7F4FCE0101960E941C2F0C
:108BA0000E94FEE10E94302681119ECB8091C5106B
:108BB0008093C610E5964EAD5FADE59741505109E3
:108BC000E5965FAF4EAFE597452B09F48DCB6296E6
:108BD0008FAD629787FD88CB63968FAD639787FFD4
:108BE00017CC82CB63E68BED9AE00E9434B70F94EA
:108BF000BA3B80E1E5EBF0E1ACE4B8E001900D9226
:108C00008A95E1F72D853E854F85588960915808F2
:108C10007091590880915A0890915B080F94BD5F3C
:108C2000609358087093590880935A0890935B0892
:108C3000CE01CD960E94F8FE2D853E854F85588940
:108C4000609158087091590880915A0890915B087A
:108C50000F94BC5F609358087093590880935A082A
:108C600090935B088CA58111A2CB81E08CA78D81AC
:108C70009E81AF81B885B0588DA79EA7AFA7B8AB2E
:108C8000BE01635D7F4F8CE498E00E94502D8FCB36
:108C90002BA13CA14DA15EA1AC962CAF3DAF4EAF38
:108CA0005FAFAC978FA198A5A9A5BAA5CBCBC601FC
:108CB000D70121968CAF9DAFAEAFBFAF219720E01B
:108CC00030E040EA50E4612F702F832D922D0F94F5
:108CD000BC5F25966CAF7DAF8EAF9FAF25976C962E
:108CE0002FAD6C9724300CF4CACDA4961FAFA49777
:108CF000AD960FAFAD97E1963FAEE197E3962FAEFD
:108D0000E39792ED892E93E5992E9BEFA92E90E49F
:108D1000B92EEBCDA4964FADA49744300CF46EC0A1
:108D20006C965FAD6C975430BCF120E030E040EAC7
:108D300050E4B601C7010F94BC5F21966CAF7DAFC4
:108D40008EAF9FAF219720E030E040EA50E4612FE2
:108D5000702F832D922D0F94BC5FA4966FAFA497B4
:108D6000AD967FAFAD97E1968FAFE197E3969FAF5A
:108D7000E3976C969FAD6C97A096CFAEA097A29606
:108D8000DFAEA297A596EFAEA597A996FFAEA997DD
:108D900094300CF0B6CFA1CDC601D70121968CAF8F
:108DA0009DAFAEAFBFAF219720E030E040EA50E486
:108DB000612F702F832D922D0F94BD5F25966CAF80
:108DC0007DAF8EAF9FAF25976C968FAD6C9781115D
:108DD000BACF20E030E040EA50E4B601C7010F947A
:108DE000BC5FA0966FAFA097A2967FAFA297A59603
:108DF0008FAFA597A9969FAFA99777CF6C96AFAD88
:108E00006C97A1112BC020E030E040E251E4A09625
:108E10006FADA097A2967FADA297A5968FADA597AF
:108E2000A9969FADA9970F94BC5FA0966FAFA0972E
:108E3000A2967FAFA297A5968FAFA597A9969FAF51
:108E4000A997A4961FAFA497AD960FAFAD97E196E3
:108E50003FAEE197E3962FAEE3973FCD6C96BFAD63
:108E60006C97B43034F120E030E040E251E4A09659
:108E70006FADA097A2967FADA297A5968FADA5974F
:108E8000A9969FADA9970F94BC5F21966CAF7DAF5B
:108E90008EAF9FAF2197D5CFA096CFAEA097A296C9
:108EA000DFAEA297A596EFAEA597A996FFAEA997BC
:108EB00028CFA4961FAFA497AD960FAFAD97E196BC
:108EC0003FAEE197E3962FAEE39782ED882E83E5E0
:108ED000982E8BEFA82E81E4B82E07CD8BE799E072
:108EE0000C948236CF92DF92EF92FF920F931F93F2
:108EF000CF93DF9388E50E944731D82E89E40E9402
:108F00004731C82E8823D1F10E941931D82F89E525
:108F10000E944731182F8AE40E944731082F882386
:108F200009F455C00E941931C82F8AE50E944731C3
:108F3000E82EF12C811104C081E50E944731F82E02
:108F4000C11001C000E0802F90E0D11001C010E0FE
:108F5000810F911D019721F4E11062C0F11060C0F2
:108F60000E946E4787E69EE0DF91CF911F910F919F
:108F7000FF90EF90DF90CF900C948236D11002C01A
:108F8000DFEFC5CF0E941D3120916709309168093C
:108F90004091690950916A090F94BC5F20E030E06C
:108FA00040EA51E40F94BC5F20E030E040EA51E435
:108FB0000F94BD5F2DEC3CEC4CEC5CE30F9431590D
:108FC0000F942961D62F653008F4A1CFD9CF1111A4
:108FD00002C0CFEFAACF0E941D3120916B093091C2
:108FE0006C0940916D0950916E090F94BC5F20E0AF
:108FF00030E040EA51E40F94BC5F20E030E842EA00
:1090000051E40F94BD5F24E336EA49EC5CE30F942E
:1090100031590F942961C62F653008F486CFD9CF16
:10902000D7FD02C0C7FF05C00E946E478EE49EE0D8
:109030009BCF0E941D319B01AC010D2FDD0F110B49
:10904000AC2FCC0FBB0B60E070E0CB01FF2091F0A8
:1090500065E0609FF001619FF00D1124EA0FFB1F96
:10906000EE0FFF1FEE0FFF1FEF51FA4F608171816E
:1090700082819381E5E0E09FE001E19FD00D112422
:10908000CA0FDB1FCC0FDD1FCC0FDD1FCF51DA4F16
:109090000F94BD5F688379838A839B83DF91CF912F
:1090A0001F910F91FF90EF90DF90CF90089585E78B
:1090B00099E00C948236CF9384E50E949531C0E00C
:1090C0008823D9F00E94F530C82F1816B4F40E94F6
:1090D00057488DE40E944936809106059091070516
:1090E0000F94D0456C2FCC0F770B81E89FE00E9446
:1090F000143E8AE00E944936CFEF8C2FCF9108951D
:109100004F925F926F927F928F929F92AF92BF9297
:10911000CF92DF92EF92FF92CF93DF93CDB7DEB77E
:109120002C970FB6F894DEBF0FBECDBF40906709F5
:10913000509068096090690970906A0920913A021C
:1091400030913B0240913C0250913D02C301B2017B
:109150000F94BD5F69837A838B839C8380906B09B6
:1091600090906C09A0906D09B0906E0920913E021C
:1091700030913F024091400250914102C501B4013B
:109180000F94BD5F6D837E838F839887C0906F0936
:10919000D0907009E0907109F0907209209142021C
:1091A000309143024091440250914502C701B601FB
:1091B0000F94BD5F69877A878B879C8720914602D1
:1091C000309147024091480250914902C301B201D7
:1091D0000F94BD5F2B013C0120914A0230914B025C
:1091E00040914C0250914D02C501B4010F94BD5FF6
:1091F0004B015C0120914E0230914F024091500290
:1092000050915102C701B6010F94BD5F6B017C0103
:109210000E94574882ED9EE00E94823683E50E94BC
:109220004731882321F00E940931809338028091D0
:109230003802811151C089EB9EE00E9482368AEC8F
:109240009EE00E94823649815A816B817C818EE248
:109250009DE20E94FA384D815E816F8178858FE3AF
:1092600092E40E94FA3849855A856B857C858CE3A7
:1092700092E40E94FA3888EC9EE00E94823680ECEC
:109280009EE00E948236B301A2018EE29DE20E941E
:10929000FA38B501A4018FE392E40E94FA38B701CD
:1092A000A6018CE392E40E94FA388AE02C960FB66D
:1092B000F894DEBF0FBECDBFDF91CF91FF90EF904E
:1092C000DF90CF90BF90AF909F908F907F906F90E6
:1092D0005F904F900C9449368DEB9EE0AECF2F926D
:1092E0003F924F925F926F927F928F929F92AF9236
:1092F000BF92CF92DF92EF92FF920F931F93CF9383
:10930000DF93CDB7DEB76A970FB6F894DEBF0FBE16
:10931000CDBF83E50E944731182F3090B4108823C9
:1093200019F00E940931382E4090B5105090B610B7
:109330006090B7107090B8108091B9109091BA10E9
:10934000A091BB10B091BC108B8B9C8BAD8BBE8B56
:109350008091BD109091BE10A091BF10B091C0102F
:109360008F8B988FA98FBA8F112329F0311003C0EA
:1093700080E00E94103486E50E944731888B0E946D
:109380000B35882309F4BFC083E40E94473188234A
:1093900009F498C00E941D316B017C01A1EEB5E07B
:1093A000BF83AE83B987A887F5E0FD831D861E863F
:1093B00028EC2F8702EC1A86212C88EC8B8792E40C
:1093C0009C87A885B985BA8BA98B15E0E989FA89AC
:1093D00081909190A190B190FA8BE98B2A85322DE2
:1093E0004B855C85C501B4010F94CB5887FF04C041
:1093F0008A86292CAB86BC862D853E854F85502FCD
:10940000C501B4010F941D62181624F48D869E8642
:10941000AF860B2D1150D1F6FD81F150FD8388856B
:109420009985449699878887F111CBCF2D853E8504
:109430004F85502F6A85722D8B859C850F94BD5F5B
:1094400020E030E040E05FE30F943159A70196013E
:109450000F94BD5F6B017C012DEB37E346E855EBC4
:109460000F941D6287FD0AC02DEB37E346E855E3F4
:10947000C701B6010F94CB58181624F580E00E945E
:10948000103415E0AE80BF8005E0D5016D917D916F
:109490008D919D915D014D01B4E08B1A9108A7015A
:1094A00096010F94BC5FF401608371838283938380
:1094B000015059F711508E819F8144969F838E836E
:1094C0001111E0CFA889AA2351F00E940B358823FF
:1094D00031F084E29DE00E9482360E945D388AE588
:1094E0000E944731882359F00E941D3169837A8395
:1094F0008B839C8360E0CE0101960E942B34832DE8
:109500000E9410340BC0311003C09889992339F39D
:109510000E9457488AE39DE00E948236332051F032
:109520008091B410811106C00E946E4785E09DE0D5
:109530000E9482360E94574887EF9CE00E94823644
:109540008091B4100E94DC380E9457488AEE9CE05B
:109550000E948236C0907F08D0908008E0908108F9
:10956000F090820820E030E0A901C701B6010F9415
:109570001D6218160CF053C042E0C701B6010F94EB
:10958000620D8DE00E9449368AE00E944936A301AF
:1095900092016091B5107091B6108091B7109091C2
:1095A000B8100F94CB5881111FC02B893C894D896D
:1095B0005E896091B9107091BA108091BB10909142
:1095C000BC100F94CB5881110FC02F89388D498D55
:1095D0005A8D6091BD107091BE108091BF10909116
:1095E000C0100F94CB5881110F94B0006A960FB63B
:1095F000F894DEBF0FBECDBFDF91CF911F910F91C9
:10960000FF90EF90DF90CF90BF90AF909F908F90A2
:109610007F906F905F904F903F902F90089585EED0
:109620009CE00E948236B3CFCF93C82F82E0C11155
:1096300084E040E060E00E9497880E9457488DEEE9
:1096400099E0CC2311F082E09AE0CF910C9482361D
:10965000FF920F931F93CF93DF93EC018B01F42EB6
:109660000E9493DA0E946E4785E599E00E94823657
:109670000115110511F401ED10E4209711F4CCE46B
:10968000D9E00E947EBE1F930F93DF93CF938CE3AC
:1096900099E09F938F9381E08F930E9419B70E9466
:1096A000AE87C0916C16C695C69587E696E10E9476
:1096B0005528DC2FDD0F1D2F1C0FEDB7FEB7379699
:1096C0000FB6F894FEBF0FBEEDBF83E00E943927AE
:1096D0004CE753E16C2F80E00E94002B1092A21601
:1096E000D093A3168DE299E00E94E5281092A2166D
:1096F0001093A31680E299E00E94E5288BE696E19C
:109700000F9474438111E1CF61E083E499E00E94FA
:10971000CD3789EE93E030E6019729F0232F2A9583
:109720000000E9F7F9CFF89489EE93E038EE01975D
:1097300029F0232F2A950000E9F7F9CF0E9493DA48
:10974000FF2051F00E94B4350E9464220E948222C0
:10975000909905C0A895FCCF0E948022F5CF909BE0
:1097600002C0A895FCCFF0E0E0E0DF91CF911F911F
:109770000F91FF9019945F926F927F928F929F92B8
:10978000AF92BF92CF92DF92EF92FF920F931F930F
:10979000CF93DF931F92CDB7DEB77C0139018B01E8
:1097A0005B01A40EB51ED12CC12CA016B10609F484
:1097B00050C0F70180809180F80151908F0159824B
:1097C000C4010F94E95E5816B9F1652DC4010F94D8
:1097D000F15EFFEFCF1ADF0AC6018F779927892B39
:1097E00021F162E070E080E090E00F944E3BC40114
:1097F0000F94E95E99818917F9F00E9457488FE725
:1098000096E00E94823681E00F90DF91CF911F9108
:109810000F91FF90EF90DF90CF90BF90AF909F900F
:109820008F907F906F905F90089562E070E080E08D
:1098300090E00E945035DBCFBE016F5F7F4FC301C8
:109840000F94922BF70180819181019691838083FF
:10985000ACCF80E0D9CF8091C5109091C6102FEF8A
:109860003FEF981751F0E92FF0E0EB53FF4E2281C4
:1098700030E09F5F9F779093C610C90108951F92B3
:109880000F920FB60F9211240F900FBE0F901F90E2
:1098900018951F920F920FB60F9211240BB60F92CC
:1098A0000F931F932F933F934F935F936F937F93E8
:1098B0008F939F93AF93BF93CF93DF93EF93FF93D8
:1098C000C091C6000091C610D091C51011E01D0FC7
:1098D0001F7790918504913108F09FC0E92FF0E047
:1098E0008827EA58F34B8F4F0D94B45F874CB64CE2
:1098F000C54CD44CDB4C0D4DDF4C0D4DE34CE74CCF
:109900000D4DEB4CEF4CF34CFA4C0D4D054DC03268
:1099100029F028F5CA3011F0CD3031F5011731F0BA
:10992000ED2FF0E0EB53FF4EC283D12FD093C51043
:10993000FF91EF91DF91CF91BF91AF919F918F9167
:109940007F916F915F914F913F912F911F910F9157
:109950000F900BBE0F900FBE0F901F901895CD3437
:1099600081F081E0CE3471F080E10CC0CA3338F46C
:10997000C033A0F6C03291F2CD32B1F7CFCFCD34A3
:1099800099F782E080938504C9CFC13359F018F468
:10999000C03221F2E9CF88E0C433A1F38BE0C833B1
:1099A00089F3E2CF83E0EECF84E0C03359F386E061
:1099B000C13341F3D9CF85E0C833B1F6E3CF87E0B7
:1099C000C23391F6DFCF89E0C13371F6DBCF8AE095
:1099D000C03351F6D7CF8CE0C73331F6D3CF8DE00B
:1099E000C63311F6CFCFC03209F498CF8EE0C3351D
:1099F00049F2BACF80ED8C0F8A3008F08FCF9FE00C
:109A0000909385048093840489CFCA3019F0CD30B7
:109A100009F084CF1092850481CFCA3019F0CD307F
:109A200009F07CCF8091A5168823A1F3973041F1EE
:109A300038F4953079F71092780210926708EACFDF
:109A40009A3011F19F3031F790918404809164082D
:109A500010926408823089F38430E9F08130D1F6C5
:109A60009923B1F09130B1F682E08093660880913D
:109A70006508882379F2109259020E946D22CACF9C
:109A800081E080935706C6CF81E080935606C2CF0F
:109A900080936608BFCF89EC9EE19093DD078093A9
:109AA000DC07B8CF8EBD0DB407FEFDCF08958FEF54
:109AB0008EBD0DB407FEFDCF8EB508959091640064
:109AC0009B7F90936400982F906A96959CBD80FD33
:109AD00003C091E0863009F490E09DBD0895CF93D6
:109AE000DF93EB010E948236CE01DF91CF910C947F
:109AF00010D4AF92BF92CF92DF92EF92FF920F936A
:109B00001F93CF93DF93CDB7DEB7E6970FB6F894E8
:109B1000DEBF0FBECDBF0091090510910A05F80107
:109B200001900020E9F731976F01C01AD10AF801BE
:109B3000CF01801B910B8C159D053CF481918F32D8
:109B4000B9F7DF0111971C92F3CF8BE1EAEFF6E151
:109B5000DE015C9601900D928A95E1F7F12CE12CE3
:109B6000EC14FD040CF05DC0F801EE0DFF1D8081CA
:109B7000811103C08FEFE81AF80A5801AE0CBF1C20
:109B8000F5018081882309F44CC0FFEFEF1AFF0A2A
:109B9000F801EE0DFF1D7F01E01AF10A819181119C
:109BA000FACFCE014C960E9476D88BE1FE017C96CE
:109BB000DE01119601900D928A95E1F7B501CE0173
:109BC00001960E9482D0CE0101960E9447338FE217
:109BD0000E9449368091391381113BC083E693E09E
:109BE0000E9410D48091D91684FF1BC019821C8258
:109BF00021E0A501BE01645E7F4FCE0101960F9466
:109C0000830B811129C08AE00E9449360E9457487F
:109C1000B5018DE595E10E946F4DCE0101960E9440
:109C200047338AE00E944936CE014C960E94473362
:109C3000E6960FB6F894DEBF0FBECDBFDF91CF9191
:109C40001F910F91FF90EF90DF90CF90BF90AF905A
:109C5000089589E393E1C4CFCE014C960E9478D752
:109C60008BE1FE013196DE015C9601900D928A95A2
:109C7000E1F7CE0101960E94473372CF2F923F92B7
:109C80004F925F926F927F928F929F92AF92BF920C
:109C9000CF92DF92EF92FF920F931F93CF93DF93B8
:109CA00000D000D000D01F921F92CDB7DEB7B82EE3
:109CB0008091B211843008F0D1C10F94813B6B01C7
:109CC0007C018091B211811108C08091C5109091E2
:109CD000C610891B8F7709F44CC781E6A82E13C0E4
:109CE0008A3019F08D3009F0F6C01092AD118091D4
:109CF0004B1190914C11FC01E95BFE4E1682892BB1
:109D0000F1F40E94FBF78091B211843008F0ECC0AE
:109D10008091C5109091C610891B8F7709F4E4C01B
:109D20000E942B4C97FFDCCF0E946E4785EC97E09A
:109D30000E9482368091C5108093C610E4CF1092A5
:109D40004C1110924B110DE411E1F8018191803218
:109D500009F446C08E3409F0A9C060EC77E0C80170
:109D60000F9448584C01892B41F06EE470E0C80113
:109D700004960F940B63009709F4C8014AE050E081
:109D800070E060E001960F94B8552B013C01809182
:109D9000471190914811A0914911B0914A11019633
:109DA000A11DB11D481659066A067B0629F060E020
:109DB0008DE897E0892851F16AE270E0C8010F94BC
:109DC0003A639C01009729F1982F901B912C9923BD
:109DD00049F09150F801E90FF11D80819826F7CFE5
:109DE0008F01B3CF4AE050E070E060E0C901019616
:109DF0000F94B855292D30E050E040E0621773070A
:109E00008407950751F060E08EE697E00F94C72F26
:109E10007ACF60E084E497E0F9CF40924711509206
:109E200048116092491170924A1180911F08813047
:109E3000E1F067E470E0C8010F940B630097A9F0AC
:109E40004AE050E070E060E001960F94B85564304D
:109E500071058105910548F483EA96E00E948236F7
:109E600060E089E996E00E9434B7C0926C08D09215
:109E70006D08E0926E08F0926F0880914D118B335F
:109E800009F441CF8091B211843008F03CCF809129
:109E9000B4118A9DC00111246DE471E18B549E4E72
:109EA0000F94166380E00F94812F2DCF8091D916E7
:109EB00080FFBBCF64E570E4C8010F944858009759
:109EC00031F0FC01838180538A3008F0AECF60E02E
:109ED0008AE197E09BCF2BE431E14DE451E16DEA5B
:109EE00071E10E94F3210FCF8091D91682FFB6C095
:109EF0001A82198271E6F72EE0E1EE2EF9E6DF2EE6
:109F00008091B211843008F0A9C00E942B228111E7
:109F1000A5C041E050E0BE016B5F7F4F8EE398E14A
:109F20000E94B0D40D8110E0019711F00FEF1FEFE8
:109F30008091461890914718A0914818B0914918FF
:109F40008093D5169093D616A093D716B093D816B3
:109F50000E942B220F3F100749F4811107C00E9475
:109F60006E4783EE97E00E948236CACF4091B411CB
:109F7000242F30E00A3061F00D3051F0882309F4CD
:109F80005FC089819A81009719F001969A8389832D
:109F90001092860489819A81F29EF001F39EF00D61
:109FA0001124EE54FE4EE80FF91F1382892B69F538
:109FB0000E94FBF70E942B22882309F4A1CF0E9464
:109FC000FEE18EE398E10E9478D78091D016882335
:109FD00091F181508093D0168D9DC001112462E0D3
:109FE000865B984F0F948049E091D01624E0E29F61
:109FF000F0011124EA5BF84F6081718182819381C5
:10A000000E9474240E94EBCF7BCF1A82198281E0D8
:10A010000F94812F8091D5169091D616A091D716C6
:10A02000B091D8168093AE119093AF11A093B01158
:10A03000B093B111BFCF0E9481D7E0921F0860CFCB
:10A040004F9DA00111244B545E4E9E012F5F3F4F48
:10A0500066E874E0802F0E94F32152CF0F94813B79
:10A060006B017C01B11004C080916406882351F01B
:10A07000C0925C08D0925D08E0925E08F0925F08A2
:10A08000BB24B3948091E2049091E304A091E40492
:10A09000B091E5040097A105B10551F140915C082C
:10A0A00050915D0860915E0870915F08840F951F64
:10A0B000A61FB71FA7019601281B390B4A0B5B0B84
:10A0C000DA01C901B7FD14C00E946E4760916A08A9
:10A0D00070916B088EE398E00E946F4D8AE00E94B9
:10A0E000493640E070E060E090E080E00E94284B5C
:10A0F0008091100290911102A0911202B09113026E
:10A10000892B8A2B8B2B79F090912F16809130160A
:10A11000981709F4F9C1C0925C08D0925D08E092EA
:10A120005E08F0925F0880919B0490919C04909946
:10A130002DC2019690939C0480939B0480919B0474
:10A1400090919C048E3E92406CF00E946E478BE191
:10A1500098E00E94823640E070E060E090E080E0AD
:10A160000E94284B0F94813B009187041091880432
:10A170002091890430918A044B015C01801A910A74
:10A18000A20AB30A9501840137FD39C08B019C01F5
:10A190000C53164F2F4F3F4F0093870410938804A2
:10A1A0002093890430938A042091A509211125C0A8
:10A1B0002091A609211121C04F9B1FC07A9B1DC071
:10A1C0002091060120FF19C0029B17C02091ED15B8
:10A1D0003091EE151216130684F02091EF1521111F
:10A1E0000CC02091890830918A08121613062CF0B1
:10A1F00020918B08222309F4CFC10E9474350F945B
:10A20000813B4B015C0180916708811108C020915E
:10A210002F169091301681E0291301C080E0209123
:10A22000EB153091EC1591E089272A3A31050CF4B1
:10A2300080E091E040918F045091900460919104EE
:10A2400070919204452B462B472B09F490E0981708
:10A2500089F0882309F4BAC1D501C4018056944419
:10A26000A24FBF4F80938F0490939004A0939104CA
:10A27000B09392044090C1105090C2106090C310EF
:10A280007090C41020918B0430918C0440918D0407
:10A2900050918E04C301B2010F94CB58882319F159
:10A2A00080918F0490919004A0919104B0919204B8
:10A2B00040928B0450928C0460928D0470928E04B4
:10A2C000892B8A2B8B2B09F449C0D501C4018056F8
:10A2D0009444A24FBF4F80938F0490939004A09317
:10A2E0009104B093920480918F0490919004A09176
:10A2F0009104B09192040097A105B10579F1881AF3
:10A30000990AAA0ABB0AB7FC29C010928F041092BE
:10A310009004109291041092920486E098E00E94BA
:10A32000823660E082EF97E00E9434B78091ED15AD
:10A330009091EE151816190624F490E080E00E9422
:10A3400077E18091890890918A081816190634F4EB
:10A3500010928A08109289080E94B3CB80919704CA
:10A3600090919804A0919904B0919A04A701960144
:10A37000281B390B4A0B5B0BDA01C901B7FDC2C1BF
:10A3800020912F16909130168091670240916802BB
:10A39000291320C19091A509899FC0011124880F1C
:10A3A000892F881F990B91958D838091A609489FCD
:10A3B000C0011124880F892F881F990B91958E83D6
:10A3C0000F94813B69837A838B839C8340E0BE0139
:10A3D0006F5F7F4FCE0105960E9452E26D8170E063
:10A3E00089E00F94783A41E0BE016F5F7F4FCE0164
:10A3F00005960E9452E26E8170E087E00F94783AF1
:10A4000080916306882309F470C100913402109191
:10A410003502C80102972091ED153091EE152817ED
:10A4200039070CF462C1809030168F821886198625
:10A430001A861B8680912F169F80891509F4E4C027
:10A44000892D90E03BE6A32EA89EF001A99EF00D79
:10A450001124E654F64F458956896789708D452B3E
:10A46000462B472B81F4418D528D638D748D452B86
:10A47000462B472B41F4458D568D678D70A1452B9A
:10A48000462B472BE1F12BE6B22EB89E9001B99EE8
:10A49000300D1124A9014654564F1A01FA01618169
:10A4A0007281838194810F946B624B015C01F10195
:10A4B00061A172A183A194A10F94D0582B013C01FA
:10A4C000F10165A176A187A190A50F94D0589B01B9
:10A4D000AC01C301B2010F94B760A50194010F94C0
:10A4E00031594B015C01288539854A855B850F947C
:10A4F0001D62181624F488869986AA86BB868F81E9
:10A500008F5F8F708F8396CFBB2019F010929D04C0
:10A510000ACE0F94813B00915C0810915D08209158
:10A520005E0830915F088090100290901102A09018
:10A530001202B0901302080D191D2A1D3B1D601B4D
:10A54000710B820B930B97FDE1CF80919D048111DC
:10A55000EACD81E080939D045F9A8091D9078E7F38
:10A560008093D9078A9A8091D9078D7F8093D907E4
:10A570008091080180958170809306018091D907B0
:10A580008B7F8093D9070E948022CDCD18161906A3
:10A590000CF0D4CD0197CECD0091C3041091C4042A
:10A5A0002091C5043091C60401151105210531051E
:10A5B00051F0601B710B820B930B6053754781093F
:10A5C000910997FD1CCE0E94642219CE80E090E094
:10A5D000DC0148CE209130165BE6259F90011124C6
:10A5E0002654364FF901EF59FF4F9081899FC001E2
:10A5F0001124880F892F881F990B91958D832E59CF
:10A600003F4FF9018081D3CEB801110F880B990B10
:10A610000F94D2585B018C0120912E0230912F02B1
:10A620004091300250913102688579858A859B85F9
:10A630000F9431599501A8010F94BD5F2B013C0186
:10A6400080903202909033029B01AC01B501C801A9
:10A650000F941D62181694F0B401990C880B990B95
:10A660000F94D2585B018C019B01AC01B201C30174
:10A670000F941D62181614F0520183014090930448
:10A680005090940460909504709096049501A801F0
:10A69000C301B2010F941D621816B4F428E431EE20
:10A6A0004AE75FE3C301B2010F94315920E037ED6F
:10A6B00043EA5CE30F94BD5F9B01AC01B501C801A7
:10A6C0000F9431595B018C01C501D801809393042B
:10A6D00090939404A0939504B0939604B501C80197
:10A6E0000F942961CB010E9477E1F4E6CF0ED11CD3
:10A6F000E11CF11CC0929704D0929804E092990456
:10A70000F0929A040E94FBF780911F08882309F4B5
:10A71000F0C180915902882309F471C080916508C5
:10A7200081116DC00E94A235811105C0809164061F
:10A73000882309F464C0F894649910C0809155028C
:10A7400090915602A0915702B091580280934E0604
:10A7500090934F06A0935006B093510660914E0619
:10A7600070914F068091500690915106789420E0A8
:10A7700030E0A9010F94CB5887FF41C001E000935E
:10A78000650880916406811138C00E94FE370093ED
:10A79000640840E36AEA78E083E991E40E940338C0
:10A7A00061E087E891E40E94E5371091E60460E0FB
:10A7B000102788E79AE069F488E998E00E94CD378D
:10A7C00080E30E9449368AE00E94493660E08BE7C8
:10A7D00098E00E94CD3786E898E00E94823680E3B8
:10A7E0000E9449368AE00E944936112331F081E8FF
:10A7F00098E09093DD078093DC070E94FEE1909142
:10A800000901892F8095817010910802811709F440
:10A810005AC02091D91620622093D916809308023D
:10A8200090FD10C064EF71E080E090E00E94503530
:10A830000E94A3D78091D91683FDBEC1112309F4CC
:10A8400042C002C00E9492D7123008F46BC100E0EF
:10A850000E947B2783E0809384020F94813B6C5994
:10A860007F4F8F4F9F4F60930E0570930F0580931E
:10A87000100590931105002331F1123021F58091DC
:10A88000D91683FF20C00F94BA46882379F081E05F
:10A890000F94D64542EB50E065EB78E08FED96E102
:10A8A0000E94B0D48FED96E10E9478D70E94353394
:10A8B000811144C10E941F330F94C54781E08093EA
:10A8C000CF160F9407480F94813B6B017C011091C8
:10A8D0000F021123F1F0809168088823D1F0409194
:10A8E0009E0450919F046091A0047091A1044601C0
:10A8F0005701841A950AA60AB70AB501A40177FD83
:10A900001AC0833009F430C10CF01FC181300CF043
:10A9100024C1212F30E0A8EEB3E00F94635FC60E90
:10A92000D71EE81EF91EC0929E04D0929F04E092AA
:10A93000A004F092A10480917D08813009F073C0D9
:10A940000F94813B6B017C018091A6049091A70438
:10A95000A091A804B091A904A7019601281B390B66
:10A960004A0B5B0BDA01C901B7FD3AC0D701C6013A
:10A97000805F984DAF4FBF4F8093A6049093A7047C
:10A98000A093A804B093A9048090D4059090D50515
:10A99000A090D605B090D7050F945A03AB01BC0127
:10A9A0004093D4055093D5056093D6057093D70591
:10A9B0008091CA079091CB07A091CC07B091CD07A9
:10A9C00088199909AA09BB09840F951FA61FB71FEB
:10A9D0008093CA079093CB07A093CC07B093CD0781
:10A9E0008091A2049091A304A091A404B091A50425
:10A9F00046015701881A990AAA0ABB0AD501C4015F
:10AA0000B7FD11C020E8C20E2EEED21E26E3E21ED4
:10AA1000F11CC092A204D092A304E092A404F0928C
:10AA2000A5040E94F9E00F94EB070E94CEBB809131
:10AA3000E104882379F10F94813B6B017C018091C3
:10AA4000DD049091DE04A091DF04B091E0044601A2
:10AA50005701881A990AAA0ABB0AD501C401B7FD91
:10AA600019C02091E10430E0A8EEB3E00F94635FD9
:10AA7000C60ED71EE81EF91EC092DD04D092DE0479
:10AA8000E092DF04F092E00480E00F94060E8AE08A
:10AA90000E9449368091DC04882359F10F94813B50
:10AAA0006B017C018091D8049091D904A091DA04C3
:10AAB000B091DB04A7019601281B390B4A0B5B0BF5
:10AAC000DA01C901B7FD15C02091DC0430E0A8EE21
:10AAD000B3E00F94635FC60ED71EE81EF91EC09246
:10AAE000D804D092D904E092DA04F092DB040F94F7
:10AAF000DD462B960FB6F894DEBF0FBECDBFDF91BB
:10AB0000CF911F910F91FF90EF90DF90CF90BF906A
:10AB1000AF909F908F907F906F905F904F903F90FD
:10AB20002F90089560E08BEB98E00E9434B78091FD
:10AB30001C0581118CCE0E94AE8789CE88ED98E0ED
:10AB40009093DD078093DC07BECE843009F0E1CE20
:10AB50000E9457488FED98E004C00E9457488EE04D
:10AB600099E00E948236D5CE0E94574887EF98E040
:10AB7000F8CF80916C0890916D08A0916E08B0910B
:10AB80006F08A7019601281B390B4A0B5B0BDA01F2
:10AB9000C901885E9340A109B109B7FD9EC88DED3A
:10ABA00097E00E948236C0926C08D0926D08E092C5
:10ABB0006E08F0926F0891C8123028F460E089ECBA
:10ABC00098E00E9434B701E043CECF93DF93C82FC3
:10ABD000D62F80916B1083FD14C08091B70981112D
:10ABE00010C08091890290918A02AC0141505109B4
:10ABF0002091ED153091EE152417350714F40E94BD
:10AC000077E140E06D2F8BE00E949788CC2339F0EC
:10AC100040E061E080E0DF91CF910D94FE0F8091E4
:10AC2000B70991E089278093780280917802882380
:10AC300089F08091EB159091EC152091ED153091F4
:10AC4000EE15821B930B97FF03C091958195910997
:10AC5000029744F41092780280916B1083FF06C033
:10AC6000C1E01AC080E00E943E4EDFCFC091B7091C
:10AC7000C11112C08091890290918A02019720919E
:10AC8000ED153091EE152817390754F70E945748F3
:10AC90008CED99E00E9482368C2FDF91CF91089540
:10ACA000AF92BF92CF92DF92EF92FF920F931F93DA
:10ACB000CF93DF93CDB7DEB764970FB6F894DEBFBE
:10ACC0000FBECDBF0E945B48D82E87FDB5C08AE578
:10ACD0000E949531882309F4C0C040E050E0BA01D9
:10ACE0008AE50E94B0317B018C014D2D63E085E047
:10ACF0000E9497882091BD103091BE104091BF10E6
:10AD00005091C01060E070E082E593E40F94BC5F66
:10AD10005B016C019701A8010F941D62181614F0D5
:10AD20007501860120E030E0A901B701C8010F9448
:10AD30001D62181624F4E12CF12C00E010E0B7019C
:10AD4000C8010F942961072E000C880B990B0F94F2
:10AD5000D2586D837E838F83988720E030E0A901ED
:10AD60000F94CB58882321F0CE0105960E94C2246F
:10AD700080E090E0A0EAB1E489879A87AB87BC873E
:10AD80001D861E861F86188A8CE40E944731882300
:10AD900009F468C00E941D316B017C0120E030E0A5
:10ADA000A901C701B6010F941D6287FF04C0F7FA1D
:10ADB000F094F7F8F094C98ADA8AEB8AFC8A209139
:10ADC000ED153091EE152430310574F08091EB15BE
:10ADD0009091EC15821B930B97FF03C09195819581
:10ADE000910901E004970CF400E063E080E00E9428
:10ADF000E555811140C083E08093240210921B0529
:10AE00000E94AE876D817E818F8198858B019C0128
:10AE1000305809831A832B833C8320E030E0A9015A
:10AE20000F94CB58882321F0CE0101960E94C224B2
:10AE300010921B050E94AE8764960FB6F894DEBF91
:10AE40000FBECDBFDF91CF911F910F91FF90EF907B
:10AE5000DF90CF90BF90AF900895E12CF12C00E2ED
:10AE600011E443CFC090DC05D090DD05E090DE0515
:10AE7000F090DF0593CF83E0E82E22E0AE01475F3C
:10AE80005F4FBE016F5E7F4FCE010D960F94633210
:10AE9000B9CF6F927F928F929F92AF92BF92CF92D3
:10AEA000DF92EF92FF920F931F93CF93DF9300D027
:10AEB00000D01F921F92CDB7DEB75C014B013A0163
:10AEC000F22E680100915C06109258061092590605
:10AED00010925A0610925B0610925C060F948D3BFE
:10AEE0008091ED159091EE158C159D051CF4C60111
:10AEF0000E9477E160E080E00E94E55581112FC15A
:10AF000010921B050E94AE871C141D0444F4C60158
:10AF10000E9477E140E060E080E00F94FE0F40E0A7
:10AF200060E088E00E94978860E081E00E94E5553B
:10AF300080E090E0A0E7B2E489839A83AB83BC838E
:10AF400080E090E0A0E8B0EC8D839E83AF83B8876B
:10AF5000BE016F5F7F4FCE0105960E94C9F787E063
:10AF60000E9409F6811158C08091BD109091BE10C9
:10AF7000A091BF10B091C0104091B7045091B80497
:10AF80006091B9047091BA04C090B304D090B40435
:10AF9000E090B504F090B604C0924C08D0924D08F1
:10AFA000E0924E08F0924F08409350085093510899
:10AFB00060935208709353088093540890935508F7
:10AFC000A0935608B093570880E090E0A8E4B2E45C
:10AFD00089839A83AB83BC83CE0101960E94F8FEDD
:10AFE0008091BB049091BC04A091BD04B091BE04BB
:10AFF0008093540890935508A0935608B09357082F
:10B0000080E090E0A0EAB0E489839A83AB83BC83BC
:10B01000CE0101960E94F8FEC12CD12C80E7E82ECB
:10B0200082E4F82EC982DA82EB82FC8280E090E032
:10B03000A0E8B0E48D839E83AF83B887BE016F5FC5
:10B040007F4FCE0105960E94C9F720E030E0A901AC
:10B050006091BF047091C0048091C1049091C204BA
:10B060000F94CB5887FF0BC0C982DA82EB82FC8237
:10B07000BE016F5F7F4F8FEB94E00E94C9F7809114
:10B08000BF049091C004A091C104B091C204809308
:10B09000C1109093C210A093C310B093C4108093BA
:10B0A000580890935908A0935A08B0935B0888E514
:10B0B00098E00E94F1F38091E00581110F94004621
:10B0C00010921B050E94AE8761E085E89AE00E941D
:10B0D000CD37809164068150809364064AE85EE132
:10B0E0006DE87AE085E00F946D33809164068823E3
:10B0F00039F00E94EBCF8091640681508093640602
:10B100008091B204882351F01092B2048091B0046F
:10B110008093A5098091B1048093A6090E946D22B5
:10B1200080917D08823011F40F941C040F94C04864
:10B130000E94AE8728960FB6F894DEBF0FBECDBF33
:10B14000DF91CF911F910F91FF90EF90DF90CF9003
:10B15000BF90AF909F908F907F906F900895E12C5B
:10B160002F2DA301B401C5010F946332CDCE4F92B0
:10B170005F926F927F92AF92BF92CF92DF92EF92E7
:10B18000FF921F93CF93DF9300D000D01F921F92A6
:10B19000CDB7DEB75C01E62EF42E642F80E00E946E
:10B1A000E555182F81111BC0EE2021F010921B05D0
:10B1B0000E94AE87812F28960FB6F894DEBF0FBE8F
:10B1C000CDBFDF91CF911F91FF90EF90DF90CF9097
:10B1D000BF90AF907F906F905F904F900895EE205A
:10B1E00029F040E06F2D83E00E94978880E090E096
:10B1F000A0E7B2E48D839E83AF83B88780E090E0C0
:10B20000A0E8B0EC89839A83AB83BC83BE016B5FFB
:10B210007F4FCE0101960E94C9F768E873E180E094
:10B2200090E00E945035C12CD12C88ECE82E81E4AE
:10B23000F82ECD82DE82EF82F88680E090E0A0E8F2
:10B24000B0E489839A83AB83BC83BE016B5F7F4F7D
:10B25000CE0101960E94C9F74090A4105090A5100D
:10B260006090A6107090A710C092A410D092A51064
:10B27000E092A610F092A71080E090E0A0E2B2E485
:10B280008D839E83AF83B887F50180819181A281F0
:10B29000B38189839A83AB83BC83BE016B5F7F4F8D
:10B2A000CE0101960E94C9F74092A4105092A510B9
:10B2B0006092A6107092A710129A64E670E080E087
:10B2C00090E00E94503576CFBF92CF92DF92EF92FE
:10B2D000FF920F931F93CF93DF9300D01F92CDB7B0
:10B2E000DEB77C016B018A01B22E61E088E79AE04B
:10B2F0000E94CD374AE85EE16FE77AE085E00F947F
:10B300006D339091640681E0890F8093640680918B
:10B31000D91682FF06C08B7F8093D9169E5F9093CB
:10B3200064060F94540480E1E5EBF0E1A3EBB4E094
:10B3300001900D928A95E1F70E94FEE18091B2049E
:10B3400081110FC081E08093B2048091A5098093A0
:10B35000B0041092A5098091A6098093B1041092BF
:10B36000A60920E030E0A901F701608171818281A6
:10B3700093810F94CB588823F1F08091B709811104
:10B380000CC08091890290918A0201972091EB155F
:10B390003091EC152817390774F080E090E0A0E7B1
:10B3A000B2E489839A83AB83BC83BE016F5F7F4F16
:10B3B000C7010E94C9F787E00E9409F6811103C006
:10B3C000B6010F94300720E030E0A901F801608158
:10B3D0007181828193810F94CB58882329F042E0B8
:10B3E0006B2DC8010E94B758129A64E670E080E0A5
:10B3F00090E00E94503581E00F900F900F900F90D9
:10B40000DF91CF911F910F91FF90EF90DF90CF9040
:10B41000BF900895CF92DF92EF92FF92CF93DF9388
:10B420006B017C01D42FC091680883E08093680889
:10B4300081E080936708C114D104E104F10431F084
:10B440000F94813BC60ED71EE81EF91E8091670837
:10B45000882389F0C114D104E104F10421F48D2F73
:10B460000E943E4EF3CF0F94813B6C197D098E09EB
:10B470009F0997FDF4CF10926708C0936808DF9189
:10B48000CF91FF90EF90DF90CF9008951F93CF93CF
:10B49000DF93D82FC62F0E94144B61E08C2F0E949F
:10B4A0004D330F94813B685370458F4F9F4F60938E
:10B4B00058067093590680935A0690935B06109233
:10B4C0005C061091680883E08093680830E020E013
:10B4D00048EB51E46AE67AE082E00E94263881E097
:10B4E0008093670880916708882309F463C060E04F
:10B4F0008C2F0E944D3380915C06882309F456C03E
:10B5000040E060E08AE00E9497880E94574880E50A
:10B510009AE00E94823630E020E04AE35AE061E49B
:10B520007AE082E00E94263841E060E070E0CB01E2
:10B530000E940A5A30E020E050E040E06DE27AE0FC
:10B5400085E00E94263810925806109259061092F3
:10B550005A0610925B0610925C060F948D3B60E0D9
:10B5600080E00E94E5558D2F0E94144B0F94813B83
:10B57000685370458F4F9F4F6093580670935906DC
:10B5800080935A0690935B0610925C0630E020E0B0
:10B5900048EB51E461E27AE082E00E94263881E0E3
:10B5A0008093670861E08C2F0E944D3381E00E94F8
:10B5B0003E4E98CF10936808DF91CF911F91089568
:10B5C000CF92DF92EF92FF920F931F93CF93DF936F
:10B5D000CDB7DEB7A0970FB6F894DEBF0FBECDBFD4
:10B5E0000E945B4887FDD1C0482F61E081E00E9446
:10B5F000978885E40E944731882309F4D5C00E94CA
:10B600001D316B017C0120E030E0A9010F941D6227
:10B6100087FF04C0F7FAF094F7F8F094F7FAF09483
:10B62000F7F8F094C98ADA8AEB8AFC8A8CE0EFE8B2
:10B63000F2E0DE01119601900D928A95E1F78AE51C
:10B640000E949531882351F040E050E0BA018AE52C
:10B650000E94B03169877A878B879C8788E50E9432
:10B660009531882351F040E050E0BA0188E50E940E
:10B67000B03169837A838B839C8389E50E949531FD
:10B68000882351F040E050E0BA0189E50E94B031D2
:10B690006D837E838F83988785E50E944731882359
:10B6A00009F489C00E941D316B017C0120E030E06B
:10B6B000A901C701B6010F941D6287FF04C0F7FA04
:10B6C000F094F7F8F094F7FAF094F7F8F094CD8A44
:10B6D000DE8AEF8AF88E198E1A8E1B8E1C8E8CE4F1
:10B6E0000E944731882309F46FC00E941D316B010D
:10B6F0007C0120E030E0A901C701B6010F941D6272
:10B7000087FF04C0F7FAF094F7F8F094CD8EDE8E40
:10B71000EF8EF8A262E070E082E40E94FB32F82E25
:10B7200080916406811131C021E0AE014B5E5F4F14
:10B73000BE016F5F7F4FCE0141960E9464598823FE
:10B7400021F16F2D81E00E94465A82E50E949531D9
:10B75000882309F442C00E94193140E050E060EAB9
:10B7600071E44D875E876F87788B20916406222372
:10B7700061F08C012F2DAE01435F5F4FBE01635E10
:10B780007F4FCE0149960E944957A0960FB6F89474
:10B79000DEBF0FBECDBFDF91CF911F910F91FF9004
:10B7A000EF90DF90CF900895C12CD12C80E8E82E47
:10B7B00080E4F82E33CFC090D805D090D905E09022
:10B7C000DA05F090DB0572CFC090DC05D090DD0586
:10B7D000E090DE05F090DF058CCF90E080E0BDCFFB
:10B7E000CF92DF92EF92FF920F931F93CF93DF934D
:10B7F000CDB7DEB76C970FB6F894DEBF0FBECDBFE6
:10B800008CE40E944731882309F4C3C00E941D3193
:10B810006B017C0120E030E0A9010F941D6287FFDD
:10B8200004C0F7FAF094F7F8F094F7FAF094F7F808
:10B83000F094C98EDA8EEB8EFC8E8CE0EFE8F2E0AD
:10B84000DE01119601900D928A95E1F788E50E943C
:10B8500095318823A1F040E050E0BA0188E50E94CC
:10B86000B031209167093091680940916909509180
:10B870006A090F94BC5F69837A838B839C8389E513
:10B880000E9495318823A1F040E050E0BA0189E59B
:10B890000E94B0312091670930916809409169098F
:10B8A00050916A090F94BC5F6D837E838F83988764
:10B8B0008AE50E949531882351F040E050E0BA01BA
:10B8C0008AE50E94B03169877A878B879C87F090E0
:10B8D000D916F2FAFF24F0F840E061E080E00E941F
:10B8E000978860E080E50E940A33E82E1D861E8658
:10B8F0001F86188A8091640681113CC02E2DAE01EE
:10B90000435F5F4FBE016F5F7F4FCE0149960E943C
:10B910006459882379F18091E00581110F940046E4
:10B92000FF2011F0EE2031F160E080E00E94465AE5
:10B93000898D9A8DAB8DBC8DB0588D8B9E8BAF8BC6
:10B94000B88F198A1A8A1B8A1C8A1D861E861F8632
:10B95000188A80916406882369F010E000E020E0F6
:10B96000AE014B5E5F4FBE016F5E7F4FCE010D9605
:10B970000E9449576C960FB6F894DEBF0FBECDBF3C
:10B98000DF91CF911F910F91FF90EF90DF90CF90BB
:10B990000895C12CD12C80E8E82E80E4F82E45CF04
:10B9A0002F923F924F925F926F927F928F929F92CF
:10B9B000AF92BF92CF92DF92EF92FF920F931F93BD
:10B9C000CF93DF93CDB7DEB7E1970FB6F894DEBF24
:10B9D0000FBECDBF89AB2091680828AB21E0209332
:10B9E0006808809108058D3409F463C4843511F426
:10B9F0000C94EE71873409F044C180910605909152
:10BA000007058A31910509F4D7C108F03DC184309A
:10BA1000910508F030C120911F088230910508F48B
:10BA200051C1213009F054C111E0029709F010E032
:10BA30000E94C73119821A821B821C821D821E82BB
:10BA40001F82188682E50E949531882309F453C12C
:10BA50000E941D316B017C0120E030E0A9010F94B0
:10BA6000CB58882309F4EAC04090B5105090B61026
:10BA70006090B7107090B8108091B9109091BA1082
:10BA8000A091BB10B091BC1088A799A7AAA7BBA78B
:10BA900080904C0890904D08A0904E08B0904F08B0
:10BAA0008091500890915108A0915208B09153088C
:10BAB0008CA79DA7AEA7BFA7A5019401C301B201A2
:10BAC0000F94CB5881110DC02CA53DA54EA55FA5A7
:10BAD00068A579A58AA59BA50F94CB58882309F45E
:10BAE000ADC0A3019201C501B4010F94BC5F20E079
:10BAF00030E040E05FE30F9431596CA37DA38EA347
:10BB00009FA328A539A54AA55BA56CA57DA58EA5F3
:10BB10009FA50F94BC5F20E030E040E05FE30F940E
:10BB200031592B013C0120E030E0A901C701B601E9
:10BB30000F94CB58881F8827881F181709F4D2C084
:10BB400080E090E0A0E8BFEB88A799A7AAA7BBA7D1
:10BB50002CA13DA14EA15FA1CA01B9010F94315999
:10BB60004B015C01A3019201C301B2010F94315951
:10BB70009B01AC01C501B4010F94BD5F0F946B62D2
:10BB80004B015C01AC019B01C701B6010F94BC5F86
:10BB90006CA77DA78EA79FA7A5019401C701B60139
:10BBA0000F94BD5F9B01AC016CA57DA58EA59FA5E3
:10BBB0000F9431596B017C0120E030E0A9010F9412
:10BBC0001D6287FD94C0C701B6010F946B626B01C3
:10BBD0007C01C301B2019058A50194010F94B76094
:10BBE00028A539A54AA55BA50F943159A70196014F
:10BBF0000F9431592CA13DA14EA15FA10F94BD5FBF
:10BC000069837A838B839C83A50194016CA17DA1B8
:10BC10008EA19FA10F94B76028A539A54AA55BA561
:10BC20000F943159A70196010F943159A301920144
:10BC30000F94BD5F6D837E838F83988720E030E013
:10BC4000A90169817A818B819C810F94CB588111E4
:10BC500066C020E030E0A9016D817E818F819885EA
:10BC60000F94CB5881115BC00E946E4784E99FE01E
:10BC70000E9482362DC08430910509F463C0459737
:10BC800039F10F94553224C08A32910509F4ECC180
:10BC900058F48C31910509F4AAC008F490C04D976E
:10BCA00081F70E94047514C08B35910509F459C2BF
:10BCB0008C35910509F459C28A35910511F7109216
:10BCC0007E0806C0213021F40E94C7310E9445FC45
:10BCD00039A9311102C00F94E23B88A9809368080A
:10BCE0000C94276980E090E0A0E8BFE32DCFC12C41
:10BCF000D12C76016ECF89E40E949531882331F0F2
:10BD00000E941D3169837A838B839C838AE40E941D
:10BD10009531882309F492CF0E941D318BCF412F9A
:10BD2000BE016F5F7F4F8CE498E00F947B3C0F94D3
:10BD3000813B60935C0870935D0880935E089093EC
:10BD40005F08C6CF80E50E949531C12CD12C7601C9
:10BD5000882321F00E9420266B017C0183E50E944C
:10BD60009531882361F00E941D3120E030E04AE7E0
:10BD700054E40F9431590F9430616B017C010E949F
:10BD8000FEE180917C13811105C060E08AEA9FE0AA
:10BD90000E9434B70F94813BC60ED71EE81EF91ED1
:10BDA0000F94813B6C197D098E099F0997FF90CFF5
:10BDB00080E00E943E4EF4CF0E941E3E89CF0F9439
:10BDC000E248811185CF8CE0EBE9F2E0DE011196CB
:10BDD00001900D928A95E1F770E060E080E50E94A5
:10BDE000A231BE016F5F7F4F0F94300771CF87E0A4
:10BDF0000E9409F6811106C060E08FE40E940A33B8
:10BE0000811166CF0E94FEE1109239026091B41058
:10BE10008CE40E940A33982E80E00E9410340F9424
:10BE2000813B60935C0870935D0880935E089093FB
:10BE30005F088091800290918102A0918202B0916E
:10BE400083028093D4049093D504A093D604B09336
:10BE5000D70480917A0290917B029093D3048093CF
:10BE6000D20484E690E090937B0280937A0281E092
:10BE70008093D7070F94C3018AE50E944731A82E0B
:10BE800088E50E944731182F89E50E944731B82E76
:10BE9000181308C0B12EA11205C011E0BB24B39441
:10BEA000AA24A39482E50E949531882309F4D2C084
:10BEB0000E941D316C8F7D8F8E8F9F8F20E030E030
:10BEC000A9010F94CB58882349F0111103C0BB205E
:10BED00009F494C0CE014C960F944234112309F416
:10BEE00088C0BB2009F482C01092B5101092B61021
:10BEF0001092B7101092B8101092B9101092BA1098
:10BF00001092BB101092BC100E94F9F7ECEDF8E211
:10BF1000C590D590E590F490E0EEF8E2459055900C
:10BF200065907490A7019601C301B2010F94CB589C
:10BF300087FF95C0A7019601C301B2010F94B760B6
:10BF40009B01AC010F94315920E030E040E85FE301
:10BF50000F94BD5F0F946B6220E030E048E452E440
:10BF60000F94315969837A838B839C838091BD10B0
:10BF70009091BE10A091BF10B091C0108CA39DA352
:10BF8000AEA3BFA320E030E040EC5FE3C301B20109
:10BF90000F9431592B013C0177FA709477F8709423
:10BFA00020E030E040EC5FE3C701B6010F94315967
:10BFB0009058DE0111966D01ECA0FDA00EA11FA10D
:10BFC000A30192010E94F2F60F944C031092B51057
:10BFD0001092B6101092B7101092B8101092B910BB
:10BFE0001092BA101092BB101092BC1080E00E9408
:10BFF0005FFFBB2019F081E00E945FFFAA2019F0CB
:10C0000082E00E945FFF0E94F9F78091D60780933B
:10C01000D707892D0E9410348091D4049091D504C3
:10C02000A091D604B091D7048093800290938102AE
:10C03000A0938202B09383028091D2049091D304A2
:10C0400090937B0280937A0283E0809384020F9422
:10C05000B0003ECE60E070E080E890E42BCFA3011A
:10C060009201C701B6016ACF80911F08813009F0A3
:10C070002FCE89E40E949531082F10E0882319F013
:10C080000E941931182F8AE40E949531F82E8823D6
:10C0900039F00E941931011106C0853068F005C0E1
:10C0A00080E0002349F0153028F083EB9FE00E94E8
:10C0B00082360ECEF110F1CF90E1E5EBF0E1ACE489
:10C0C000B8E001900D929A95E1F7002391F0B4E069
:10C0D0001B02F0011124E654F94E40815181628126
:10C0E000738140934C0850934D0860934E087093B1
:10C0F0004F08FF2091F024E08202F0011124EA555C
:10C10000F94E80819181A281B381809350089093F0
:10C110005108A0935208B093530840E050E0BA0190
:10C1200086E40E94B0316B017C0120E030E0A9017F
:10C130000F941D6218168CF420E030E040E752E4C2
:10C14000C701B6010F94B76069837A838B839C83A0
:10C15000CE0101960E94F8FEBBCD60E070E0CB01FD
:10C16000F3CF8FE080937E08B3CD809105058823BF
:10C1700081F1893009F0ACCD67EAA62E62E0B62ED7
:10C1800075EBC72E70E1D72EE12C00E010E0D50151
:10C190008D915D010E949531F82E882361F0133056
:10C1A00011F4082FFE2C0E941D31F601608371836B
:10C1B00082839383EF2C1F5FF4E0CF0ED11C1430E9
:10C1C00031F7EE2009F457C00E94F9F70F94B00040
:10C1D0007FCD57EAC52E52E0D52EF12CE12C00E0A0
:10C1E00010E0D6018D916D010E949531382E882383
:10C1F000D9F10E941D314B015C01133059F0F70158
:10C20000E959F64F20813181428153810F94BC5FFF
:10C210004B015C01F701EB54FF4E208131814281DB
:10C220005381C501B4010F94BC5F2B013C012DEB80
:10C2300037E346E855EB0F941D6287FD0AC02DEBEE
:10C2400037E346E855E3C301B2010F94CB58181603
:10C250005CF41330C1F48092C1109092C210A0928D
:10C26000C310B092C410032D1F5FB4E0EB0EF11C9D
:10C27000143009F0B6CF002309F4A8CF81EC90E187
:10C280000E94F1F3A3CFF701E356F74F5F01A3013B
:10C29000920160817181828193810F94BD5FD5018C
:10C2A0006D937D938D939C931397812F0E94E9F555
:10C2B000DBCF80910605909107058937910511F430
:10C2C0000C94B36B08F0F4C18E34910509F4BDC62B
:10C2D00008F0FEC08A31910509F4FEC508F094C04B
:10C2E0008431910509F444C508F071C0813191058C
:10C2F00009F403C508F044C0029708F0C2CC80E5F9
:10C300000E949531C12CD12C7601882321F00E9406
:10C3100020266B017C0183E50E949531882361F022
:10C320000E941D3120E030E04AE754E40F94315977
:10C330000F9430616B017C010E94FEE18091090540
:10C3400090910A05009709F4D2C40F948E48809109
:10C3500006059091070564ED7FE0892B11F46CECE4
:10C360007FE030E020E048EB51E482E00E94263894
:10C3700040E0C701B6010E940A5A0F94C048A8CCF9
:10C38000429709F07ECC83E50E949531882311F411
:10C390000C945D6A0F94813B60935C0870935D0818
:10C3A00080935E0890935F080E941D3120E030E08A
:10C3B0004AE754E40F9431590F94306160931002AE
:10C3C00070931102809312029093130281CC8731F3
:10C3D000910509F402C570F48531910509F4F9C499
:10C3E000469709F04ECC8091D91682FD71CC0E94FF
:10C3F00092D76ECC8831910509F404C5499709F0AC
:10C4000040CC0E94F05B64CC8032910509F4E8C511
:10C41000C0F58D31910509F4CCC570F48B319105CF
:10C4200009F46DC54C9709F02CCC809109059091C9
:10C430000A050F9437494CCC8E31910509F4C0C5DB
:10C440004F9709F01ECC0F945A036C8F7D8F8E8FFF
:10C450009F8FBE016F5F7F4FCE014C960E94072BCE
:10C46000CE0101960F948E480E945748BE016F5F1F
:10C470007F4F87E490E10E946F4D8AE00E94493629
:10C4800027CC8B34910509F4D8C5B0F481329105DD
:10C4900009F4CFC58934910509F0F3CB80E50E94FA
:10C4A0004731882309F414CC0E94F530853608F012
:10C4B00084E6809313050CCC8C34910509F4C1C536
:10C4C0008D34910509F0DDCB81E00F948C0300CC15
:10C4D0008C36910509F4FCCB08F07FC085359105B9
:10C4E00011F40C94A06A68F58235910509F4D5C75A
:10C4F000F8F48035910509F4B6C78135910509F046
:10C50000C0CB0E9493DA0E940FE281E00F948C036B
:10C510000E94043668EE73E080E090E00E9450359F
:10C520000E94822260E08EE191E10E9434B7D0CB7C
:10C530008335910509F4B9C78435910509F423CFF2
:10C54000A0CB8936910509F470C698F58C35910514
:10C5500011F40C94C56A8836910509F092CB80914C
:10C560006B1083FDB5CB0E945B4887FDB1CB89E49E
:10C570000E949531882311F40C9403720E94F530C7
:10C5800090E01816190614F481E090E026E0289F48
:10C59000F001299FF00D1124E05EF74F8081918119
:10C5A0000E9477E161E080E00F94CF4C0F94984CAB
:10C5B0008FCB8A36910509F463C68B36910509F055
:10C5C00060CB80E50F947633823008F081CBE82F82
:10C5D000F0E0EB55F64F10827BCB8237910511F4DA
:10C5E0000C94666BA0F58F36910509F483C6C8F4E8
:10C5F0008D36910509F4BBC58E36910509F041CB06
:10C600008EE40E949531882309F462CB0E94412672
:10C6100060934711709348118093491190934A1188
:10C6200057CB8037910509F453CB8137910509F039
:10C6300028CB83E50E949531882309F4A1C60E9486
:10C64000F5308D3308F097C680930F0241CB8637C3
:10C65000910511F40C94766BD0F48337910511F4A5
:10C660000C946E6B8537910509F00BCB8091090511
:10C6700090910A05009711F40C94726BDC012C91D7
:10C68000222311F40C94726B0F948E4821CB8737C0
:10C69000910511F40C94AF6B8837910509F0F1CA3C
:10C6A00081E08093D7078093D6070F94C30110CB06
:10C6B0008039E1E09E0711F40C94276F08F075C1F2
:10C6C0008E3C910511F40C94016D08F07FC08E3BF7
:10C6D000910509F489C6C0F58C38910509F45DC649
:10C6E00028F48D37910509F48CCECBCA8139910598
:10C6F00011F40C94BB6B8B39910509F0C2CA83E528
:10C700000E949531882309F4E3CA0E94F530182F5E
:10C710008C3308F08CE38093E1040F94813B6B0130
:10C720007C01212F30E0A8EEB3E00F94635FC60ECA
:10C73000D71EE81EF91EC092DD04D092DE04E092FE
:10C74000DF04F092E004C4CA8B3C910511F40C9410
:10C75000656C80F5883C910511F40C94346C893C2F
:10C76000910509F08ECA0E945B4887FDB1CA07EAAD
:10C7700012E08CE6E82E80E1F82E9BEAC92E92E0CA
:10C78000D92ED8018D918D010E944731882359F00F
:10C790000E941D310F943061F701608371838283A1
:10C7A00093830E948CE1F4E0EF0EF11CC016D106D9
:10C7B00041F78ECA8C3C910511F40C94886C8D3C29
:10C7C000910509F05ECA0E94443782CA8C3221E08A
:10C7D000920711F40C94E06D08F08CC08D3D91052A
:10C7E00011F40C94556D08F04AC0833D910511F485
:10C7F0000C94516D8C3D910509F043CA82E40E946E
:10C800004731882341F080917A0290917B02909386
:10C8100015028093140282E50E944731882341F07B
:10C82000809114029091150290937B0280937A027A
:10C8300083E50E949531882331F00E94193190934D
:10C840007B0280937A028091010590910205A0916C
:10C850000305B0910405892B8A2B8B2B09F038CA6C
:10C8600060917A0270917B028CE691E10E94143E05
:10C8700085E20E9449368AE00E94493629CA8A3FE9
:10C88000910511F40C94EB6E8232914009F0F9C9D4
:10C890008AE50E949531882311F40C94AC6D0E94B6
:10C8A0001D3120E030E040E050EC0F94CB5887FF82
:10C8B00002C00C94CD6D0E941D3120E030E040E0BC
:10C8C00050E40F941D62181614F40C94D36D0E945A
:10C8D0001D31209188103091891040918A1050911B
:10C8E0008B100F9431590F942961CB010F94353C73
:10C8F0000C94B26D8F32B1E09B0711F40C94236F4E
:10C9000078F58D32F1E09F0711F40C94F66D8E32BC
:10C91000914009F0B6C983E50E944731182F88235A
:10C9200069F00E9419319C0190938A0280938902D8
:10C9300091E0232B09F090E09093B70980E50E94E5
:10C940004731882311F40C94016F209189023091B2
:10C950008A02232B11F00E9409318093B709B8C9CC
:10C96000803331E0930711F40C94776E8336914055
:10C9700009F087C980E50E949531082F882321F0AE
:10C980000E94F5308093540283E50E949531182F60
:10C99000882311F40C94A8710E9409318093250218
:10C9A000812F0E94C2330C94AB71883FB1E09B078A
:10C9B00011F40C948A7008F072C08C3AF1E09F0771
:10C9C00011F40C945F6F08F043C08D3931E0930788
:10C9D00011F40C94D17178F58A39B1E09B0709F410
:10C9E00077C98C39914009F04CC98091010588784C
:10C9F00011F00C942B6F80910305867011F00C944C
:10CA00002B6F0E9457488DE092E10E948236809100
:10CA100059020E94DC3840915502509156026091B3
:10CA20005702709158028DEE91E10E94FA388AE027
:10CA30000E9449364DC9843AF1E09F0711F40C94E5
:10CA40005B6F853A914009F01CC90E94724740C94A
:10CA5000853F31E0930711F40C94827068F4863EB0
:10CA6000B1E09B0711F40C941070843F914009F0E1
:10CA700008C90E94C8DD2CC9863FF1E09F0711F468
:10CA80000C948670873F914009F0FBC861E083E514
:10CA90000E940A3391E089270F948C1119C98C36B2
:10CAA00033E0930709F414C908F0D2C08B35B2E023
:10CAB0009B0711F40C94AD7068F48C30F2E09F0782
:10CAC00011F40C949C708835924009F0DAC80E94E9
:10CAD000E05AFEC88D3B32E0930711F40C942D719F
:10CAE0008E3B924009F0CDC80E945B48182F87FD0D
:10CAF000EFC88AE50E949531812C912C90E2A92EF5
:10CB000091E4B92E882341F040E050E0BA018AE573
:10CB10000E94B0314B015C01412F64E083E00E9430
:10CB2000978820E030E0A901C501B4010F941D628F
:10CB300018167CF580E090E0A0EAB0E489839A833F
:10CB4000AB83BC832091BD103091BE104091BF10CB
:10CB50005091C010C501B4010F94BD5F6B017C0101
:10CB600020E030E042E553E40F94CB5887FD06C047
:10CB7000C12CD12C82E5E82E83E4F82ECC8EDD8EFC
:10CB8000EE8EFF8EBE016F5F7F4FCE014C960E94EE
:10CB9000AAF785E50E944731882311F40C9431717E
:10CBA0000E941D316B017C0120E030E0A901C7012A
:10CBB000B6010F941D6287FF04C0F7FAF094F7F8EE
:10CBC000F094F7FAF094F7F8F094C982DA82EB82E5
:10CBD000FC8244E061E0CE0101960E94B75820E05B
:10CBE00030E0A901C501B4010F941D6218165CF56F
:10CBF00080E090E0A0EAB0E489839A83AB83BC83B1
:10CC0000A50194016091BD107091BE108091BF107C
:10CC10009091C0100F94BC5F6B017C0120E030E06C
:10CC2000A9010F941D6218161CF0C12CD12C76019D
:10CC3000CC8EDD8EEE8EFF8EBE016F5F7F4FCE01FC
:10CC40004C960E94AAF710921B050E94AE8740C81E
:10CC5000873EB3E09B0711F40C94C171C0F4843893
:10CC6000F3E09F0711F40C943D71803A934011F06A
:10CC70000C94415E2091090530910A059091D916D6
:10CC800092609093D916C9010F94374921C8883E04
:10CC900033E0930711F40C94EA71893E934011F04C
:10CCA0000C94415E0F94074881110C94685E0E94B9
:10CCB0001F330F94C5470F945A036D3371058105D7
:10CCC000910520F086ED92E10E94767282ED92E16C
:10CCD0000E94767284EE809313058EEB92E10E949F
:10CCE00082368AEB92E10E9476720C94685E60E074
:10CCF0008CED9FE00E9434B72ACB8091010584FD22
:10CD000019C08091030587FD15C0809104058370CB
:10CD100089F460E08FEE9FE00E9434B70E94743582
:10CD20005F988A988091080181708093060112981B
:10CD30000C94685E88E50E94473181115F9889E50F
:10CD40000E94473181118A988AE50E9447318823E1
:10CD500029F08091080181708093060185E40E948A
:10CD60004731882311F40C94685E12980C94685E25
:10CD70008091D91683FF25C087E090E10E9482361A
:10CD80008091D91683FF17C08AEF96E10E9476D86A
:10CD90008BE1EAEFF6E1DE01119601900D928A95A2
:10CDA000E1F770E060E0CE0101960F947B0CCE01BC
:10CDB00001960E94473388EF9FE00E9482360C94D0
:10CDC000685E0E94574888E190E10E9482360C9488
:10CDD000685E0E94A3D70C94685E809109059091CB
:10CDE0000A05FC012191222331F02032D9F7DF011D
:10CDF00011971C92F7CF60E00F94804910921305B1
:10CE00000C94685E83E50E949531882321F00E948E
:10CE100041260E94742484E50E9495318823A9F05C
:10CE20000E9441266B017C010F940104C092D00541
:10CE3000D092D105E092D205F092D305CD28CE282C
:10CE4000CF2819F081E080937D08809164068823C3
:10CE5000F9F080E090E0A0EAB1E489839A83AB83A3
:10CE6000BC831C8E1D8E1E8E1F8E18A219A21AA2A4
:10CE70001BA210E000E020E0AE014F5F5F4FBE015B
:10CE8000645E7F4FCE0180960E9449570C94685E85
:10CE90000E94CD35882381F00E94EBCF0E94F135AE
:10CEA00083EF98E00F9416471092AE111092AF11D5
:10CEB0001092B0111092B11161E082EC9EE10E94DB
:10CEC000CD374AE85EE162E270E185E00F946D33B0
:10CED0000F94C0480C94685E8091D91683FD02C0FF
:10CEE0000C94685E83E50E949531882311F40C94BC
:10CEF000685E0E9441260E9474240C94685E83E45C
:10CF00000E944731882361F188E390E10E948236D4
:10CF1000809141188823F9F0BE016F5F7F4F8EE347
:10CF200098E10E9409D8CE0101960E9410D4CE014A
:10CF300001960F94604880913913882339F080E27C
:10CF40000E94493689E393E10E9410D48AE00E944E
:10CF500049360C94685E8EE290E10E948236F6CFEC
:10CF600083E50E949531882301F10E94F530182F46
:10CF70008C3308F08CE38093DC040F94813B6B01CD
:10CF80007C01212F30E0A8EEB3E00F94635FC60E62
:10CF9000D71EE81EF91EC092D804D092D904E092A0
:10CFA000DA04F092DB040C94685E0F94DD460C9476
:10CFB000685E8091D9168E7F8093D9160C94685E36
:10CFC0008091D91683FD02C00C94685E0F943B32A9
:10CFD0008091090590910A050F945D470C94685E55
:10CFE0008091D91682FD0E94FEE18091D91683FDC1
:10CFF00002C00C94685E60E080E50E940A33182F3E
:10D00000682F8091090590910A050F94804983E566
:10D010000E949531882321F00E9441260E947424A9
:10D020000E94EBCF11110C94685E0E94F1350C94B4
:10D03000685E0E94794D0C94685E0E94F1350C94F4
:10D04000685E0F9454040C94685E70E060E083E5C1
:10D050000E94FB328E34910531F40E941BE10F9443
:10D06000C0480C94685E82EB90E10E948236609129
:10D07000C6077091C70789EA90E10E94E83860917D
:10D08000C8077091C9078CE990E10E94E838609167
:10D09000C6077091C7078091C8079091C907681BA0
:10D0A000790B80917D08815021E030E0823010F0D2
:10D0B00030E020E0621B730B81E990E10E94E838C8
:10D0C0008AE00E94493689E890E10E948236809188
:10D0D000CA079091CB07A091CC07B091CD078C8F58
:10D0E0009D8FAE8FBF8FBE016F5F7F4FCE014C967D
:10D0F0000E94072BBE016F5F7F4F8CE790E10E947B
:10D100006F4D8091CE079091CF07A091D007B0913D
:10D11000D1078C8F9D8FAE8FBF8FBE016F5F7F4F0A
:10D12000CE014C960E94072BBE016F5F7F4F8CE6AD
:10D1300090E10E946F4D20E030E04AE754E46091B6
:10D14000D2077091D3078091D4079091D5070F949F
:10D15000B760AB01BC0184E590E10E94FA388DE62E
:10D160000E9449368AE00E9449360C94685E80919C
:10D170006B1083FF02C00C94685E0E945B48F82E1F
:10D1800087FF02C00C94685E89E40E949531882371
:10D1900011F40C940E720E94F53090E018161906E6
:10D1A00014F481E090E026E0289FF001299FF00D23
:10D1B0001124E05EF74F8081918110E00E9477E1B9
:10D1C00061E081E00F94CF4C2091ED153091EE1588
:10D1D0008091EB159091EC1582179307F4F485EC90
:10D1E00090E19F938F9380ED90E19F938F931F9297
:10D1F0000E9419B70F900F900F900F900F9001E0C1
:10D200000F94984C002311F40C94685E40E0612F59
:10D210008F2D0F94FE0F0C94685E8AEB90E1112322
:10D2200001F3012FEDCF182FEBCF0E945B48182F91
:10D2300087FD0AC085ED90E10E948236812F0F9410
:10D24000060E8AE00E944936B8A9B0936808E196B4
:10D250000FB6F894DEBF0FBECDBFDF91CF911F9107
:10D260000F91FF90EF90DF90CF90BF90AF909F9085
:10D270008F907F906F905F904F903F902F90089588
:10D2800080E50F947633F82EE1E0E81710F40C9463
:10D29000685E81E40E9447316091A509062F10E085
:10D2A000811102C00FEF10E089E40E9495318823BC
:10D2B00011F40C9420720E94F53090E018161906B3
:10D2C00014F481E090E026E0289FF001299FF00D02
:10D2D0001124E05EF74F04811581EF2DF0E0EB554E
:10D2E000F64F0F3F110519F010F00FEF10E000831B
:10D2F0000C94685E83E50E944731882329F083E51A
:10D300000F94763380936B100E94574886EE90E11D
:10D310000E94823680916B10882351F110E000E06A
:10D3200020E080916B1090E0B0E0A0E0002E04C0FF
:10D33000B695A795979587950A94D2F780FF12C066
:10D34000FF24F394F20E222319F08CE20E94493656
:10D35000F801EE0FFF1FE452FF4E859194910E9459
:10D3600082362F2D0F5F1F4F05301105D1F6EECD00
:10D3700088ED90E1F2CD8CE380930F020C94685E0F
:10D380000E94574860910F028DEE90E10E94F238A2
:10D390008AE00E9449360C94685E80916B1083FF8E
:10D3A00002C00C94685E89E40E949531882311F4D0
:10D3B0000C942C720E94F53090E01816190614F4A3
:10D3C00081E090E026E0289FF001299FF00D1124D4
:10D3D000E05EF74F828193810E948E3561E080E0AC
:10D3E0000F94CF4C0C94685E80916B1083FF02C049
:10D3F0000C94685E89E40E949531882311F40C94A2
:10D4000037720E94F53090E01816190614F481E086
:10D4100090E026E0289FF001299FF00D1124E05EA6
:10D42000F74F8281938110E00E948E3560E081E0A9
:10D430000F94CF4C2091890830918A0880918708F9
:10D4400090918808821793071CF483E091E102C051
:10D4500084EF90E160E00E9434B760E0812F0F9488
:10D46000790E0C94685E83E50E944731882369F049
:10D470008091DB07882331F088E191E10E948236B8
:10D480000C94685E82E191E1F9CF0E947435269A8E
:10D490002E980F94C0480C94685E80917E088F7D12
:10D4A000806180937E080C94685E80917E088F7EF8
:10D4B000806280937E080C94685E8091010584FDF3
:10D4C0000CC08091030587FD08C08091040583701E
:10D4D00021F40E940FE20C94685E0E94FEE188E550
:10D4E0000E944731882331F05F9A8091D9078E7F5F
:10D4F0008093D90789E50E944731882331F08A9AC1
:10D500008091D9078D7F8093D9078AE50E944731A2
:10D51000882359F0809108018095817080930601DD
:10D520008091D9078B7F8093D90785E40E9447318A
:10D53000882311F40C94685E0E9480220C94685E2B
:10D5400083E50E944731882311F40C94685E0F94A0
:10D55000813B60935C0870935D0880935E089093B4
:10D560005F080E941D3120E030E04AE754E40F9448
:10D5700031590F9430616093E2047093E304809317
:10D58000E4049093E5040C94685E0E945B4887FF76
:10D5900002C00C94685E8091010584FD09C08091F1
:10D5A000030587FD05C080910405837009F489C0D7
:10D5B00027EAC22E22E0D22E3CE6E32E30E1F32E03
:10D5C00010E0D6018D916D010E949531882309F4F8
:10D5D00065C0133009F06DC00E941D314B015C0124
:10D5E00020E030E040EA51E40F94CB5887FF4EC072
:10D5F000A501940160918C1070918D1080918E1016
:10D6000090918F100F94B7602B013C01AC019B01EE
:10D610006091990970919A0980919B0990919C0958
:10D620000F9431596093990970939A0980939B09DB
:10D6300090939C09A301920160919C1070919D10A0
:10D6400080919E1090919F100F94315960939C107F
:10D6500070939D1080939E1090939F106091850908
:10D660007091860980918709909188090F94D0580C
:10D67000A30192010F9431590F9430616093850991
:10D6800070938609809387099093880980928C1003
:10D6900090928D10A0928E10B0928F101F5FF4E0C8
:10D6A000EF0EF11C143009F08CCF0E94DAE10C94DB
:10D6B000685E0E941D31F701648B758B868B978B9A
:10D6C000EDCF81E00F9400320C94685E0F949B3193
:10D6D00081E496E10E941EDD0C94685E0E94A936EA
:10D6E0000C94685E0F94C0480C94685E0091090524
:10D6F00010910A0594E0F12C40E09150F9F0F80106
:10D700008081282F2B7F213499F421812133B1F49A
:10D71000813411F1853409F441E098012E5F3F4FC7
:10D7200089012F5F3F4FF80180818032C9F3E5CF37
:10D73000803521F4818180538A3078F341110E9431
:10D740005748FF2021F08DE291E10E948236C80106
:10D750000E9450360C94685EFF24F394DECF0F9441
:10D7600099010C94685E1092D7071092D6070F9417
:10D77000C3010C94685E70E060E083E50E94FB32B8
:10D78000823040F00E946E4780E391E10E94823631
:10D790000C94685E8C01112788E40E9495318823DF
:10D7A000C1F00E9419318A3A91050CF44BC00E94D5
:10D7B00019318D3291400CF048C00E94193126E099
:10D7C000209FF001219FF00D1124E05EF74F91831F
:10D7D000808382E40E9495318823A9F00E94193148
:10D7E0000597B4F10E9419318D389105A4F50E9476
:10D7F000193126E0209FF001219FF00D1124E05EF9
:10D80000F74F9383828386E40E949531882311F435
:10D810000C94685E0E94193197FD20C00E94193156
:10D820008F3F910509F0ECF40E94193126E0209F0A
:10D83000F001219FF00D1124E05EF74F9583848362
:10D840000C94685E8AEA90E0BACF8CE291E0B7CFA0
:10D8500085E090E0CECF8CE890E0CBCF90E080E008
:10D86000E5CF8FEF90E0E2CF0E945B48182F87FF53
:10D8700002C00C94685E00919C0884E40E9495317B
:10D88000F82E8823B1F00E941D314B015C0120E08D
:10D8900030E0A9010F94CB588823A9F024E01202AC
:10D8A000F0011124E856F74F80829182A282B38260
:10D8B0000F2D602F83E50E940A3380939C080E94FD
:10D8C00033C90C94685E80E0F8CF0E945B4887FF04
:10D8D00002C00C94685EB7EAEB2EB2E0FB2E10E0BB
:10D8E00000E0D7018D917D010E944731882349F0E6
:10D8F0000E941D31F801E459FF4E64A375A386A36D
:10D9000097A30C5F1F4F0031110559F70C94685E07
:10D910008091020587FD2DC0809103058E7049F529
:10D920004091A0105091A1106091A2107091A3108D
:10D9300085E591E10E94FA384091A4105091A5101C
:10D940006091A6107091A71082E591E10E94FA38CB
:10D950004091A8105091A9106091AA107091AB103D
:10D960008DEB9DE20E94FA388AE00E9449360C94C1
:10D97000685E83E50E949531882391F00E941D31F5
:10D980006093A0107093A1108093A2109093A310A5
:10D990006093A8107093A9108093AA109093AB1075
:10D9A00080E50E949531882351F00E941D316093DB
:10D9B000A0107093A1108093A2109093A31082E501
:10D9C0000E949531882351F00E941D316093A4106C
:10D9D0007093A5108093A6109093A71084E50E94E1
:10D9E0009531882311F40C94685E0E941D31609378
:10D9F000A8107093A9108093AA109093AB100C9468
:10DA0000685EA9EAEA2EA8E0FA2E10E088E5810F08
:10DA10000E944731882351F00E941D31F701608335
:10DA2000718382839383812F0E94E9F51F5FF4E065
:10DA3000EF0EF11C133051F78091030587FF02C0F0
:10DA40000C94E66080910405837011F00C94E660FC
:10DA50004091A9085091AA086091AB087091AC0858
:10DA600085E691E10E94FA384091AD085091AE08E8
:10DA70006091AF087091B0088FE392E40E94FA3889
:10DA80004091B1085091B2086091B3087091B40808
:10DA90008CE392E40E94FA388AE00E9449360C94A2
:10DAA000685E0E9480480C94685E0E945B48082F64
:10DAB00087FF02C00C94685E83E50E949531002EBA
:10DAC000000C110B7801EE0CFF1C882359F10E9409
:10DAD0001931F701EA5CFD4F91838083000F111F1C
:10DAE000000F111F98012B573D4F7901BC01990F71
:10DAF000880B990B0F94D2582AE037ED43E25CE390
:10DB00000F94315904531A4FD8012D913D914D91E5
:10DB10005C910F943159F701608371838283938301
:10DB20000C94685E0E94574885E40E94493680E361
:10DB3000800F0E944936F701EA5CFD4F60817181D8
:10DB400080E791E10E94143E85E20E9449368AE016
:10DB50000E9449360C94685E83E50E9495318111DC
:10DB60000C944F648091030587FD23C080910405C8
:10DB70008370F9F40E94574840914506509146063B
:10DB8000609147067091480688E791E10E94FA3853
:10DB90008AE00E9449360C94685E60E070E080E0A4
:10DBA00090EC0C94696460E070E080E090E40C9488
:10DBB000696482E50E9447318111DCCF0C94685E74
:10DBC00064E071E083E50E94A2318C0168EE73E0AD
:10DBD00080E50E94A2318938F3E19F0710F088E8C0
:10DBE00093E1B8010E9494800C94685E85E40F94E0
:10DBF0007633811174C080E50E944731882351F04B
:10DC00000E941D316093F0157093F1158093F21509
:10DC10009093F31589E40E944731882381F00E9494
:10DC20001D312CEA35EC47E25EE30F9431596093E5
:10DC3000F4157093F5158093F6159093F71584E419
:10DC40000E944731882381F00E941D312CEA35EC77
:10DC500047E25EE30F94B7606093F8157093F9158F
:10DC60008093FA159093FB150E9457484091F01548
:10DC70005091F1156091F2157091F3158DE891E1D5
:10DC80000E94FA382CEA35EC47E25EE36091F41525
:10DC90007091F5158091F6159091F7150F94B76076
:10DCA000AB01BC0189E891E10E94FA382CEA35EC1D
:10DCB00047E25EE36091F8157091F9158091FA15CD
:10DCC0009091FB150F943159AB01BC0185E891E1AE
:10DCD0000E94FA388AE00E9449360C94685E0E94DD
:10DCE0006E4781E991E10E9482360C94685E80E57E
:10DCF0000E944731882351F00E941D3160938C08A7
:10DD000070938D0880938E0890938F0889E40E9409
:10DD10004731882381F00E941D312CEA35EC47E21F
:10DD20005EE30F943159609390087093910880934B
:10DD300092089093930884E40E944731882381F0ED
:10DD40000E941D312CEA35EC47E25EE30F94B76088
:10DD50006093940870939508809396089093970821
:10DD60000E94574840918C0850918D0860918E0810
:10DD700070918F088BEA91E10E94FA382CEA35EC19
:10DD800047E25EE36091900870919108809192085B
:10DD9000909193080F94B760AB01BC0187EA91E1C1
:10DDA0000E94FA382CEA35EC47E25EE36091940871
:10DDB0007091950880919608909197080F94315929
:10DDC000AB01BC0183EA91E10E94FA388AE00E942B
:10DDD00049360C94685E83E40E944731882321F021
:10DDE0000E9419310E944A27609152027091530299
:10DDF0008FEA91E10E94143E8AE00E9449360C9419
:10DE0000685E11110C94685E0E9457488AED91E19A
:10DE10000E9482368091B709882391F082EC91E1CB
:10DE20000E9482366091890270918A0289EC91E1A8
:10DE30000E94143E85EC91E10E9482360C94685E4B
:10DE40008EEB91E1EDCF0E941C390C94685E0E942C
:10DE5000FEE10C94685E88E40E944731882321F03B
:10DE60000E9409318093E60482E50E944731082F21
:10DE700083E50E944731182F011102C0882341F029
:10DE80000E946D22112321F00E94093180935902D2
:10DE900084E40E944731882311F40C94685E0E9448
:10DEA0001D316093550270935602809357029093F0
:10DEB00058020C94685E0E946F490C94685E0F943F
:10DEC000E24881110C94685E7BEAC72E78E2D72E77
:10DED00025EB30E13DA32CA3CE0101961C017C0172
:10DEE00010E000E0F6016591759185919491ACA1E7
:10DEF000BDA18D909D90AD90BD90BDA3ACA3A5019B
:10DF000094010F94BC5F2B013C01F70140825182C8
:10DF10006282738220E030E040EA51EC0F941D628F
:10DF200087FD0AC020E030E040EA51E4C301B201BD
:10DF30000F94CB58181684F4F801EE58FE4BE49178
:10DF40001E1654F4B7FAB094B7F8B094D7018D9276
:10DF50009D92AD92BC921397F70181909190A19000
:10DF6000B1907F0120E030E040EA51ECC501B401FE
:10DF70000F941D6287FD3FC020E030E040EA51E48D
:10DF8000C501B4010F94CB581816ACF10F5F1F4FA9
:10DF9000F4E0CF0ED11C0330110509F0A3CF69EADC
:10DFA000E62E68E0F62E10E0F10181919191A191A9
:10DFB000B1911F01F70181939193A193B1937F01D7
:10DFC000812F0E94E9F51F5F133071F70F94B000A5
:10DFD00060E08EE192E10E9434B763E972E084E68A
:10DFE00090E00E9494806AEB72E084E690E00E94E8
:10DFF00094800C94685E0E946E478CE392E10E94CC
:10E00000823661E08EE292E10E9434B70E94AE87D0
:10E0100068E270E088EC90E00E9494800C94685E66
:10E0200084E50E9447318823A1F0109215051092D3
:10E0300016051092170510921805109219058FEF0A
:10E040000E94822461E070E084E50E94FB328093AC
:10E05000190583E50E944731882321F00E94193178
:10E060000E94822483E40E944731882331F080910A
:10E070002302803210F40E94D43380E50E9447319D
:10E08000882331F00E941931803210F40E94D43379
:10E0900085E50E944731882311F40C94685E0E9444
:10E0A0001931803210F00C94685E41E050E060E07D
:10E0B00070E0082E04C0440F551F661F771F0A9496
:10E0C000D2F7409550956095709500911505109187
:10E0D000160520911705309118054023512362231E
:10E0E000732340931505509316056093170570939D
:10E0F00018059091230289130C94685E10926A109F
:10E100000C94685E0F94F1180C94685E0F94CE0125
:10E110000C94685E209349060F94E5181092490606
:10E12000882311F40C94685E0E9457488AE592E1B6
:10E130000E9482360C94685E8091D91682FF05C0D9
:10E1400080648093D9160C94685E83FD02C00C94A1
:10E15000685E0F943B320C94685E0E945B48082F07
:10E1600087FF02C00C94685E85E50E9447318823D2
:10E1700059F10E941D314B015C01E02E002E000C74
:10E18000FF0820E030E0A9010F941D6287FF04C062
:10E19000B7FAB094B7F8B09420E030E84BE354E419
:10E1A000C501B4010F941D62970153E0220F331F84
:10E1B0005A95E1F728523A4F1816D4F1D9018D92A9
:10E1C0009D92AD92BC9213978CE40E9447318823B4
:10E1D00011F40C94685E0E941D316B017C01002ECD
:10E1E000000C110B20E030E0A9010F941D6287FFA5
:10E1F00004C0F7FAF094F7F8F09420E030E84BE32D
:10E2000054E4C701B6010F941D62980143E0220F48
:10E21000331F4A95E1F728523A4F18169CF0D9015E
:10E220001496CD92DD92ED92FC9217970C94685E55
:10E2300080E090E8ABE3B4E4F90180839183A283AA
:10E24000B383C2CF80E090E8ABE3B4E4F901848308
:10E250009583A683B7830C94685E0E9450560C94F5
:10E26000685E28E01202F0011124E852FA4FC080E3
:10E27000D180E280F3800C94D465A0909D09B09089
:10E280009E09C0909F09D090A0098BE40E9495310F
:10E29000882339F10E941D317B018C0120E030E0A0
:10E2A000A9010F941D6287FD0AC020E030E040E222
:10E2B00051E4B701C8010F94CB581816A4F48FE3AA
:10E2C0000E9449368BE40E94493680E792E10E9421
:10E2D000823688E692E10E94823685E692E10E94CB
:10E2E0008236750186019701A801B501C6010F9418
:10E2F000CB58882361F00E94FEE1C701D8018093CA
:10E300009D0990939E09A0939F09B093A0098091C5
:10E31000010590910205A0910305B0910405892B98
:10E320008A2B8B2B11F00C94685E0E945748409109
:10E330009D0950919E0960919F097091A00984E800
:10E3400092E10E94FA388AE00E9449360C94685E95
:10E3500001110C94D0640E94574888E992E10E9410
:10E36000823680912502811106C083E992E10E94E4
:10E3700082360C94685E8FE892E10E9482360C949B
:10E38000685E81E080931F081092D11360E083E5FE
:10E390000E940A3381110C94685E0F94AA2F0C948A
:10E3A000685E83E50E944731882341F00E9409316D
:10E3B0008093E0050E9427330C94685E0E945748C2
:10E3C00085EA92E10E9482368091E0050E94DC3865
:10E3D0000C94685E0E94E8720C94685E10910605C9
:10E3E0000F94813B60935C0870935D0880935E0896
:10E3F00090935F08112311F40C94685E812F0E94A2
:10E4000049DA0C94685E83E50E949531882311F403
:10E410000C94D6620E9419310C94D06283E50E945C
:10E420009531182F811108C082E50E949531082F7F
:10E43000882311F40C9413690E9419310C94DE683E
:10E4400083E50E949531882311F40C946D690E9434
:10E4500041268B010C946D6983E50E9495318823D8
:10E4600011F40C94685E0E9419310C94EC6983E5F8
:10E470000E949531182F811107C082E50E949531C5
:10E48000882311F40C94685E0E9419310C94146A6C
:10E49000DF92EF92FF920F931F93CF93DF93EC01E4
:10E4A000E0906A08F0906B088AE0D82E6AE070E08D
:10E4B000CE010F940B638C01009711F0FC011082C8
:10E4C000CE010E94E62B81E00E94D05C011511056F
:10E4D00019F0E801D992EACFC701DF91CF911F91DE
:10E4E0000F91FF90EF90DF900C94E62B4F925F928C
:10E4F0006F927F928F929F92AF92BF92CF92DF9254
:10E50000EF92FF920F931F93CF93DF93CDB7DEB7B8
:10E510007C014DB65EB660906A0870906B088DB64F
:10E520009EB66AE070E0C7010F9406586C018C013A
:10E530000E191F09892B21F4C7010F9418588C015B
:10E54000C80101962DB73EB7281B390B0FB6F894BA
:10E550003EBF0FBE2DBF8DB79EB701965C01A801CF
:10E56000B7010F943958F501E00FF11F1082C50172
:10E570000E94E62B81E00E94D05CC114D10451F0CE
:10E5800076019FEFE91AF90A0FB6F8949EBE0FBE06
:10E590008DBEC5CF0FB6F8949EBE0FBE8DBEC30113
:10E5A0000E94E62B0FB6F8945EBE0FBE4DBEDF9103
:10E5B000CF911F910F91FF90EF90DF90CF90BF9080
:10E5C000AF909F908F907F906F905F904F90089545
:10E5D0004F925F926F927F928F929F92AF92BF9273
:10E5E000CF92DF92EF92FF920F931F93CF93DF931F
:10E5F000CDB7DEB7C059D1090FB6F894DEBF0FBE54
:10E60000CDBF0E943533882369F083E50E944731EE
:10E61000882301F120E040E070E060E088ED97E8B9
:10E620000E949A83C057DF4F0FB6F894DEBF0FBE2B
:10E63000CDBFDF91CF911F910F91FF90EF90DF90B1
:10E64000CF90BF90AF909F908F907F906F905F9092
:10E650004F90089583E40E944731882319F00E9467
:10E66000CD87E0CF80905C0990905D09A0905E0915
:10E67000B0905F098091650980FF05C090916B1093
:10E68000986090936B10869581708093B70986E7A8
:10E690009FE00E9476728091EB089091EC089E01B9
:10E6A0002F5F3F4F7901009799F09F938F938DE6ED
:10E6B0009FE09F938F933F932F930F946258C701CE
:10E6C0000E9448720F900F900F900F900F900F9034
:10E6D0008091E9089091EA08009799F09F938F93B1
:10E6E00084E69FE09F938F93FF92EF920F9462587E
:10E6F000C7010E9448720F900F900F900F900F90DB
:10E700000F906E0131E8C30ED11C6091C808709162
:10E71000C9088091CA089091CB08860123E041E0A6
:10E720000F9498539F938F9382E59FE09F938F93CD
:10E73000FF92EF920F946258C7010E9448728AE4D8
:10E740009FE00E94767287E08093D9078093C3058B
:10E750000F900F900F900F900F900F908091E40802
:10E760008823F9F06091E5087091E6088091E70848
:10E770009091E80823E041E00F9498539F938F9382
:10E7800081E49FE09F938F93FF92EF920F946258E2
:10E79000C7010E9448720F900F900F900F900F903A
:10E7A0000F908091ED088823A1F01F928F931F9204
:10E7B0001F9284E39FE09F938F93FF92EF920F94B9
:10E7C0006258C7010E9448720FB6F894DEBF0FBEB0
:10E7D000CDBF8091EE088823A9F01F928F931F92DE
:10E7E00081E08F9384E39FE09F938F93FF92EF925A
:10E7F0000F946258C7010E9448720FB6F894DEBFAA
:10E800000FBECDBF4090EF085090F0086090F10827
:10E810007090F20820E030E0A901C301B2010F942A
:10E82000CB58811104C08091650982FF20C0860108
:10E8300021E041E0C301B2010F9498539F938F935D
:10E840008091650982FB882780F91F928F9387E268
:10E850009FE09F938F93FF92EF920F946258C701AE
:10E860000E9448720FB6F894DEBF0FBECDBF609114
:10E87000BA087091BB088091BC089091BD088E01C8
:10E880000F581F4F23E041E00F949853782E692EC4
:10E890006091B6087091B7088091B8089091B90856
:10E8A000860123E041E00F9498536F927F929F93EB
:10E8B0008F9386E19FE09F938F93FF92EF920F9447
:10E8C0006258C7010E9448726091BE087091BF08EB
:10E8D0008091C0089091C10823E041E00F949853C3
:10E8E0008BE09FE00E947672DF92CF9281E09FE002
:10E8F0009F938F93FF92EF920F946258C7010E94EB
:10E9000048728091C7088F938091C6088F938AEFD1
:10E910009EE09F938F93FF92EF920F946258C701EE
:10E920000E9448726091C2087091C3088091C40827
:10E930009091C50823E041E00F9498539F938F93E3
:10E9400080EF9EE09F938F93FF92EF920F94625817
:10E95000C7010E9448728CE0ECECF8E0A9EAB8E04C
:10E9600001900D928A95E1F78CE0E8EDF8E0ADE9D1
:10E97000B8E001900D928A95E1F780E00E94E9F5F8
:10E9800081E00E94E9F582E00E94E9F58091640946
:10E9900080937E0881E08093E0050E94273383EF17
:10E9A00098E09F938F938FEF98E39F938F93FF92BD
:10E9B000EF920F9462580FB6F894DEBF0FBECDBF32
:10E9C000C7010E944872809163098F938091620908
:10E9D0008F93809161098F93809160098F93BF928B
:10E9E000AF929F928F9282EE9EE09F938F93FF92C1
:10E9F000EF920F946258C7010E9448720FB6F894C4
:10EA0000DEBF0FBECDBF0ECE4F925F926F927F9250
:10EA10008F929F92AF92BF92CF92DF92EF92FF922E
:10EA20000F931F93CF93DF9300D000D01F921F92BC
:10EA3000CDB7DEB783E50F947633863028F087E3D1
:10EA40009EE00E9482363FC0833009F464C1B0F476
:10EA5000813021F1823009F450C084E29EE00E94AE
:10EA600082360E940B358823A1F08091B4100E9459
:10EA7000DC380E945D380F94B00025C0843009F462
:10EA800090C1853051F780E00E9410340E9400341C
:10EA9000F2CF86E19EE00E948236EDCF0E940034E4
:10EAA00010920E0210920D0280911405811125C062
:10EAB0008EE40E94473181111DC084E09EE0909356
:10EAC000DD078093DC0728960FB6F894DEBF0FBEF3
:10EAD000CDBFDF91CF911F910F91FF90EF90DF900D
:10EAE000CF90BF90AF909F908F907F906F905F90EE
:10EAF0004F9008958AE09EE0E2CF80910D029091C0
:10EB00000E0297FF03C08BED9DE09BCF009709F0AD
:10EB1000A8C01D821E821F8218868DEC9CECACE47E
:10EB2000BEE389839A83AB83BC83BE016B5F7F4F57
:10EB3000CE0101960E94AAF780910D0290910E02DB
:10EB4000893191050CF0B3C021E0209339029C017A
:10EB50002F5F3F4F30930E0220930D0265E00F941C
:10EB60007E5F80FF03C024E0291B922F24E09202E5
:10EB7000F0011124E654F94E80809180A280B38088
:10EB800094E08902F0011124EA55F94E4080518049
:10EB9000628073808DEC9CECACE4BEE38D839E833D
:10EBA000AF83B88719821A821B821C82CE0101961C
:10EBB0006C01E12CF12C00EA10E4A3019201C501E3
:10EBC000B4010E94F2F619821A821B821C82B601DD
:10EBD000CE0105960E94AAF78092B5109092B610C9
:10EBE000A092B710B092B8104092B9105092BA10DB
:10EBF0006092BB107092BC101092140500910D022F
:10EC000010910E0289E1E82EF12C093111050CF466
:10EC10007801B70184E79DE00E94143E69E170E04D
:10EC20008FE69DE00E94143E8AE00E94493610164D
:10EC300011060CF020CF1F9289E18F93FF92EF9283
:10EC400088E59DE09F938F9386E69DE09F938F9349
:10EC50001F920E9419B70FB6F894DEBF0FBECDBF4A
:10EC60000ACF815065E00F947E5F80FF03C024E0EF
:10EC7000291B922F25E09202F0011124E80FF11DCB
:10EC800087FDFA95EE0FFF1FEE0FFF1FEF51FA4FB2
:10EC90008091BD109091BE10A091BF10B091C01096
:10ECA00080839183A283B3831092390245CF80E0A1
:10ECB00090E0A0EAB0E48093BD109093BE10A093C2
:10ECC000BF10B093C01080E892E00E94D7F60E9477
:10ECD000FEE18FEF9FEF90930E0280930D0287EC81
:10ECE0009DE00E94823685EB9DE00F948E4863E99B
:10ECF00072E084E690E00E9494806AEB72E084E621
:10ED000090E00E9494808FEA9DE00E94767281E0FC
:10ED10000E94103471CF89E40E949531882371F0EC
:10ED20000E941931182F853068F064E070E08CE99A
:10ED30009DE00E94143E89E99DE083CE8AE40E9412
:10ED4000C737C1CE8AE40E9495318823B9F30E9467
:10ED50001931082F853048F064E070E086E89DE0C6
:10ED60000E94143E83E89DE06CCE8AE50E949531B6
:10ED70008823A9F00E941D3125E01202F001112420
:10ED8000E00FF11D07FDFA95EE0FFF1FEE0FFF1FBD
:10ED9000EF51FA4F60837183828393836CCE8AE54F
:10EDA000CECF8AE50E9495318823C9F30E941D3198
:10EDB00060934506709346068093470690934806F5
:10EDC0005ACECF93DF93C091B311C093780981E6F7
:10EDD000C89FE0011124CB54DE4E80916B1080FF60
:10EDE00005C00E945748CE010E945036CE010E94B5
:10EDF000E62B80E0DF91CF910C94D05C8F929F92B4
:10EE0000AF92BF92CF92DF92EF92FF92CF936B01BE
:10EE10007C0120E030E0A9010F94CB5887FFA3C00C
:10EE20006DEB77E386E095EBA70196010F94BD5F4C
:10EE30006B017C0120E030E040E251E40F94315955
:10EE400020E030E048EC52E40F9431594B015C0172
:10EE500020E030E040E251ECC701B6010F94CB58FE
:10EE6000181654F420E030E048EC52E4C701B60133
:10EE70000F941D6287FD8BC020E030E0A901C7011F
:10EE8000B6010F94CB5887FF73C060E070E080EA52
:10EE900090ECA50194010F94BD5F20E030E040E2CA
:10EEA00051E40F94B7600F9429616B017C01F7FC6A
:10EEB00064C020E137E240E050E00F94315FCA01C6
:10EEC000B9012AE030E040E050E00F94315F605D2E
:10EED0006093BC05C701B60128EE33E040E050E086
:10EEE0000F94315F9AE0892E912CA12CB12CCA018C
:10EEF000B901A50194010F94315F605D6093BD0578
:10EF0000C701B60124E630E040E050E00F94315FE5
:10EF1000CA01B901A50194010F94315F605D60934E
:10EF2000BE058EE28093BF05C701B601A50194011D
:10EF30000F94315FC62FCA01B901A50194010F9446
:10EF4000315F605D6093C005C05DC093C1058CEB0F
:10EF500095E0CF91FF90EF90DF90CF90BF90AF9072
:10EF60009F908F9008956DEB77E386E095E35CCFFB
:10EF700060E070E080EA90E48CCFF094E094D0946C
:10EF8000C094C11CD11CE11CF11C6DE2A1CF20E09A
:10EF900030E0A901C701B6010F94CB5887FF6AC0C2
:10EFA00060E070E080EA90ECA50194010F94BD5FF1
:10EFB00020E030E040E251E40F94B7600F94296103
:10EFC0004B015C0120E030E0A901C701B6010F94BC
:10EFD0001D6287FD0BC020E030E040E251E4C70134
:10EFE000B6010F94CB5860E287FD13C0B7FC47C051
:10EFF000C501B40128EE33E040E050E00F94315FEA
:10F00000CA01B9012AE030E040E050E00F94315FDE
:10F01000605D6093BD05C501B40124E630E040E0C9
:10F0200050E00F94315F8AE0C82ED12CE12CF12CF6
:10F03000CA01B901A70196010F94315F605D609329
:10F04000BE058EE28093BF05C501B401A7019601FC
:10F050000F94315FC62FCA01B901A70196010F9421
:10F06000315F605D6093C005C05DC093C1058DEBED
:10F0700095E06FCF60E070E080EA90E495CFB094C7
:10F08000A09490948094811C911CA11CB11C6DE2F1
:10F09000C0CF6091360270913702072E000C880BAA
:10F0A000990B0F94D2582AE037ED43E25CE30F94BA
:10F0B00031592091CC053091CD054091CE0550912C
:10F0C000CF050F9431596093850270938602809327
:10F0D0008702909388020895E0914708E23030F467
:10F0E000F0E0EB55F64F80913D08808308958091C4
:10F0F000CE168823C1F081508093CE16EAEFF6E158
:10F10000882351F08150990B2BE1289FF001299F12
:10F11000F00D1124E05DF84E8BE1A5E1B7E101901F
:10F120000D928A95E1F72091CE16211105C08091AC
:10F13000D91680628093D91681E090E0A0E0B0E01B
:10F14000211103C080E090E0DC01809335089093AA
:10F150003608A0933708B093380810923A0881E037
:10F160008093340883E0809384020895CF93DF93E3
:10F17000EC01CB01BA010F94D25829EC38EC48ECE1
:10F180005EE30F94B76020E030E040E05FE30F946F
:10F19000BD5F0F9430616883DF91CF9108958091B6
:10F1A0005202909153020C944A27E091470886E05E
:10F1B000E802F0011124E05EF74F80913D0890E0F5
:10F1C000958384830895CF93DF93EC01CB01BA013B
:10F1D0000F94D25820E030E0A9010F94BD5F0F9446
:10F1E00030616883DF91CF9108958F929F92AF92A3
:10F1F000BF92CF92DF92EF92FF92CF936B017C018F
:10F2000020E030E0A9010F94CB5887FD9FC06DEB43
:10F2100077E386E095E3A70196010F94BD5F6B014C
:10F220007C0120E030E040E251E40F94315920E0CD
:10F2300030E048EC52E40F9431594B015C0120E07E
:10F2400030E0A901C701B6010F94CB5820E030E0AF
:10F2500040EA50E487FF04C020E030E040EA50EC90
:10F26000C501B4010F94BD5F20E030E040E251E4FD
:10F270000F94B7600F9429616B017C018BE2F7FE5C
:10F2800009C0F094E094D094C094C11CD11CE11C3E
:10F29000F11C8DE28093BB05C701B60120E137E286
:10F2A00040E050E00F94315F8AE0882E912CA12C31
:10F2B000B12CCA01B901A50194010F94315F605DC1
:10F2C0006093BC05C701B60128EE33E040E050E092
:10F2D0000F94315FCA01B901A50194010F94315F08
:10F2E000605D6093BD05C701B60124E630E040E0F3
:10F2F00050E00F94315FCA01B901A50194010F9448
:10F30000315F605D6093BE058EE28093BF05C701EB
:10F31000B601A50194010F94315FC62FCA01B9014E
:10F32000A50194010F94315F605D6093C005C05DDD
:10F33000C093C1058BEB95E0CF91FF90EF90DF90EC
:10F34000CF90BF90AF909F908F9008956DEB77E333
:10F3500086E095EB60CF8F929F92AF92BF92CF9253
:10F36000DF92EF92FF92CF936B017C0120E030E0BF
:10F37000A9010F94CB5887FDAAC06DEB77E386E017
:10F3800095E3A70196010F94BD5F6B017C0120E01E
:10F3900030E0A9010F94CB5887FF9EC0C701B6018A
:10F3A000905820E030E040E251E40F94315920E0E1
:10F3B00030E040E251E40F94315920E030E040EA7F
:10F3C00050E40F94BD5F20E030E040E251E40F9440
:10F3D000B7600F9429616B017C0180E28093BB05CB
:10F3E00060E280E1C81687E2D806E104F1048CF0FF
:10F3F000C701B60120E137E240E050E00F94315FF1
:10F40000CA01B9012AE030E040E050E00F94315FDA
:10F41000605D6093BC0560E288EEC81683E0D806A4
:10F42000E104F1048CF0C701B60128EE33E040E0BE
:10F4300050E00F94315FCA01B9012AE030E040E0AA
:10F4400050E00F94315F605D6093BD0560E284E63B
:10F45000C816D104E104F1048CF0C701B60124E61A
:10F4600030E040E050E00F94315FCA01B9012AE07A
:10F4700030E040E050E00F94315F605D6093BE0586
:10F480008AE0882E912CA12CB12CC701B601A501D0
:10F4900094010F94315FC62FCA01B901A5019401EF
:10F4A0000F94315F605D6093BF058EE28093C0056D
:10F4B000C05DC093C1058BEB95E0CF91FF90EF90BD
:10F4C000DF90CF90BF90AF909F908F9008956DEB9D
:10F4D00077E386E095EB55CF20E030E040E251E461
:10F4E000C701B60162CFCF93DF93EC01CB01BA0124
:10F4F0000F94D25820E030E040E251E40F94B7601E
:10F5000020E030E0A9010F94BD5F688379838A838E
:10F510009B83DF91CF910895CF93DF93EC01CB01D3
:10F52000BA010F94D25820E030E040E251E40F9449
:10F53000B76020E030E0A9010F94BD5F6883798354
:10F540008A839B83DF91CF9108950F94D25820E056
:10F5500030E040E251E40F94B76020E030E0A901D0
:10F560000F94BD5F0C94AB79CF93DF93EC01CB018B
:10F57000BA010F94D2582AE037ED43E25DE30F94CD
:10F58000B76020E030E0A9010F94BD5F0F943061B7
:10F59000688379838A839B83DF91CF910895CF938A
:10F5A000DF93EC01CB01BA010F94D2582AE037ED7A
:10F5B00043E25DE30F94B76020E030E0A9010F94CF
:10F5C000BD5F688379838A839B83DF91CF910895A0
:10F5D000CF93DF93EC01CB01BA010F94D25820E016
:10F5E00030E0A9010F94BD5F688379838A839B8390
:10F5F000DF91CF910895CF93DF93EC01CB01BA0156
:10F600000F94D25820E030E0A9010F94BD5F6883C9
:10F6100079838A839B83DF91CF910895CF93DF9382
:10F62000EC01CB01BA010F94D25820E030E048EC55
:10F6300052E40F94B76020E030E0A9010F94BD5F61
:10F64000688379838A839B83DF91CF910895CF93D9
:10F65000DF93EC01CB01BA010F94D25820E030E0E7
:10F6600048EC52E40F94B76020E030E0A9010F9419
:10F67000BD5F688379838A839B83DF91CF910895EF
:10F680000F94D25820E030E048EC52E40F94B76079
:10F6900020E030E0A9010F94BD5F0C94F578CF9382
:10F6A000DF93EC01CB01BA010F94D25820E030E097
:10F6B000A9010F94BD5F0F94296179836883DF915D
:10F6C000CF910895CF93DF93EC01CB01BA010F9452
:10F6D000D25820E030E0A9010F94BD5F68837983A0
:10F6E0008A839B83DF91CF910895CF93DF93EC01C1
:10F6F000CB01BA010F94D25820E030E04AE754E43D
:10F700000F94B76020E030E0A9010F94BD5F6883DB
:10F7100079838A839B83DF91CF9108950F94D25888
:10F7200020E030E048EC52E40F94B76020E030E095
:10F73000A9010F94BD5F0C94FE762CEA35EC47E2EC
:10F740005EE36091A9057091AA058091AB05909147
:10F75000AC050F94B7606093F8157093F91580931A
:10F76000FA159093FB1508952CEA35EC47E25EE319
:10F770006091AD057091AE058091AF059091B00597
:10F780000F9431596093F4157093F5158093F61525
:10F790009093F71508952CEA35EC47E25EE360910B
:10F7A000A9057091AA058091AB059091AC050F94C5
:10F7B000B7606093F8157093F9158093FA159093DC
:10F7C000FB1508952CEA35EC47E25EE36091AD0548
:10F7D0007091AE058091AF059091B0050F943159AD
:10F7E0006093F4157093F5158093F6159093F715C3
:10F7F000089580913D0890913E08A0913F08B091F6
:10F8000040088093550290935602A0935702B093FC
:10F8100058020895E091A205E63010F581E08E0FC0
:10F820008093A205409135085091360860913708C1
:10F830007091380890913A088091330828E0E29F4F
:10F84000F0011124ED59FA4F20916516309166169A
:10F8500031832083428353836483758396838783B4
:10F860000895FC01A081B1811C92A281B3818C9189
:10F870008F5F8C930280F381E02D90818CE0989FC4
:10F88000800D1124E7E6F6E113AE84AF0895CF9220
:10F89000DF92EF92FF92CF93DF9300D01F92CDB70C
:10F8A000DEB76B017C0120E030E0A9010F94CB585A
:10F8B00087FD1CC06DEB77E386E095E3A701960119
:10F8C0000F94BD5F69837A838B839C8360E2CE0152
:10F8D00001960F94EC040F900F900F900F90DF9112
:10F8E000CF91FF90EF90DF90CF9008956DEB77E38D
:10F8F00086E095EBE3CF0F94D25820E030E04AE762
:10F9000054E40F94B76020E030E0A9010F94BD5F8C
:10F910000C94477CCF92DF92EF92FF926B017C01B7
:10F9200020E030E0A9010F94CB5887FD26C06DEB95
:10F9300077E386E095E3A70196010F94BD5F6B0125
:10F940007C0120E030E0A9010F94CB5820E030E0AA
:10F9500040E05FE387FF04C020E030E040E05FEB81
:10F96000C701B6010F94BD5F0F942961CB01FF90D1
:10F97000EF90DF90CF900D94AE066DEB77E386E0CD
:10F9800095EBD9CF0F94D25820E030E0A9010F9425
:10F99000BD5F0C948A7C0F94D25820E030E0A9011E
:10F9A0000F94BD5F0F942961CB010D94AE060F94A7
:10F9B000D25829EC38EC48EC5EE30F94B76020E0B5
:10F9C00030E040E05FE30F94BD5F0F943061862F1D
:10F9D0000D9405070D948D3B0D948D3B6FEF809139
:10F9E0003D080D941E396CED76EB82E00D94744A5F
:10F9F00061EE76EB81E00D94744A66EE76EB80E082
:10FA00000D94744A67E974EB83E00D94744ACF92C5
:10FA1000DF92EF92FF92CF93DF9300D01F92CDB78A
:10FA2000DEB76B017C0120E030E0A9010F94CB58D8
:10FA300087FD1BC06DEB77E386E095E3A701960198
:10FA40000F94BD5F69837A838B839C83CE0101967B
:10FA50000F9488050F900F900F900F90DF91CF912A
:10FA6000FF90EF90DF90CF9008956DEB77E386E005
:10FA700095EBE4CF0F94D25820E030E040E251E41F
:10FA80000F94B76020E030E0A9010F94BD5F0C94A3
:10FA9000077D80912F1690913016891B8F7011F47D
:10FAA0000C94A23581E0089581E00C94C2338091DA
:10FAB0008402882351F06091A7057091A80530E079
:10FAC00020E041E081E00C944729089584E00D9402
:10FAD000ED3783E00D94ED3782E00D94ED370F9410
:10FAE000D25820E030E0A9010F94BD5F0F9430613F
:10FAF000862F0D94E3069091B41081E089270C9431
:10FB0000103461E08DE398E00C942B340F94EB2FCC
:10FB10000C94F9F780E090E0A0E8B0E48093BD1089
:10FB20009093BE10A093BF10B093C01083EE92E0EC
:10FB30000E94D7F6E091B205E430C9F480E090E08D
:10FB4000A8ECB2E48093B5109093B610A093B710D0
:10FB5000B093B81080E090E8AAECB2E48093B910BA
:10FB60009093BA10A093BB10B093BC102EC080E04D
:10FB700090E0A0EBB1E48093B5109093B610A09301
:10FB8000B710B093B8108093B9109093BA10A093A7
:10FB9000BB10B093BC10EE0FFF0BED53FD4F8081F7
:10FBA00091818330910549F18430910591F102975B
:10FBB00061F480E090E0A2E3B3E48093B510909309
:10FBC000B610A093B710B093B8108BEC92E00E94DF
:10FBD000D7F61092BD101092BE101092BF10109266
:10FBE000C01083EE92E00E94D7F68091B2058F5F3D
:10FBF0008530A4F48093B205089580E090E0A2E3FC
:10FC0000B3E48093B5109093B610A093B710B0935F
:10FC1000B81080E090E8A4E3B3E4A0CF1092B2055E
:10FC20000895CF93DF9300D01F92CDB7DEB70F9426
:10FC300030610F94D05869837A838B839C83CE0183
:10FC400001960F9469040F900F900F900F90DF9121
:10FC5000CF9108950F94D2582AE037ED43E25DE347
:10FC60000F94B76020E030E0A9010F94BD5F0C94C1
:10FC7000117ECF92DF92EF92FF92CF93DF9300D06D
:10FC80001F92CDB7DEB76B017C0120E030E0A90107
:10FC90000F94CB5887FD1BC06DEB77E386E095E3AF
:10FCA000A70196010F94BD5F69837A838B839C8340
:10FCB000CE0101960F9469040F900F900F900F9052
:10FCC000DF91CF91FF90EF90DF90CF9008956DEB93
:10FCD00077E386E095EBE4CF0F94D2582AE037ED36
:10FCE00043E25DE30F94B76020E030E0A9010F9498
:10FCF000BD5F0C94397E0F94D25820E030E0A9010A
:10FD00000F94BD5F0C94397ECF92DF92EF92FF92F9
:10FD10006B017C0120E030E0A9010F94CB5887FDF6
:10FD200026C06DEB77E386E095E3A70196010F947B
:10FD3000BD5F6B017C0120E030E0A9010F94CB583E
:10FD400020E030E040E05FE387FF04C020E030E0E7
:10FD500040E05FEBC701B6010F94BD5F0F942961CE
:10FD6000CB01FF90EF90DF90CF900D9404066DEBE8
:10FD700077E386E095EBD9CF0F94D25820E030E0BE
:10FD8000A9010F94BD5F0C94847E0C94DAE10C946D
:10FD9000DAE10C94DAE10C94DAE10C948CE10C9445
:10FDA0008CE10C948CE10C948CE1CF92DF92EF9279
:10FDB000FF92CF93C82F0F94813B6B017C0124EA03
:10FDC00030E74DE75FE36091260270912702809152
:10FDD0002802909129020F94CB5887FD18C08AEF12
:10FDE00090E0A0E0B0E08C0D9D1DAE1DBF1D809386
:10FDF0004D0590934E05A0934F05B0935005C093C9
:10FE00001E02CF91FF90EF90DF90CF90089580E099
:10FE100090E0DC01E8CFCF92DF92EF92FF920F9358
:10FE20001F930F94813B00911E0510911F05209197
:10FE30002005309121056B017C01C01AD10AE20A2C
:10FE4000F30A9701860137FD11C020911D05209509
:10FE500020931D056A547C4F8F4F9F4F60931E0562
:10FE600070931F05809320059093210581E0909168
:10FE70001D05911101C080E01F910F91FF90EF903F
:10FE8000DF90CF9008950F94C048109267081092A9
:10FE900078020E94CD35882351F08091D91682FDD9
:10FEA00006C089EC9EE19093DD078093DC0761E05A
:10FEB00082EC9EE10E94CD370D941C044F925F921C
:10FEC0006F927F928F929F92BF92CF92DF92EF922A
:10FED000FF920F931F93CF93DF9300D000D01F9218
:10FEE0001F92CDB7DEB77C016A014901FB01908109
:10FEF0008CE0989F800D1124982FF7012081822F8C
:10FF0000880F820F880F8093A2169093A316411535
:10FF1000510571F1FA82E9827C836B83011121C062
:10FF2000AE014B5F5F4FB401C6010E9451266C01C8
:10FF30006D817E818F81988561157105810591059F
:10FF4000B9F00E94E427F70180818F5F80838531BB
:10FF500038F3CE0101960E94317CE2CFB12C8601AC
:10FF600029C08A01B12C26C0452846284728B1F768
:10FF700028960FB6F894DEBF0FBECDBFDF91CF91AC
:10FF80001F910F91FF90EF90DF90CF90BF909F90C7
:10FF90008F907F906F905F904F900895B39407C0BB
:10FFA000B1102EC001151105C9F20F5F1F4F0115C9
:10FFB0001105A9F2AE014B5F5F4FB401C6010E946B
:10FFC00051266C014D805E806F807884411451040D
:10FFD00061047104A9F0F0E24F1651046104710448
:10FFE000F9F2D301C2018D97A109B1090297A105C8
:10FFF000B10530F04BE2441651046104710471F60E
:020000021000EC
:10000000F7018081482F4B0D5527551F463151056B
:1000100034F0853020F0CE0101960E94317C81E0E1
:10002000411451046104710409F480E0B80EF70131
:1000300080818B0D8083BB2009F496CFBA94AE01EA
:100040004B5F5F4FB401C8010E9451268C016D8146
:100050007E818F8198850E94E427EDCFEF92FF92F9
:100060000F931F93CF93DF9300D000D000D01F9247
:100070001F92CDB7DEB77C0120913B08422F022EA4
:10008000000C550B80913C08833099F1843051F17C
:100090008FE692E25F932F939F938F938E010F5F72
:1000A0001F4F1F930F930F946258C7010E9477E16F
:1000B0004FE350E0B8018EED97E00F942B630F9063
:1000C0000F900F900F900F900F902B960FB6F89403
:1000D000DEBF0FBECDBFDF91CF911F910F91FF907B
:1000E000EF9008958BE792E227FDD4CF86E692E267
:1000F000D1CF84E892E2CECFE091470885E1E802D3
:10010000F0011124E951FA4E868197810C942E80DA
:10011000E091470886E0E802F0011124E05EF74F25
:10012000808191810C942E800F931F93CF93DF9346
:100130008C01EB019091531620915416921305C037
:100140000F94EB070E94FBF7F5CF8091521634E035
:10015000839FF0011124EB5AF94E11830083D3835E
:10016000C2839F5F909353168F5F281739F0809357
:100170005216DF91CF911F910F9108951092521650
:10018000F8CF63E972E084E690E00E9494806AEB25
:1001900072E084E690E00C94948081110C94C1800C
:1001A00068EB71E084E190E00C9494800E94C8DDDB
:1001B0000C94CD800F94F1180C94CD800F94CE0147
:1001C0000C94C180CF93DF93CDB7DEB720E2488592
:1001D00059856F818E810F942A35DF91CF910895D3
:1001E000282F109245088091350890913608A091EB
:1001F0003708B0913808B7FF08C010923508109240
:10020000360810923708109238088091BA05882372
:1002100031F080913508809339081092340880912C
:1002200033081816FCF4082E000C990B821B910958
:1002300020913908022E000C330B2817390794F04F
:1002400097FF02C090E080E080933908092E000CEF
:10025000AA0BBB0B8093350890933608A093370800
:10026000B0933808809139086623A9F090913A0834
:10027000891714F480933A0820913A08022E000C52
:10028000330B2C5F3F4F482F082E000C550B2417C3
:1002900035071CF4845080933A0808955F926F925A
:1002A0007F928F929F92AF92BF92CF92DF92EF9206
:1002B000FF920F931F93CF93DF9361E081E00E9441
:1002C000F080C0913A0885E0982E9C0ED1E092EC27
:1002D000E92E92E2F92E882483947D2E7C1A6C2ECE
:1002E000619424EAC22E22E2D22E12E01C1B33E0DB
:1002F000532E4DE6A42E42E2B42EC11141C0DD239F
:10030000D9F0809139081816BCF040913508509109
:10031000360860913708709138084F5F5F4F6F4F14
:100320007F4F409335085093360860933708709399
:1003300038088F5F8093390880918402882341F0C8
:1003400030E020E041E06DEC72E2862D0E9447290A
:1003500080916508882309F487C0C23051F48091E8
:100360003908823009F445C08091840281115AC055
:10037000D0E0CF5F9C12C1CF83E08093330818C0D8
:10038000C13031F790913908913031F08091840279
:1003900081111EC0D0E0DCCF80913208109232086B
:1003A0008823A1F3C093660880913408882371F3F1
:1003B000DF91CF911F910F91FF90EF90DF90CF9041
:1003C000BF90AF909F908F907F906F905F900895B7
:1003D0001F92FF92EF927F9281E0913009F080E0CE
:1003E0008F930E94E2800F900F900F900F900F90CC
:1003F000D1CF8091320810923208882309F4B4CF0B
:100400008091590288258093590250928402A11448
:10041000B10411F00E946D2280913408882309F400
:10042000A3CFC6CF81E090913908923009F080E0E7
:100430009091590221EB32E2911102C02DEA32E291
:1004400001E044EB52E2612F0E94422A91CF809159
:10045000320810923208882371F0C09366088091A8
:100460003408882341F0A4CFC23009F082CF9091A4
:100470003908923061F380918402882309F478CF9F
:100480001F92DF92CF921F9381E0923009F080E0BB
:100490008F930E94E2800F900F900F900F900F901B
:1004A00067CF2F923F924F925F926F927F928F927F
:1004B0009F92AF92BF92CF92DF92EF92FF920F93F3
:1004C0001F93CF93DF934C010F941858019684012A
:1004D000080F191FC8010F94185801966801C80E1B
:1004E000D91EF8016080C1E0611001C0C0E0F601D2
:1004F0003080D1E0311001C0D0E0AA24A394611073
:10050000A12C60E085E00E94F08050903A08752CA4
:100510009EE0E92EF12C252C21948A2D90E0019665
:100520005C01AC0EB11CAD0EB11C71101DC08091F0
:1005300084028823A1F0E0912402E2506DED72E282
:10054000E33038F4F0E0EE0FFF1FE551FD4F60811E
:10055000718130E020E043E0822D0E944729D1E004
:10056000611013C0D2E011C0D2E06110D1E0D71108
:100570000CC080918402882341F030E020E041E00B
:10058000B4018D2F85190E944729C1E0CD0F472C5A
:100590004518662079F0C7110BC08091840288232A
:1005A00039F030E020E041E0B801842D0E94472975
:1005B000C2E0CD0F332071F0C7110BC080918402CF
:1005C000882339F030E020E041E0B601842D0E941C
:1005D0004729CF5FF3E0AF16B1040CF4CF5FC7112A
:1005E00062C080918402882309F45AC030E020E080
:1005F00042E06AEE72E2842D0E944729D0911B05E9
:1006000093EF9E0D90931A058EEF8E0D8093460802
:1006100020919F162E151F0411F00CF041C020915F
:10062000A1169217E8F59EE39093A2168093A31665
:1006300065E470E080E090E00E94E42761E36D0FE4
:10064000062E000C770B880B990B0E94E42760E2C2
:1006500070E080E090E00E94E4278091EB1590919B
:10066000EC150F94AE060E94BF296FE270E080E0A7
:1006700090E00E94E4270E940B7F811109C085E071
:100680008D9FF0011124E85AF94F8481811108C02F
:100690008091ED159091EE150F94AE060E94BF2942
:1006A00092E090938402ECE0EE0EF11C7394FAE475
:1006B000EF16F10409F039CFCF5FC0933308DF9113
:1006C000CF911F910F91FF90EF90DF90CF90BF904F
:1006D000AF909F908F907F906F905F904F903F90E2
:1006E0002F90089585EF92E20C94518282E093E27C
:1006F0000C94518284E293E20C9451828FEB93E24A
:100700000C9451828AE793E20C94518287EA93E237
:100710000C9451828AEF93E20C9451828DED93E216
:100720000C9451828DE593E20C9451828EE393E216
:100730000C9451828F929F92AF92BF92EF92FF9250
:100740000F931F93CF93DF93EC018B01E42EF22ED6
:1007500080916516909166168C179D0709F43EC02E
:100760002091130527FD1092130527EBC23BD207FA
:1007700009F03FC08255914C71F40F94813B6E514A
:100780007B4F8F4F9F4F6093A3057093A405809379
:10079000A5059093A605D0936616C093651630E024
:1007A00020E00093350810933608209337083093E3
:1007B0003808E0923A08F0923308C255D14C21F43F
:1007C00010921C051092A20582E08093840281E0C1
:1007D000809334081092B7051092B105DF91CF9144
:1007E0001F910F91FF90EF90BF90AF909F908F90CF
:1007F000089521ECC235D20771F6825B974B19F050
:10080000C2E5D1ECC8CF0F94813B8090A3059090B6
:10081000A405A090A505B090A605681979098A09D4
:100820009B0997FFEDCF8091D9078770873041F7FB
:10083000C9E2D4E8B0CFCF93DF93EC010E940A7CE9
:1008400020E040E070E060E0CE01DF91CF910C94B9
:100850009A8320E040E070E060E080EA93EB0E9441
:100860009A8381E080931C051092630810926208BD
:10087000089520E040E070E060E082E09DE70C94A5
:100880009A838091B709811114C080918902909157
:100890008A0201972091EB153091EC152817390742
:1008A00044F420E040E070E060E087E390EC0C94DA
:1008B0009A830C94398421E020931C05FC018081EB
:1008C0009181A281B3818093260290932702A09305
:1008D0002802B093290220E040E070E060E08091BF
:1008E0003008909131080C949A83CF93DF9300D015
:1008F0001F92CDB7DEB78DEC9CECACECBCE38983EA
:100900009A83AB83BC83CE0101960E945B840F90D7
:100910000F900F900F90DF91CF910895CF93DF93B9
:1009200000D01F92CDB7DEB78DEC9CECACECBDE3F4
:1009300089839A83AB83BC83CE0101960E945B843A
:100940000F900F900F900F90DF91CF910895CF935C
:10095000DF9300D01F92CDB7DEB780E090E0A0E833
:10096000BFE389839A83AB83BC83CE0101960E9447
:100970005B840F900F900F900F90DF91CF910895AF
:10098000CF93DF9300D01F92CDB7DEB780E090E029
:10099000A0E2B1E489839A83AB83BC83CE01019644
:1009A0000E945B840F900F900F900F90DF91CF917A
:1009B00008958FEF80933D0820E040E070E060E014
:1009C00084EB9AE90C949A8381E080931C05109241
:1009D000D9071092C30520E040E070E060E08BE1B1
:1009E00095E80E949A838AE797E29093DD078093C7
:1009F000DC07089581E080931C058091D9078770FA
:100A0000873051F01092D9071092C3058AE797E218
:100A10009093DD078093DC078091B4108093B30539
:100A200080E00E94103420E040E070E060E08CE65E
:100A300096E80C949A8380918402882341F030E0F8
:100A400020E041E065E071E282E00E944729809168
:100A5000C3058770873041F420E040E070E060E03B
:100A60008EE495E80C949A83089520E040E070E0CD
:100A700060E085E695E80E949A8381E08093140502
:100A80008091B405811107C08AEE90E29093DD0752
:100A90008093DC07089580EF90E2F8CF8091840284
:100AA000882341F030E020E041E066EF70E281E031
:100AB0000E9447298091320810923208882321F041
:100AC0001092B4050C94358508950F931F93CF931E
:100AD000DF9300D000D000D01F92CDB7DEB7809159
:100AE00084028823F1F01F9289E18F938091B405ED
:100AF00090E001969F938F9382EE90E29F938F9365
:100B00008E010F5F1F4F1F930F930F946258B80110
:100B100087ED90E20E94C3290FB6F894DEBF0FBEA6
:100B2000CDBF84E08093840280911405811108C0B8
:100B300020E040E070E060E08BEA95E80E949A8354
:100B40002A960FB6F894DEBF0FBECDBFDF91CF91CE
:100B50001F910F910895CF92DF92EF92FF92CF9362
:100B6000DF9300D01F92CDB7DEB78091320810928C
:100B70003208882331F18091B4058F5F8093B405EA
:100B80008931E0F081E08093140520E040E070E0DE
:100B900060E08BEE96EB0E949A8381ED90E2909359
:100BA000DD078093DC070F900F900F900F90DF917F
:100BB000CF91FF90EF90DF90CF9008950E94358500
:100BC000F2CF609135087091360880913708909186
:100BD0003808611571058105910509F43EC00F942F
:100BE000D2582DEC3CEC4CEC5CE30F943159209145
:100BF000BD103091BE104091BF105091C0100F94A5
:100C0000BD5F6B017C0120E030E040E850EC0F94C8
:100C1000CB5887FD53C020E030E040E850E4C701E6
:100C2000B6010F941D6218160CF44FC0C092BD108F
:100C3000D092BE10E092BF10F092C01083EE92E00E
:100C40000E94D7F682E080938402109235081092B9
:100C50003608109237081092380880918402882351
:100C600009F4A1CFC090BD10D090BE10E090BF108D
:100C7000F090C01020E030E0A901C701B6010F9448
:100C8000CB5827E137EB41ED58E387FF04C027E15C
:100C900037EB41ED58EBC701B6010F94BD5F698397
:100CA0007A838B839C836BE2CE0101960F94EC04D4
:100CB000BC018AEC90E20E94C32975CFC12CD12CD3
:100CC00090E8E92E90ECF92EB1CFC12CD12C80E820
:100CD000E82E80E4F82EAACF80918402882341F088
:100CE00030E020E041E065E071E282E00E944729C7
:100CF0008091C3058770873079F41092B20520E0A7
:100D000040E070E060E089E091EC0E949A8381E02D
:100D10008093B1050C948A7D08952F923F924F9253
:100D20005F926F927F928F929F92AF92BF92CF927B
:100D3000DF92EF92FF920F931F93CF93DF9300D038
:100D400000D0CDB7DEB71C017A8369832B833C8347
:100D50004D835E832701380181E0809334080E942F
:100D60000A7C83E0809384023092A1052092A00542
:100D700089819A8190939F0580939E058B819C81A8
:100D8000AD81BE8180939A0590939B05A0939C05AD
:100D9000B0939D05409296055092970560929805F4
:100DA00070929905F12CE12CC0923508D09236084A
:100DB000E0923708F0923808B0926616A092651655
:100DC00090929505809294058C8D8093930526963C
:100DD0000FB6F894DEBF0FBECDBFDF91CF911F914C
:100DE0000F91FF90EF90DF90CF90BF90AF909F90CA
:100DF0008F907F906F905F904F903F902F900895CD
:100E00002F923F924F925F926F927F928F929F921A
:100E1000AF92BF92CF92DF92EF92FF920F931F9308
:100E2000CF93DF9300D000D000D0CDB7DEB71C0148
:100E30007987688769011A830983EB82BA01550FA4
:100E4000880B990B0F94D25820E030E0A9010F9441
:100E5000BD5F4B015C0120E030E040E05FEC0F94AF
:100E60001D6218162CF0812C912CA12C2FECB22E87
:100E7000C501B4010F9429612B013C01B601DD0CC1
:100E8000880B990B0F94D25820E030E0A9010F9401
:100E9000BD5F4B015C0120E030E040E05FE40F9477
:100EA000CB5887FD05C0812C912CA12C9FE4B92E35
:100EB000E885F98560817181072E000C880B990BFC
:100EC0000F94D25820E030E0A9010F94BD5F6B0170
:100ED0007C01C301B2010F94D2589B01AC01C70140
:100EE000B6010F94BC5F0F9430616C837D838E8359
:100EF0009F83C501B4010F9429617B018C01E41823
:100F0000F50806091709FB81FF9389809A808AE812
:100F1000A82E83EBB82ECC80DD80A30192016885DA
:100F20007985C1010E948D860F9029960FB6F8949D
:100F3000DEBF0FBECDBFDF91CF911F910F91FF900C
:100F4000EF90DF90CF90BF90AF909F908F907F9069
:100F50006F905F904F903F902F90089520E040E079
:100F600070E060E082E591EC0C949A830E94043674
:100F70000E9493DA0C94AE8780E798E00E94F3CF4A
:100F80000E94AE870D94C0480E94AE878FE795E21D
:100F90009093DD078093DC0708950E941F330F9420
:100FA000C54781E08093CF160F9407480C94AE8715
:100FB0006F927F928F929F92AF92BF92CF92DF9269
:100FC000EF92FF920F931F93CF93DF9381E0809373
:100FD0001C0561E00E94F080C0913A0885E0882EEF
:100FE0008C0ED1E00DEC17E895E8E92E95E2F92E8C
:100FF00082E0982E9C1A24ECC22E27E8D22E30E9EB
:10100000A32E35E2B32E7D2E7C1A6C2E6194C11175
:1010100030C0DD23D9F0809139081816BCF040911A
:1010200035085091360860913708709138084F5F45
:101030005F4F6F4F7F4F4093350850933608609352
:101040003708709338088F5F809339088091840245
:10105000882341F030E020E041E06DE975E2862D23
:101060000E944729CF5F8C12D2CF83E08093330850
:1010700023C0C13081F580913908813089F0809199
:101080008402882309F444C0DF92CF92BF92AF92CA
:101090007F9281E090913908913089F180E02FC0F2
:1010A0008091320810923208882349F30E94C48745
:1010B00080913408882319F3DF91CF911F910F910C
:1010C000FF90EF90DF90CF90BF90AF909F908F9068
:1010D0007F906F900895C23029F680913908823050
:1010E000C9F080918402882399F01F930F93FF9297
:1010F000EF929F9281E090913908923079F68F9328
:101100000E94E2800F900F900F900F900F900F9021
:10111000D0E0A8CF8091320810923208882309F3DA
:101120000E94CD87809134088823D9F2C5CF611100
:101130006093240240931B058C3008F03AC0E82FDE
:10114000880FFF0B8827E855F7478F4F0D94B45F42
:10115000DB88B488BF88DE88C288C588C888D48800
:10116000CB88D988CE88D18886E793E821E0209380
:101170001C0520E040E070E060E00C949A838EE76C
:1011800093E8F4CF82E893E8F1CF86E893E8EECFD6
:101190008AE893E8EBCF8EE893E8E8CF82E993E81A
:1011A000E5CF86E993E8E2CF109266088EE491E8F5
:1011B000DDCF0C94AE8782E793E8D8CF8AE793E837
:1011C000D5CFCF930F94CE010E94C8DDC82F8823BE
:1011D00019F080E00F948C118C2F0E94CD80CF915C
:1011E0000C94AE870F931F93CF93DF93CDB7DEB7E9
:1011F0006E970FB6F894DEBF0FBECDBF282F082E16
:10120000000C330B90911F02409120028F3F39F068
:10121000F901EE0FFF1FEF5DFD4F908141814F936C
:101220009F933F938F938CE09FE19F938F938E01C9
:101230000F5F1F4F1F930F930F9462584FE350E0BF
:10124000B8018EED97E00F942B630E94AE870FB626
:10125000F894DEBF0FBECDBF6E960FB6F894DEBF1A
:101260000FBECDBFDF91CF911F910F9108958FEFEA
:101270000C94F288809147080C94F288E091A205C2
:10128000EE2389F0E150E093A20588E0E89FF001A9
:101290001124ED59FA4F6281738127814681808143
:1012A00091810C949A830C94AE872F923F924F9227
:1012B0005F926F927F928F929F92AF92BF92CF92E6
:1012C000DF92EF92FF920F931F93CF93DF9300D0A3
:1012D0001F92CDB7DEB761E081E00E94F0802091DF
:1012E0003A082B832C83822F8B5F898389E0821BB2
:1012F0008A8388E0782E721A87E0682E621A86E068
:10130000582E521A85E0482E421A84E0382E321A9E
:10131000222E21942B8121115BC0809139088823D2
:1013200099F180918402882359F081E090913908E5
:10133000911180E024E047E158E2622D0F942A35B4
:101340008091A50980933D088B81853009F0A2C06A
:101350001092470880913908853009F45FC1809167
:101360008402882309F43AC211E08091390885305B
:1013700009F010E080913D080F94050700E09C0102
:1013800044EF57E2642D83C08091320810923208F6
:10139000882339F20E943E8980913408882309F419
:1013A000C0CF0F900F900F900F90DF91CF911F91B2
:1013B0000F91FF90EF90DF90CF90BF90AF909F90F4
:1013C0008F907F906F905F904F903F902F900895F7
:1013D0008B818130C1F5809139088130E1F08091B5
:1013E0008402882309F4ACCF11E080913908813060
:1013F00009F010E080917A0290917B020F94AE0682
:1014000061E02C81621B00E09C0141E158E2812FE8
:101410000E94422A95CF8091320810923208882388
:10142000F1F2E12C10E000E027EE33E04AE050E07A
:101430006AE772E081E198E20E94008780913408B7
:10144000882369F2AECF8B81823009F08AC1809106
:101450003908823009F44EC0809184028823D1F08B
:1014600011E080913908823009F010E06091450662
:101470007091460680914706909148060E94477CED
:1014800062E02C81621B00E09C014BE058E2812F5E
:101490000E94422A8091A60980933D089B81963044
:1014A00009F0E6C081E080934708809139088630D2
:1014B00009F4C9C080918402882391F011E08091E1
:1014C0003908863009F010E080913D080F94050737
:1014D00000E09C0144EF57E2652D812F0E94422AD3
:1014E0009B819F5F9B832981291314CF8AE080937E
:1014F000330857CF8091320810923208882309F4BC
:10150000ABCF20E030E04AE754E4609145067091AB
:10151000460680914706909148060F94315920E085
:1015200030E0A9010F94BD5F20E030E04AE754E4C9
:101530000F94BD5F0F9430611F92912C812C8EE42B
:10154000A82E83EBB82E6B0110EDE12E17E0F12EE3
:1015500000E010E028E13CEF4FEF5FEF65E476E05C
:101560008BE098E20E948D860F908091340888234A
:1015700009F472CF16CF809139088330C9F0809179
:101580008402882309F486CF11E0809139088330E2
:1015900009F010E08091ED159091EE150F94AE06D4
:1015A00063E02C81621B00E09C0144E058E22FCFF5
:1015B0008091320810923208882309F30F949F35E6
:1015C000E12C0AEE1CE72CE231E050E040E06DEE49
:1015D00075E184E098E20E940087809134088823B6
:1015E00071F2DFCE8091320810923208882309F41C
:1015F000C4C00F949F35E12C03EB1BEC2CE830E0CA
:1016000050E040E069E878E080E098E20E940087DE
:1016100080913408882309F4B0C0C3CE8091320889
:1016200010923208882309F49ACE0F949F356CE605
:1016300078E784EF97E20F94A937809134088823E4
:1016400009F48DCEAECE80913208109232088823F4
:1016500009F430CF0F949F356CE678E784EF97E27A
:101660000F94A93780913408882309F423CF99CEA9
:101670002B81273099F5809139088730B9F0809116
:101680008402882309F42CCF11E080913908873037
:1016900009F010E080913602909137020F94AE0667
:1016A00000E09C014FEE57E2662D17CF8091320883
:1016B00010923208882319F3E12C09E418E727EE89
:1016C00033E04AE050E066E372E08FEE97E20E947A
:1016D000008780913408882391F263CE8B81883013
:1016E00009F062C0809139088830D9F08091840275
:1016F000882309F4F5CE11E080913908883009F08B
:1017000010E060919D0970919E0980919F099091D0
:10171000A0090E94FE7600E09C0145EE57E2672D8D
:10172000DCCE80913208109232088823F9F26DE9FC
:1017300079E085EE97E20F9463378091340888232F
:10174000A9F22FCE80913208109232088823A1F19D
:1017500089E294E80E941B8480913408882361F117
:1017600020CE8B81833009F406CF843009F0E8CD98
:1017700080913908843009F435CF80918402882320
:1017800009F488CE11E080913908843009F010E026
:101790008091890890918A080F94AE0600E09C0120
:1017A00040E058E2632D33CE9B81993009F098CE0A
:1017B00080913908893031F280918402882309F4BC
:1017C0008FCE81E090913908993009F080E023E0D4
:1017D0004AED57E26A810F942A3582CE8091A6099C
:1017E00080933D087DCE5F926F927F928F929F9201
:1017F000AF92BF92CF92DF92EF92FF920F931F931F
:10180000CF93DF93D1E08091ED159091EE15892B68
:1018100009F4D0E061E081E00E94F080C0913A08D4
:101820008C2E45E0942E9C0EAA24A39484E0F82EDE
:10183000FC1A83E0D82EDC1A82E0C82ECC1A7A2C4F
:101840007C1A6C2E619487E0B82EBC1AC111B9C005
:1018500080913908882309F496C0809184028823F6
:1018600059F081E090913908911180E024E045ED34
:1018700057E2662D0F942A358091A60980933D0882
:10188000C430E9F4A092470880913908843009F403
:1018900048C180918402882391F011E08091390839
:1018A000843009F010E080913D080F94050700E0B6
:1018B0009C014EEB57E26F2D812F0E94422A10E0CF
:1018C00000E035E0E32E5C2E581800933D08CE1161
:1018D0001FC0F801EE0FFF1FEE5DFE4B8591949146
:1018E0009093490880934808809139088C1709F42F
:1018F0002DC180918402882359F081E090913908AC
:101900009E1180E023E044EB57E2652D0F942A35C9
:101910008E2D0F5F1F4F96E0E92E8630B1F6809135
:10192000890890918A08892B19F4DD2309F42EC1C6
:10193000C73009F580913908873009F418C18091C2
:1019400084028823C1F086EB97E89F938F938BEAFC
:1019500097E29F938F93BF9281E0909139089730DF
:1019600009F080E08F930E94E2800F900F900F901B
:101970000F900F900F9088E0D1E0CF5FC91166CF34
:10198000809333080EC08091320810923208882369
:1019900009F463CF0E943E8980913408882309F4BA
:1019A0005CCFDF91CF911F910F91FF90EF90DF906F
:1019B000CF90BF90AF909F908F907F906F905F90EF
:1019C0000895C13009F060C080913908813009F470
:1019D0003FC080918402882309F44ECF11E08091AA
:1019E0003908813009F010E08091ED159091EE15E5
:1019F0000F94AE0600E09C014EEC57E2672D812F5C
:101A00000E94422A8091A50980933D08C33009F0C5
:101A100033CF1092470880913908833009F46CC0A5
:101A200080918402882309F44ACF11E0809139081B
:101A3000833009F010E080913D080F94050700E025
:101A40009C014EEB57E26D2D812F0E94422A14CF4C
:101A50008091320810923208882309F4BACF0F948B
:101A60009F35E12C0CEE1CE72CE231E050E040E029
:101A70006DEE75E18EEC97E20E940087809134084C
:101A8000882309F4A6CF8DCFC23009F0BBCF809157
:101A900039088230B9F080918402882309F4ECCEB1
:101AA00011E080913908823009F010E080918908B6
:101AB00090918A080F94AE0600E09C014AEC57E230
:101AC0006C2D9DCF8091320810923208882319F333
:101AD0000F949F35E12C03EB1BEC2CE830E050E039
:101AE00040E069E878E08AEC97E20E940087809104
:101AF0003408882381F255CF809132081092320841
:101B0000882309F48DCF0F949F356CE678E78EEB30
:101B100097E20F94A93780913408882309F480CF85
:101B200040CF8091320810923208882309F4B1CE58
:101B30000F949F356CE678E78EEB97E20F94A93708
:101B400080913408882309F4A4CE2BCF80913208E9
:101B500010923208882309F4CCCE88EC9DE80E94CC
:101B60001B8480913408882309F4C3CE1ACF809156
:101B7000320810923208882309F4E1CE0E94B68719
:101B800080913408882309F4DACE0BCF87E0F5CEB4
:101B90004F925F926F927F928F929F92AF92BF927D
:101BA000CF92DF92EF92FF920F931F93CF93DF9329
:101BB00000913D0861E081E00E94F080C0913A0808
:101BC00010E0000F111F0E5D1E4B95E0592E5C0EAC
:101BD00021E9E22E27E2F22ED3E0DC1B3EEEC32EFB
:101BE0003CE7D32E43E8A42E47E2B42E82E0782EC1
:101BF0007C1A54EB852E57E2952E81E0682E6C1AE4
:101C00004C2E4194C11137C0809139088823B1F01E
